:100000000C943A080C9489080C9489080C9489087B
:100010000C9489080C9489080C9489080C9489081C
:100020000C9489080C94121B0C9489080C94890870
:100030000C9442360C9489080C9489080C94890815
:100040000C9489080C9489080C94CE170C94890898
:100050000C942E0E0C9489080C94F80D0C948908BD
:100060000C94F51D0C9489080C94AD310C948908FE
:100070000C94518B0C9489080C944D860C9489082F
:100080000C9489080C9489080C948908201E251E5C
:100090002A1E331E4A1E611E711E811EBC1EA82010
:1000A000611E6A1F7B1FAA1FC81FE51F3F209A20E1
:1000B00078220A23C7234724B02460256727C42752
:1000C00031287B28C62813296429C629252ABF2A56
:1000D0005A2B542CCC3100324332B332CB320C3356
:1000E000C3338A348A348A348A348A348A348A34E8
:1000F0008A348A348A348A343F34413446345E3414
:1001000060340A0D426174743A002025642043650E
:100110006C6C7320004C6F772042617474206C65A6
:1001200076656C3A2025642E2564000A0D466F75AD
:100130006E6420424C2D4374726C3A20002564009A
:100140000A0D0A0D21214D495353494E4720424C77
:100150002D4354524C3A2025642121000A0D3D00C4
:100160000A0D43616C2E2070726573737572652081
:1001700073656E736F72004F4B0A0D000A0D466C6B
:10018000696768742D74696D65202575206D696EC9
:100190002020546F74616C3A2575206D696E000AD9
:1001A0000D436F6E74726F6C3A200048656164692C
:1001B0006E67486F6C64004E6F726D616C202841F1
:1001C00043432D4D6F646529000A0D3D0A0D000A59
:1001D0000D4A4554492B2056657273696F6E207322
:1001E000706F6E736F72656420627920466C7969F6
:1001F0006E67686967682E63682C2070726F67612C
:100200006D6D6564206279204D617274696E570A64
:100210000D00416E676C654E69636B2020202020C5
:100220002020416E676C65526F6C6C20202020206E
:1002300020204163634E69636B2020202020202012
:100240002020416363526F6C6C20202020202020EE
:1002500020205961774779726F20202020202020AC
:1002600020204865696768742056616C7565202098
:1002700020204163635A202020202020202020209D
:1002800020204761732020202020202020202020B3
:100290002020436F6D706173732056616C7565200B
:1002A0002020566F6C74616765205B302E31565D7F
:1002B00020205265636569766572204C6576656CB1
:1002C00020204779726F20436F6D70617373202017
:1002D00020204D6F746F722031202020202020209C
:1002E00020204D6F746F722032202020202020208B
:1002F00020204D6F746F722033202020202020207A
:1003000020204D6F746F7220342020202020202068
:1003100020204D6F746F7220352020202020202057
:1003200020204D6F746F7220362020202020202046
:1003300020206E6320616C742073706565642020DA
:100340002020313920202020202020202020202083
:100350002020536572766F2020202020202020202E
:100360002020486F7665726761732020202020204E
:10037000202043757272656E74205B302E31415DB2
:1003800020204361706163697479205B6D41685D11
:100390002020486967687420536574706F696E74B3
:1003A00020204D6F746F72203720202020202020C5
:1003B00020204D6F746F72203820202020202020B4
:1003C0002020436F6D7061737320536574706F6983
:1003D0006E744932432D4572726F722020202020A6
:1003E0002020424C204C696D697420202020202060
:1003F00020204750535F4E69636B2020202020202F
:1004000020204750535F526F6C6C2020202020200A
:10041000202021212120494E434F4D504154494233
:100420004C4520212121002A002E000A0D204441A4
:1004300043206F7220493243204552524F522120AF
:10044000436865636B204932432C203356726566DE
:100450002C2044414320616E6420424C2D43747231
:100460006C005B25695D005B25695D002B204D6993
:100470006B726F4B6F70746572202B0048573A5641
:1004800025642E25642053573A25642E2564256360
:100490000053657474696E673A25642025730048BB
:1004A00061726477617265204572726F7220313AB1
:1004B0002564202121004D697373696E6720424CC9
:1004C0002D4374726C3A25642121004D6978657260
:1004D000204572726F722100493243204552524FBB
:1004E00052212121004865696768743A202025352A
:1004F0006900536574706F696E743A2535690050F0
:10050000726573737572653A253569004F66667357
:1005100065743A202025356900486569676874204C
:10052000636F6E74726F6C0044495341424C454492
:100530000048656967687420636F6E74726F6C0041
:1005400044495341424C4544006163742E20626526
:100550006172696E67004E69636B3A20202020202B
:100560002025356900526F6C6C3A20202020202015
:1005700025356900436F6D706173733A2020202523
:100580003569004B313A25346920204B323A253405
:100590006920004B333A25346920204B343A253406
:1005A0006920004B353A25346920204B363A2534F2
:1005B0006920004B373A25346920204B383A2534DE
:1005C0006920004E693A2534692020526F3A25345B
:1005D00069200047733A253469202047693A253459
:1005E00069200050313A253469202050323A2534B0
:1005F00069200050333A253469202050343A25349C
:100600006920004779726F202D2053656E736F72D9
:10061000004E69636B25346920282533692E2569CE
:100620002900526F6C6C25346920282533692E25EA
:1006300069290047696572253469202825336929AD
:10064000004E69636B2025346920282533692E25E7
:10065000782900526F6C6C20253469202825336975
:100660002E257829005961772020253469202825F6
:10067000336929004E69636B2025346920282533AE
:100680006929282533692900526F6C6C202534694B
:1006900020282533692928253369290059617720C5
:1006A0002025346920282533692928253369290024
:1006B000414343202D2053656E736F72004E696372
:1006C0006B2025346920282533692900526F6C6C12
:1006D00020253469202825336929005A202020202C
:1006E00025346920282533692900566F6C746167A9
:1006F000653A2020202533692E253169560043753F
:100700007272656E743A2020202533692E25316976
:100710004100506F7765723A2020202020253469EF
:1007200057004469736368617267653A20253569CB
:100730006D41680052656365697665720052432DAC
:10074000525353493A202020202534690052432D2A
:100750005175616C6974793A202534690052432DD2
:100760004368616E6E656C733A25346900436F6D42
:10077000706173730048656164696E673A20202573
:1007800035690056616C75653A2020202025356951
:1007900000536F6C6C3A20202020202535690050D2
:1007A0006F7469313A202025336900506F746932C3
:1007B0003A202025336900506F7469333A20202590
:1007C000336900506F7469343A2020253369005032
:1007D0006F7469353A202025336900506F7469368B
:1007E0003A202025336900506F7469373A2020255C
:1007F000336900506F7469383A20202533690053FB
:100800006572766F202000536574706F696E742076
:100810002025336900506F736974696F6E3A202523
:1008200033690052616E67653A2533692D25336956
:100830000045787465726E436F6E74726F6C202021
:10084000004E693A2534692020526F3A25346920D8
:100850000047733A253469202047693A25346920D6
:100860000048693A253469202043663A25346920D6
:1008700000424C2D4374726C204572726F7273206B
:100880000025336420253364202533642025336418
:10089000200025336420253364202533642025334C
:1008A000642000253364202533642025336420250B
:1008B00033642000424C2054656D7065726174751C
:1008C0007265002533692025336920253369202589
:1008D00033692000253369202533692025336920B9
:1008E00025336920002533692025336920253369A4
:1008F000202533692000424C2D4374726C20666FB2
:10090000756E642000202563202020256320202090
:10091000256320202025632000202563202020251A
:1009200063202020256320202025632000202563CC
:100930002020202D2020202D2020202D200031308F
:1009400000313100313200466C696768742D54699A
:100950006D65202000546F74616C3A2535756D69A2
:100960006E004163743A20202535756D696E00284C
:10097000726573657429000A0D47656E657261744E
:10098000696E672064656661756C74205061726180
:100990006D6574657220536574202564000A0D55D9
:1009A00073696E6720506172616D65746572205362
:1009B0006574202564000A0D47656E65726174696F
:1009C0006E672064656661756C74204D6978657228
:1009D000205461626C65000A0D4D697865722D4383
:1009E0006F6E6669673A20272573272028257520B2
:1009F0004D6F746F727329000A0D3D000A0D41435B
:100A000043206E6F742063616C6962726174656407
:100A1000210D0A0000008F001E01AD013B02CA0239
:100A20005803E603740402058F051B06A706330767
:100A3000BE074808D2085B09E3096B0AF20A780B83
:100A4000FD0B810C040D860D070E870E060F840F1B
:100A500000107B10F5106E11E5115B12CF124213DE
:100A6000B31323149214FE146A15D3153B16A11662
:100A700005176717C81727188318DE1837198E1936
:100A8000E319361A871AD61A231B6E1BB61BFD1BD9
:100A9000411C831CC31C001D3C1D751DAB1DE01DAE
:100AA000121E421E6F1E9A1EC31EE91E0D1F2E1F10
:100AB0004D1F691F841F9B1FB01FC31FD31FE11F42
:100AC000EC1FF51FFB1FFF1F002016010008886E9A
:100AD00000020101BF6F010302022270020403033E
:100AE000C070030504045A71040605056873050700
:100AF0000606CB73061607073D74000908086474E0
:100B0000080A0909E075090B0A0AEC760A0C0B0BB6
:100B1000F8770B0D0C0C04790C0E0D0D607E0D0F8B
:100B20000E0E107A0E100F0F1C7B0F1110107E7C12
:100B300010121111547D111312127C7F1214131311
:100B4000F77B131514149C75140015154D810700BF
:100B5000161688802532692E2531695600253364A2
:100B6000256320253033646D005374617475730000
:100B70004552524F523A20253264002534692025CF
:100B800032693A25303269002534696D25630020C9
:100B90004A4554492B2073706F6E736F7265640001
:100BA000627920466C79696E67686967682E636848
:100BB00000542533692025336920253369202533E6
:100BC00069002533692025336920253369202533C1
:100BD00069002532692E25316956002533692E2595
:100BE000316941002533692E253169410025346979
:100BF00057202536696D4148002532756D2F7320C9
:100C00005361743A2564200020203344004E6F461F
:100C100078004447505300486F6D653A2533646D42
:100C2000202533642563004E6F204E61766943743E
:100C3000726C2100492533692025336920253369E9
:100C40002025336900253369202533692025336940
:100C5000202533690043757272656E7473205425C4
:100C600033692E25316941002533692E25316941CB
:100C700020004932432533692533692533692533FB
:100C80006900253369202533692025336920253300
:100C900069002533694E202533695220202B4E00F0
:100CA00025336947202020202B52202D4E202D5205
:100CB000002533693D48472F34202533693D47617E
:100CC000730025632533693D53503125632533690E
:100CD0003D5350330025632533693D53503225631E
:100CE0002533693D535034007377697463686564D4
:100CF000204869676874207600566172696F2077B2
:100D000069746862656570205E0025632533693DFE
:100D100048442025632533693D4841002563253338
:100D2000693D48502025632533693D484D002563C2
:100D30002533693D48562025632533693D485A00CF
:100D400025632533693D48472025632533693D4E9A
:100D5000470025632533693D537450256325336966
:100D60003D5347500025632533693D537444256343
:100D70002533693D4472430025632533693D475956
:100D80005025632533693D4759490025632533695B
:100D90003D47594425632533693D4D61490025632D
:100DA0002533693D4E474725632533693D4E5343FF
:100DB0000025632533693D4E574325632533693D3F
:100DC0004E414C0025632533693D4E502563253344
:100DD000693D4E440025632533693D4E4925632511
:100DE0000020004C6F6F70696E6776616C756520CE
:100DF000253269640025632533693D4C474C2563E2
:100E00002533693D4C48790025632533693D4C54B1
:100E1000680025632533693D4647502563253369BE
:100E20003D4359430025632533693D464E522563B2
:100E30002533693D5550370025632533693D4747C4
:100E40005025632533693D47537400256325336975
:100E50003D47474925632533693D44537400256365
:100E60002533693D4E435425632533693D52435430
:100E70000025632533693D4E435025632533693D85
:100E8000524350004D74657374203C2B76203C2BEC
:100E90005E253369004D6F746F723D2532692053B2
:100EA000703D2532690053455454494E473D253124
:100EB0006920003C202B203E746F53544F524574E0
:100EC0006F20253169004F4B21000A0D7777772E6F
:100ED0004D696B726F4B6F707465722E646520285C
:100EE000632920486953797374656D7320476D6277
:100EF00048000A0D74686520757365206F6620745C
:100F000068697320736F66747761726520697320F6
:100F10006F6E6C79207065726D6974746564200AF7
:100F20000D6F6E206F726967696E616C204D696B21
:100F3000726F4B6F707465722D4861726477617265
:100F400065004143542044534C004A657469207342
:100F50006174656C6C6974005370656B7472756D47
:100F600020736174656C6C697420284C6F772072F3
:100F700065736F6C7574696F6E29005370656B745F
:100F800072756D20736174656C6C697420283230E1
:100F9000343829005370656B7472756D20736174F9
:100FA000656C6C6974004D756C74697369676E610A
:100FB0006C2050504D000A0D52656365697665726C
:100FC0003A2000756E6B6E6F776E2E205573696ECA
:100FD000672050504D2E2E2E006E6F74207375704A
:100FE000706F7274656420627920686172647761E1
:100FF000726521000A0D3D3D3D3D3D3D3D3D3D3D80
:101000003D3D3D3D3D3D3D3D3D3D3D3D3D3D3D3D10
:101010003D3D3D3D3D3D3D3D3D000A0D466C696712
:101020006874436F6E74726F6C0A0D4861726477F6
:101030006172653A25642E25640A0D536F667477D4
:101040006172653A5625642E2564256320000A0DD9
:101050003D3D3D3D3D3D3D3D3D3D3D3D3D3D3D3DC0
:101060003D3D3D3D3D3D3D3D3D3D3D3D3D3D3D3DB0
:101070003D3D3D0011241FBECFEFD0E4DEBFCDBF0C
:1010800011E0A0E0B1E0ECE3FCE101E00BBF02C045
:1010900007900D92AC3FB107D9F718E0ACEFB1E083
:1010A00001C01D92AF3FB107E1F77AEAE2E0F0E05C
:1010B00081E280935700D4907E010894E11CF11CDA
:1010C00020EF37EF41E050E087016FE0DA01C9011E
:1010D0002F5F3F4F4F4F5F4FABBFFC018791F80130
:1010E00081938F01615067FFF1CFF7016EE081912D
:1010F00078277095615067FFFACF8889781729F0B3
:10110000F7E9DF1611F40000FECF0E944A090C94A3
:101110001D8E0C94000080914806E82FFF27EE0FEB
:10112000FF1FEE58F84F808191818D5E9F4F14F024
:1011300010920301808191818A5B9F4FCCF4809152
:1011400003018823A9F481E08093030180918B043B
:101150008F5F80938B04853038F088EE93E0909316
:1011600033028093320204C066E970E00E94EB39DA
:1011700080918B04992790931906809318060895FF
:101180001F93CF93DF93182F882389F082E091E09B
:101190009F938F9383EB94E19F938F93E0915404FB
:1011A000F091550409950F900F900F900F9080913A
:1011B0006B06823308F044C084EF91E00E94D91896
:1011C000EC01112329F0CE010E94E2188823D9F303
:1011D000C2E0D0E026E530E080911E0190911F0131
:1011E0008217930730F02196255D3F4FC730D10518
:1011F00098F380916B069927C89F9001C99F300D85
:10120000D89F300D1124209300011123D9F068ECF0
:1012100070E08C2F0E94EB39DF93CF938AE091E04E
:101220009F938F9383EB94E19F938F93E09154046A
:10123000F091550409958DB79EB706968DBF02C0F3
:1012400080930001112311F1809100016AE00E9456
:10125000708D892F99279F938F93809100010E9411
:10126000708D99279F938F9385E191E09F938F9342
:1012700083EB94E19F938F93E0915404F091550494
:1012800009952DB73EB7285F3F4F2DBFDF91CF9116
:101290001F910895CFEFD0E4DEBFCDBF88249924FD
:1012A00014B815B8B7EEEB2EB3E0FB2E8EEC9FEF23
:1012B000E80EF91EF7FEFACF85E18093020181E87E
:1012C00087B93E9A8FEF88B98BE184B911E015B9DF
:1012D0008EE38AB987E48BB9469A84B7877F84BF47
:1012E000809160008861809360001092600084ECBF
:1012F00099E0909333028093320210922E03109261
:101300002D031092770710927607109230031092F7
:101310002F03109232031092310384EC94E0A0E08A
:10132000B0E08093960190939701A0939801B093B9
:10133000990128980E9442190E9413190E94BB1417
:101340000E94FE350E94861C812F0E9461310E94FE
:10135000B8660E946E820E94848A809102018C305D
:1013600010F4299A01C0299878940E947B308091CA
:101370007A02826080937A0210927D020E94164562
:1013800084EF91E00E94D9187C0180917A0280FD5F
:1013900005C0C7010E94E2188823B9F38BE291E0EF
:1013A0009F938F93A3EBAA2EA4E1BA2EBF92AF9284
:1013B000E0915404F0915504099580EA9FE00E9461
:1013C000D9187C0100E010E00F900F900F900F9063
:1013D000C4E1D7E0F8ECCF2EF6E0DF2E0E941645F0
:1013E00080917A0280FD05C0C7010E94E21888231F
:1013F000B9F3F60180811816A4F40BC00E941645BB
:1014000080917A0280FD05C0C7010E94E2188823FE
:10141000B9F3C7010E94E218882319F48881882350
:101420006CF7888187FF1AC00F5F1F4F1F930F93C0
:10143000015010408DE391E09F938F93BF92AF9244
:10144000E0915404F091550409958091FF018F5F5C
:101450008093FF018DB79EB706968DBF0F5F1F4F1C
:10146000E4E0F0E0CE0EDF1E28960C30110508F403
:10147000B5CF00E010E0C1E1D7E0E8ECEE2EE6E009
:10148000FE2E8B8187FD1EC0F70180811816D4F4D3
:101490000F5F1F4F1F930F930150104080E491E0A6
:1014A0009F938F9383EB94E19F938F93E0915404E8
:1014B000F0915504099582E0809330028DB79EB774
:1014C00006968DBF8B8180788B830F5F1F4FE4E082
:1014D000F0E0EE0EFF1E28960C30110590F28CE520
:1014E00091E09F938F93C3EBD4E1DF93CF93E0918F
:1014F0005404F09155040995909146068091FF019E
:101500000F900F900F900F90981728F4809171040E
:1015100080618093710480E691E09F938F93DF93C5
:10152000CF93E0915404F0915504099588EE93E02F
:101530000E94D9187C010E948C1C0F900F900F9074
:101540000F90C7010E94E2188823D9F387E791E042
:101550009F938F93DF93CF93E0915404F0915504C0
:10156000099580E00E94AD3A809102010F900F90A2
:101570000F900F908A3011F0843110F0289801C03C
:10158000289A80ED97E0909333028093320285E5AC
:1015900080938D048EE090E00E94B02E9927182F42
:1015A00000278FE090E00E94B02E080F111D1093CD
:1015B0000502009304028AE090E00E94B02E992771
:1015C000182F00278BE090E00E94B02E080F111D0D
:1015D00010930302009302020F5F1F4F39F08091B6
:1015E0000402909105028F5F9F4F41F41092050213
:1015F00010920402109203021092020280910202E1
:10160000909103029F938F93809104029091050221
:101610009F938F938CE791E09F938F93DF93CF936A
:10162000E0915404F091550409958DB79EB7089642
:101630008DBF8FE991E09F938F93DF93CF93E091DC
:101640005404F09155040995809154060F900F9021
:101650000F900F90E0915404F091550482FF07C061
:101660008BEA91E09F938F93DF93CF9308C087EB32
:1016700091E09F938F9383EB94E19F938F930995D0
:101680000F900F900F900F900E94EF2188E893E148
:10169000909393018093920181E080938C040E9447
:1016A000C00880916E060E94EA8989EC91E09F93C0
:1016B0008F93DF93CF93E0915404F09155040995F3
:1016C00080ED97E00E94D9187C018AEF90E00E949B
:1016D000D9186C0183E08093F0050F900F900F9064
:1016E0000F908FEC91E09F938F93DF93CF93E091D6
:1016F0005404F091550409951092FE010F900F903B
:101700000F900F90809108028111FFCFC6010E94B7
:10171000E2188823D1F084E690E00E94D9186C0189
:101720000E94408B8091FE01882329F08091FD0169
:101730008F5F8093FD019091FD018091FC019817CE
:1017400021F41092FD011092FE018091360288234F
:1017500009F446C280911001882309F441C2109215
:10176000360280918B04882319F00E948B0802C0F6
:101770000E9417480E941645209102012A3011F05C
:10178000243110F0289801C0289A80913303909159
:101790007104882339F0809133038150809333039F
:1017A000977F0AC080916F00806280936F001092D3
:1017B0007307109272079860909371048091920160
:1017C000909193010197909393018093920180915E
:1017D000920190919301892B21F080917B028823C3
:1017E000C9F18091920190919301892BD9F40E94C3
:1017F0008B3185E090E090939301809392018091EA
:101800002A0690912B06019690932B0680932A0628
:10181000809171048160809371048091F1058260F0
:101820008093F10580910801909109018F5F9F4F8E
:1018300019F580912A038823F9F080E197E29093CB
:1018400033028093320280E890E090930901809304
:10185000080112C02A3011F0243110F0289801C07C
:10186000289A8091320290913302892B29F4809139
:1018700071048E7F8093710480913602882309F071
:10188000AFC180910E01882311F00E9459190E9466
:10189000FE140E947E10C7010E94E218882309F4FA
:1018A0002CC184E190E0E80EF91E80917B029091BA
:1018B0007104882339F09260909371048091F1054E
:1018C00082600CC09D7F90937104809192019091F1
:1018D0009301079728F08091F1058D7F8093F105A2
:1018E0008091920190919301079728F08091710463
:1018F0008E7F8093710480910501882321F08150AF
:101900008093050125C080939704109204031092E0
:10191000030310920203109201031092000310922D
:10192000FF0280910801909109018F5F9F4F81F420
:1019300080913303882361F488E99AE3909333021A
:101940008093320280E09CE090930901809308012B
:101950008091F201893C48F081508093F20180919E
:1019600071048B7F8093710430C080915E0888235E
:10197000E1F080917104846080937104809108018A
:10198000909109018F5F9F4F81F480912A038823F2
:1019900061F088E99AE3909333028093320280E009
:1019A00098EA90930901809308011092170410920D
:1019B000160410921504109214048FEF9FEF909369
:1019C0008E0880938D081092F20180910001282FDB
:1019D000332780911E0190911F0182179307CCF449
:1019E0008091F80280628093F802809108019091C2
:1019F00009018F5F9F4FC1F480E797E19093330215
:101A00008093320280E093E0909309018093080173
:101A10000BC08091320290913302892B29F480917E
:101A2000F8028F7D8093F8020E943E6B84E08093E1
:101A3000310280912A03882329F45AEA852E55E041
:101A4000952E12C0809107028F5F80930702813329
:101A500059F41092070280910002909101020196C0
:101A600090930102809300020894811C911C82E7EC
:101A700088168BE0980609F040C0882499242091AC
:101A80000402309105022F5F3F4F309305022093EF
:101A90000402809102029091030201969093030246
:101AA00080930202832F9927682F8EE090E00E9496
:101AB000B82E80910402909105029070682F8FE0FB
:101AC00090E00E94B82E8091020290910302892F2B
:101AD0009927682F8AE090E00E94B82E8091020238
:101AE000909103029070682F8BE090E00E94B82ED6
:101AF00084E190E00E94D9187C0180910603883C23
:101B000008F46AC080910A038A3018F48AE080934E
:101B10000A0300919E0310919F031093A103009369
:101B2000A0038091450890914608A0914708B09184
:101B30004808209196013091970140919801509169
:101B40009901BC01CD010E94C58DDA01C901209126
:101B50000A03332744275527BC01CD010E94C58DB8
:101B600030939F0320939E03201B310BC9010197E3
:101B7000029738F09FEF2E3F390719F02F5F3F4F44
:101B8000B1F480910602882339F581E080939B03AC
:101B9000809102018A3011F0843110F0289A01C03E
:101BA0002898429A809109038093060215C090916B
:101BB000060280910803891750F042988091020133
:101BC0008A3011F0843110F0289801C0289A9923A6
:101BD00019F09150909306020E948C6B0E948582AE
:101BE00080913102882309F08DCD0E94D9668ACD7B
:101BF0001F920F920FB60F9211248F939F93EF9322
:101C0000FF93809107018823E1F480912202909153
:101C1000230201969093230280932202FC01EA5B47
:101C2000FA4FE081ED3019F08A3A910539F41092BB
:101C300023021092220281E080930701E093C60004
:101C400004C01092230210922202FF91EF919F9103
:101C50008F910F900FBE0F901F9018951F920F92AB
:101C60000FB60F9211242F933F934F935F936F936F
:101C70007F938F939F93AF93BF93CF93EF93FF93F4
:101C800090E080910802813029F48091C600809311
:101C9000CE00CCC080910802823029F48091C60029
:101CA00080939A04C3C08091C60080931A02509119
:101CB00028025A3A10F09093290280911A028D302E
:101CC00009F065C080912902823009F060C09093CC
:101CD0002902852F992786569B4FFC013297408118
:101CE0002091240230912502241B3109DC01119737
:101CF0008C91281B3109C9019F7090932502809314
:101D0000240246E0969587954A95E1F7982F935CD3
:101D1000909326022F733070235C209327028081DA
:101D2000981729F48C91281711F491E006C090E0DF
:101D3000809117028F5F80931702C0911902CC2304
:101D400009F074C0992309F471C081E080931902ED
:101D5000580F509316025150E52FFF27E656FB4FC0
:101D60008DE0808380919C04823509F05FC00E94E1
:101D7000EF2188E190E02CE00FB6F894A8958093CD
:101D800060000FBE20936000C09330024FC02091CE
:101D90002902822F992781309105F9F0823091052F
:101DA0001CF4892B21F040C0029711F13DC08091B5
:101DB0001A02833239F480911902882319F481E0E0
:101DC0008093290280911A0280939A0481E0809383
:101DD000280280911A02992722C02F5F209329029E
:101DE000E52FFF27E656FB4F80911A02808309C03A
:101DF000E52FFF27E656FB4F80911A0280835A3A5F
:101E000020F45F5F5093280202C0109229022091B3
:101E10001A028091240290912502820F911D9093C5
:101E200025028093240202C010922902FF91EF91B3
:101E3000CF91BF91AF919F918F917F916F915F9162
:101E40004F913F912F910F900FBE0F901F901895BB
:101E5000AC01A0E0B0E09D01A817B90748F4E6E4A2
:101E6000F5E08191280F311D1196A417B507C8F32D
:101E70003F70FD01EA5BFA4FC90156E096958795E0
:101E80005A95E1F7835C80831196FD01EA5BFA4F76
:101E90002F733070822F835C8083A95BBA4F8DE0F3
:101EA0008C9310920701809146058093C600089597
:101EB000A0E0B0E0EEE5FFE00C94E98D2C859D8577
:101EC0000E85BB2483E2809346059F599093470576
:101ED0002093480533E0E32EF12C002309F49EC043
:101EE000CF84D888BE016D5E7F4FA989BA89015021
:101EF000109709F493C01097B9F0F601EB0DF11D9E
:101F0000B3949081119791F4002349F1FB016E5F26
:101F10007F4FDB01C080D1806E5F7F4F0D90BC9101
:101F2000A02DBB24015002C090E019C01097B9F059
:101F3000F601EB0DF11DB3944081119791F400234C
:101F400041F1FB016E5F7F4FDB01C080D1806E5F8E
:101F50007F4F0D90BC91A02DBB24015002C040E0EA
:101F600018C01097B1F0F601EB0DF11DB39410817C
:101F7000119781F4002371F0FB013296DB01CD90C3
:101F8000DC90BF016E5F7F4FA081B181BB24015007
:101F900001C010E0F701EA5BFA4F892F869586951C
:101FA000835C80830894E11CF11CF701EA5BFA4F23
:101FB000892F99278370907024E0880F991F2A95A4
:101FC000E1F755279A0194E0369527959A95E1F720
:101FD000822B835C80830894E11CF11CF701EA5B8F
:101FE000FA4F4F705070440F551F440F551F812FEB
:101FF000992726E0969587952A95E1F7842B835CAF
:1020000080830894E11CF11CF701EA5BFA4F1F730F
:10201000135C10830894E11CF11C6ACFC7010E9475
:10202000280FE9E00C94058EA3E07A2F4091160268
:102030004650442309F458C0E72FFF27E656FB4FCC
:1020400080818D537F5FE72FFF27E656FB4F20816E
:102050002D537F5FE72FFF27E656FB4F30813D531F
:102060007F5FE72FFF27E656FB4F60816D537F5F51
:102070009927880F991F880F991F522F52955F70CB
:10208000582B822F99278F709070F4E0880F991F3A
:10209000FA95E1F7232F26952695282B832F99274C
:1020A00083709070E6E0880F991FEA95E1F7682B3E
:1020B00041504F3FC9F0EA2FFF27E656FB4F5083B0
:1020C000AF5F41504F3F81F0EA2FFF27E656FB4FAD
:1020D0002083AF5F41504F3F39F0EA2FFF27E6568C
:1020E000FB4F6083AF5FA5CF8DE994E0909315021D
:1020F00080931402A350A09313020895A2E0B0E0CD
:10210000E4E8F0E10C94EF8D80911902882309F442
:1021100026C40E94141080919B04823609F02AC3C1
:1021200080919C0499278037910509F4C1C08137BB
:102130009105C4F48A36910509F492C28B36910553
:1021400044F48B34910571F18636910509F471C11F
:1021500011C38D36910509F47BC08E36910509F4C3
:102160005FC008C384379105D1F1853791054CF4E0
:102170008137910509F4A3C08337910509F4F1C0B3
:10218000F9C28737910509F42DC2883791052CF4DF
:102190008537910509F4E9C1EDC28937910509F444
:1021A0007FC1E8C2E0911402F09115028081918113
:1021B0009093DF018093DE0120914303309144032B
:1021C000821B930B845E9D4F68E671E00E94908DA8
:1021D000845B90409093420380934103CBC28091F3
:1021E0001602A0911402B0911502853140F080E1F1
:1021F000E5E7F4E00D9001928A95E1F70DC08D912D
:102200009D910D90BC91A02D8093750490937604C0
:10221000A0937704B093780480EF809311024BC0B1
:10222000809107018823E1F38DE490E09F938F93E1
:102230008BEB96E09F938F9381E08F938F938EE447
:102240008F930E94580F8DB79EB707968DBF92C28D
:10225000A0911402B09115021C91113081F48DE40B
:10226000EBEBF6E00D9001928A95E1F70E94B82F12
:102270001983809171048F7E8093710401C019824B
:10228000809107018823E1F381E090E09F938F9391
:10229000CE0101969F938F9381E08F938F938DE46E
:1022A0008F930E94580FADB7BEB71796ADBF62C2ED
:1022B00081E080931C028FEF809305015BC2E09167
:1022C0001402F0911502E0818E2F8A508A3058F462
:1022D0008983882311F481E003C0863010F085E003
:1022E000898361E00EC08E2F84518A3070F4898317
:1022F000882311F481E003C0863010F085E08983E3
:1023000060E089810E94383012C0E983EF3F19F400
:102310000E941B3089838981882311F481E003C0E6
:10232000863010F085E0898389810E94CE2E8091CD
:1023300007018823E1F383E790E09F938F9387E47D
:1023400096E09F938F9381E090E09F938F93CE01CF
:1023500001969F938F9382E08F9381E08F9381E525
:1023600077C12091140230911502D9018C918150CE
:10237000853008F045C0F9018181853509F040C0FC
:1023800080912A038823E1F52F5F3F4F83E7E7E43D
:10239000F6E0D9010D9001928A95E1F7F901829159
:1023A0000E94372F809188069927AA27BB27BC0156
:1023B000CD0124EC39E040E050E00E94518DDC0179
:1023C000CB018093D6019093D701A093D801B0930D
:1023D000D901809189069927AA27BB27BC01CD0185
:1023E0000E94518DDC01CB018093D2019093D301E7
:1023F000A093D401B093D5010E941B30898301C002
:102400001982809107018823E1F381E090E09F9396
:102410008F93CE0101969F938F9381E08F938F933B
:1024200083E58F930E94580F8DB79EB707968DBF97
:1024300026C0E0911402F0911502E0818E2F8150A8
:10244000853018F48E2F0E94CE2E0E941B30898377
:10245000809107018823E1F381E090E09F938F93BF
:10246000CE0101969F938F9381E08F938F9386E4A3
:102470008F930E94580FADB7BEB71796ADBF80912E
:102480002A03882329F46EE670E089810E94EB39E3
:1024900080E00E94C00880916E060E94EA896AC1AD
:1024A000E0911402F09115028081992787FD9095A3
:1024B00090938D0780938C078181992787FD909554
:1024C00090938F0780938E078281992787FD90953F
:1024D00090939107809390078381992787FD90952A
:1024E00090939307809392078481992787FD909515
:1024F00090939507809394078581992787FD909500
:1025000090939707809396078681992787FD9095EA
:1025100090939907809398078781992787FD9095D5
:1025200090939B0780939A078085992787FD9095C4
:1025300090939D0780939C078185992787FD9095AF
:1025400090939F0780939E078285992787FD90959A
:102550009093A1078093A0078385992787FD909585
:102560009093A3078093A20705C1E0911402F09114
:10257000150280810E9457358A83882319F481E0EF
:10258000898301C01982809107018823E1F388E0E3
:1025900090E09F938F9389E097E09F938F9321E042
:1025A00030E03F932F9380911402909115029F93F6
:1025B0008F933F932F93CE0102969F938F933F93D8
:1025C0002F93CE01820F931F9F938F9384E08F935D
:1025D00081E08F9385E58F930E94580FEDB7FEB78A
:1025E00073963CC080911302893008F4C3C02091D7
:1025F0001402309115022F5F3F4F88E0A9E0B7E049
:10260000F90101900D928A95E1F7D9018E910E940E
:10261000AD348A83882319F481E0898301C019824B
:10262000809107018823E1F321E030E03F932F936D
:10263000CE0102969F938F933F932F93CE01820FEB
:10264000931F9F938F9382E08F9381E08F9387E511
:102650008F930E94580FEDB7FEB73B96EDBF8AC02F
:102660000E949D898983823019F0843009F082C0EC
:10267000F8948091C1008F738093C1008091C9004C
:102680008F738093C9008091C100877E8093C100C1
:102690008091C900877E8093C9008091C80087FF20
:1026A00003C08091CE00F9CF8091C00087FF03C0A6
:1026B0008091C600F9CFE0911402F091150280815B
:1026C000882359F581E0809308021092CD0080E4C0
:1026D00090E08093CC008091CD008093C5008091E4
:1026E000CC008093C4008091CA008F7D8093CA0083
:1026F0008091CA008F7E8093CA008091C9008B7F31
:102700008093C9008091CA0084608093CA00809140
:10271000CA0082608093CA0003C082E080930802EE
:102720008091CA00877F8093CA008091C200877F12
:102730008093C2008091C9008E7F8093C9008091F0
:10274000C10088618093C1008091C9008861809335
:10275000C9008091C10080688093C1008091C90048
:1027600080688093C90010926E0010926F001092E2
:102770007000789480919C0499278336910509F420
:102780009CC0843691056CF48136910509F475C0BE
:10279000823691050CF07EC08B34910509F450C04F
:1027A000D6C08736910509F4CFC0883691052CF440
:1027B0008436910509F4A6C0CAC08437910529F072
:1027C0008637910509F4BCC0C2C080911602A09161
:1027D0001402B0911502803140F080E1E5E7F4E0A9
:1027E0000D9001928A95E1F70DC08D919D910D900C
:1027F000BC91A02D8093750490937604A0937704E8
:10280000B0937804809107018823E1F31F928091AF
:1028100004018F9384E58F930E94580F8AEF809371
:1028200011028FEF8093050180EA9FE00E94D91882
:1028300090930A02809309020F900F900F9087C027
:10284000E0911402F0911502808191819093DF0153
:102850008093DE012091430330914403821B930B4C
:10286000845E9D4F68E671E00E94908D845B90408D
:1028700090934203809341036AC0E0911402F09167
:102880001502808180930601803298F08FE1809359
:1028900006010FC0A0911402B09115028BE0EDE883
:1028A000F4E00D9001928A95E1F78091960480936F
:1028B00032068FEF809305014AC080910D029091FE
:1028C0000E02892B89F4E0911402F0911502E08147
:1028D000EE2351F08AE0E89FC00111240E94D9182C
:1028E0009093680480936704E0911402F0911502BC
:1028F00090818AE0989FC001112490930E028093EA
:102900000D0215C08FEF80930501E0911402F09144
:10291000150290818AE0989FC001112490931002C3
:1029200080930F02892B19F081E080931E0280EAC8
:102930009FE00E94D91890930A028093090207C071
:1029400081E080931D0203C081E0809321021092F8
:102950001902109215021092140210921302E3E071
:10296000CE5F0C940B8E982F8091C00085FFFCCF1A
:102970009093C60008950F931F9388E18093C10040
:102980008091C00082608093C0008091C100806807
:102990008093C1008091C10080648093C10000E0F9
:1029A00010E00093C5008AE290E08093C40080911B
:1029B0000F02909110020E94D91890936A0480939C
:1029C00069048CED90E00E94D9189093990480934B
:1029D000980410926B0484E580936C0410926F0449
:1029E0008BE080936D0410926E0410931502009397
:1029F0001402109213021F910F910895A0E1B0E00C
:102A0000E4E0F5E10C94EC8D80910701882309F452
:102A1000C1C28091090290910A020E94E2188823A3
:102A200061F010920C0210920B02109210021092A0
:102A30000F0210920E0210920D0280910B029091E3
:102A40000C02892B41F080914405909145050E942C
:102A5000E218882329F480911F02882309F460C0BA
:102A600080910701882309F45BC080911B0201E279
:102A700011E08430A8F00E94032280E590E09F934B
:102A80008F931F930F9381E08F938F9388E48F939D
:102A90000E94580F2DB73EB7295F3F4F2DBF34C05E
:102AA0001092750282E194E09F938F9388EF91E2F8
:102AB0009F938F93E0915404F0915504099584E11C
:102AC00090E09F938F931F930F9381E090E09F93EB
:102AD0008F938BE192E09F938F9382E08F9381E0BD
:102AE0008F9388E48F930E94580F80911B02982F38
:102AF0008F5F80931B022DB73EB7215F3F4F2DBFE5
:102B0000943010F010921B0280910B0290910C02F5
:102B10000E94D918909345058093440510921F0296
:102B200080912002882351F180910701882331F19F
:102B30000E94032280E590E09F938F9381E291E0D1
:102B40009F938F9321E030E03F932F9380E291E0B9
:102B50009F938F933F932F9384E792E09F938F935C
:102B600083E08F9381E08F938CE48F930E94580FC2
:102B7000109220028DB79EB70F968DBF80911D02D7
:102B80008823D1F0809107018823B1F08AE090E09A
:102B90009F938F938BE694E09F938F9381E08F9325
:102BA0008F9386E58F930E94580F10921D022DB7C8
:102BB0003EB7295F3F4F2DBF809121028823D9F076
:102BC000809107018823B9F08BE090E09F938F9369
:102BD0008DE894E09F938F9381E08F93809104011F
:102BE0008F9387E48F930E94580F109221028DB724
:102BF0009EB707968DBF80919804909199040E948A
:102C0000E218882309F461C080910701882309F440
:102C10005CC0809163069927880F991F880F991FC0
:102C20007C010027F7FC0095102F80918103909183
:102C30008203A0918303B0918403BC01CD01A8015C
:102C400097010E94C58D309386042093850480915E
:102C5000790390917A03A0917B03B0917C03BC012E
:102C6000CD01A80197010E94C58D3093880420935F
:102C7000870480910D038093890480910C038093D5
:102C80008A0488E090E09F938F9385E894E09F9377
:102C90008F9381E08F9383E08F938BE68F930E94D5
:102CA000580F80918B042DB73EB7295F3F4F2DBF42
:102CB000853018F086E080938B0483E690E00E94D4
:102CC000D918909399048093980480910F02909161
:102CD0001002892B41F08091690490916A040E944E
:102CE000E218882321F480911E02882339F1809113
:102CF0000701882319F10E94A23882E490E09F9393
:102D00008F9380EF95E09F938F9381E08F938F93C4
:102D100084E48F930E94580F10921E028DB79EB7C5
:102D200007968DBF80910F0290911002009731F0AD
:102D30000E94D91890936A048093690480910D02CF
:102D400090910E02892B09F4B8C08091670490918C
:102D500068040E94E218882309F4AFC0809107013B
:102D6000882309F4AAC0809163069927880F991FC8
:102D7000880F991F7C010027F7FC0095102F809188
:102D8000810390918203A0918303B0918403BC01DD
:102D9000CD01A80197010E94C58D30935A0420935C
:102DA00059048091790390917A03A0917B03B091AB
:102DB0007C03BC01CD01A80197010E94C58D309311
:102DC0005C0420935B0420914508309146084091B3
:102DD000470850914808DA01C90163E0880F991F3C
:102DE000AA1FBB1F6A95D1F7820F931FA41FB51F9F
:102DF000820F931FA41FB51F209196013091970158
:102E00004091980150919901BC01CD010E94C58D5E
:102E100030935E0420935D0480914D0390914E03A6
:102E2000A0914F03B091500339E0B595A7959795C0
:102E300087953A95D1F780935F04809149039091EB
:102E40004A03A0914B03B0914C0329E0B595A79597
:102E5000979587952A95D1F78093600480915103C7
:102E600090915203A0915303B091540309E0B5959A
:102E7000A795979587950A95D1F7809361048EE081
:102E800090E09F938F9389E594E09F938F9381E0E7
:102E90008F938F9383E48F930E94580F80910D023C
:102EA00090910E020E94D918909368048093670451
:102EB0002DB73EB7295F3F4F2DBF809106018F3F51
:102EC00071F1992714E0880F991F1A95E1F78E5E2A
:102ED0009D4F40E150E0BC01CE0101960E94A48BC1
:102EE00080E190E09F938F93CE0101969F938F9303
:102EF00081E090E09F938F9386E091E09F938F9382
:102F000082E08F9381E08F9381E48F930E94580F2A
:102F10008FEF809306018DB79EB70B968DBF809182
:102F200032068823D1F0809107018823B1F081E037
:102F300090E09F938F9382E396E09F938F9381E03D
:102F40008F938F9382E48F930E94580F10923206D2
:102F50002DB73EB7295F3F4F2DBF80911C028823BC
:102F6000C9F0809107018823A9F084E390E09F9342
:102F70008F9382E797E09F938F9381E08F938F9356
:102F800080E58F930E94580F10921C028DB79EB758
:102F900007968DBFE6E0C05F0C94088E1F920F92DB
:102FA0000FB60F9211242F933F935F936F937F93EC
:102FB0008F939F93AF93BF93EF93FF9320E0809104
:102FC0003102882329F080913102815080933102AF
:102FD00080913004882319F08150809330048091CF
:102FE00039028150809339028F3F09F05BC089E03C
:102FF0008093390280913702909138020196909324
:1030000038028093370280910F018F5F8170809327
:103010000F01882319F481E080933602349903C0AC
:1030200081E080933A028091320290913302892BA1
:1030300021F180913202909133020B9750F08091F0
:103040003202909133020A979093330280933202B6
:1030500004C0109233021092320280913202909199
:103060003302209108013091090182239323892B97
:1030700011F021E008C020E006C08FEF9FEF909391
:1030800009018093080180910201222331F08A30E6
:1030900011F45A9A07C0479A05C08A3011F45A9819
:1030A00001C0479880913A02882309F472C02091A8
:1030B000F201222309F06DC08091540683FF69C09C
:1030C00086B19927FC01E071F07084FF14C08091F3
:1030D0003402909135020196909335028093340228
:1030E0008091340290913502895E934008F451C07A
:1030F00020933A024EC08091340290913502892B80
:1031000009F443C080913402909135028A5691406F
:10311000E0F5809134029091350269E270E00E94FE
:103120007C8D8091340290913502860F971F909389
:1031300035028093340280913402909135020B97CE
:1031400050F080913402909135020A979093DF01FC
:103150008093DE0104C0F093DF01E093DE018091F3
:10316000DE019091DF012091430330914403821BE3
:10317000930B845E9D4F68E671E00E94908D845BA6
:103180009040909342038093410310923502109235
:103190003402FF91EF91BF91AF919F918F917F91F9
:1031A0006F915F913F912F910F900FBE0F901F90E5
:1031B00018952091370230913802280F391FC90124
:1031C000019608952091370230913802821B930BAB
:1031D000892F99278695807490700895CF93DF93F7
:1031E0000E94D918EC01CE010E94E2188823D9F37D
:1031F000DF91CF910895CF93DF930E94D918EC010E
:1032000009C080911001882329F0909310018FEC60
:1032100080937A00CE010E94E218982F882389F3C8
:10322000DF91CF9108959FB7F8945F983E9A469AA0
:103230008091B0008F708093B0008091B000836067
:103240008093B0008091B1008B738093B100809126
:10325000B1008B608093B1001092B2008FEF809329
:10326000B3008091B00080688093B00080917000BE
:103270008A7F8093700080917000826080937000DC
:103280009FBF08958AE090E00E94D9189093400271
:1032900080933F0282E085BD83EA84BD17BC84EB46
:1032A00088BD86E086BD80916E00816080936E004F
:1032B0000895A0E0B0E0EFE5F9E10C94EB8D80918A
:1032C0007E06E82FFF27E456FE4F9681D08080913E
:1032D0000E01A92FBB27A7FDB095CB2FDB2F813087
:1032E00009F0DDC020918103309182034091830376
:1032F00050918403BD01CE010E94518D97FF04C0FF
:1033000061587F4F8F4F9F4F7B018C01F7E01595E0
:103310000795F794E794FA95D1F78D2D992787FDB6
:103320009095A92FB92F2091790330917A0340917C
:103330007B0350917C03BC01CD010E94518D97FF0E
:1033400004C061587F4F8F4F9F4FE7E09595879559
:1033500077956795EA95D1F7F801E701C61BD70B7A
:10336000E80BF90B20911E0430911F04C90153E0B2
:10337000880F991F5A95E1F7821B930BAA2797FD97
:10338000A095BA2FC81BD90BEA0BFB0B80917506D1
:103390009927AA27BB27BC01CD019E01AF010E943E
:1033A000518D97FF04C061507E4F8F4F9F4FFC019E
:1033B000EB0149E0F595E795D795C7954A95D1F783
:1033C0008091C101992736E0880F991F3A95E1F75E
:1033D00040910C0150910D0120917D063327841BF3
:1033E000950BB9010E94908D80910C0190910D0177
:1033F000860F971F90930D0180930C0180910C0113
:1034000090910D0197FD0F9624E0959587952A954B
:10341000E1F790932D0280932C028091AC0680FFFF
:1034200007C080912C0290912D028C0F9D1F06C029
:1034300080912C0290912D028C1B9D0B90932D025C
:1034400080932C0280917606282F3327220F331F7A
:10345000220F331F80912C0290912D028217930727
:103460007CF080917706282F3327220F331F220FFD
:10347000331F80912C0290912D022817390724F4D4
:1034800030932D0220932C0280910201843108F4A4
:10349000C2C080910E018F5F80930E01BEC020914B
:1034A000790330917A0340917B0350917C03BD01F5
:1034B000CE010E94518D97FF04C061587F4F8F4FFE
:1034C0009F4F7B018C01C7E015950795F794E79412
:1034D000CA95D1F78D2D992787FD9095A92FB92FE2
:1034E00020918103309182034091830350918403A2
:1034F000BC01CD010E94518D9B01AC0197FF04C01E
:1035000021583F4F4F4F5F4FB7E05595479537953F
:103510002795BA95D1F72E0D3F1D401F511F809161
:1035200079069927AA27BB27BC01CD010E94518D9E
:1035300097FF04C061507E4F8F4F9F4FFC01EB01FE
:10354000A9E0F595E795D795C795AA95D1F780910C
:10355000C001992776E0880F991F7A95E1F740918D
:103560000A0150910B0120917D063327841B950B96
:10357000B9010E94908D80910A0190910B01860FF4
:10358000971F90930B0180930A0180910A019091FB
:103590000B0197FD0F9664E0959587956A95E1F785
:1035A00090932B0280932A028091AC0681FF07C082
:1035B00080912A0290912B028C0F9D1F06C0809152
:1035C0002A0290912B028C1B9D0B90932B028093CF
:1035D0002A0280917A06282F3327220F331F220FC9
:1035E000331F80912A0290912B02821793077CF05F
:1035F00080917B06282F3327220F331F220F331F82
:1036000080912A0290912B022817390724F43093D5
:103610002B0220932A0210920E01E7E0CDB7DEB70D
:103620000C94078E1F920F920FB60F9211242F93B6
:103630003F934F935F938F939F93EF93FF9380916B
:10364000020190913B02843108F04CC0992309F0AB
:103650001CC18091B00086FF24C08091B0008F7B98
:103660008093B00080912C0290912D0287559E4F3F
:1036700090932F0280932E0225E08D3D920718F043
:103680008CED95E005C08757914030F487E791E0D5
:1036900090932F0280932E0280912E0290912F0200
:1036A000BAC08091B00080648093B00080917C06A5
:1036B000282F33278DED96E0289FA001299F500DDC
:1036C000389F500D1124CA0120913C0230913D02D7
:1036D000821B930B90932F0280932E0281E08093A4
:1036E0000E01D0C0992309F0D0C08091B00086FFB0
:1036F00097C08091B0008F7B8093B000E0913E0234
:10370000EE23F1F480917C06282F33278DED96E08F
:10371000289FA001299F500D389F500D1124CA01E8
:1037200020913C0230913D02821B930B90932F021B
:1037300080932E0210923D0210923C02469AA2C043
:1037400089EA93E090932F0280932E028E2F99277F
:1037500083309105D9F08430910534F4813091059E
:1037600049F0029761F020C08430910591F00597EF
:1037700099F01AC080912C0290912D0204C0809182
:103780002A0290912B0287559E4F1DC080910908F7
:1037900005C08091E00702C0809114089927880F26
:1037A000991F880F991FEFCFFF27EE0FFF1FEE58CD
:1037B000F84F20813181220F331F80912E0290918A
:1037C0002F02820F931F90932F0280932E028091DD
:1037D0002E0290912F0255E08D3D950718F08CED4B
:1037E00095E005C08757914030F487E791E09093CA
:1037F0002F0280932E0220912E0230912F022C5BFB
:10380000304030932F0220932E0280913C02909101
:103810003D02820F931F90933D0280933C0232C081
:103820008091B00080648093B0008CEB90E0909326
:103830002F0280932E0280913C0290913D0284548D
:103840009F4F90933D0280933C02809130028823E9
:1038500021F080913303833320F480913002823051
:1038600011F4469801C0469A80913E028F5F809382
:103870003E0290917C06981728F481E080930E0117
:1038800010923E0281E080933B0220912E02309103
:103890002F0241E02F37340730F08FEF8093B300D1
:1038A0002F5F30400FC02F3F3105C9F0C0F0A90194
:1038B0004F5F50404F37510550F480E88093B3007C
:1038C0002058304030932F0220932E0212C08FEFE9
:1038D0008093B30050932F0240932E020AC0809130
:1038E0002E028093B30010922F0210922E0210929B
:1038F0003B02FF91EF919F918F915F914F913F918B
:103900002F910F900FBE0F901F90189510927C0072
:103910008FEC80937A000895CF93DF931092450245
:1039200086E987BD83E090E00E94B02EC82F863ED6
:1039300008F4C65FC8BD84E690E00E94FB18809141
:103940001401909115018152934010F0C0EF02C014
:10395000C530F8F0C8BD82E390E00E94FB1887E212
:1039600094E09F938F9383EB94E19F938F93E091E7
:103970005404F0915504099580911401909115011A
:103980000F900F900F900F908152934010F4C550FC
:10399000DFCF6C2F83E090E00E94B82ECF3018F07C
:1039A000CCE8D0E002C0C0E0D0E0CA3FD105F8F4D6
:1039B000C7BD82E390E00E94FB1889E294E09F93E8
:1039C0008F9383EB94E19F938F93E0915404F09154
:1039D0005504099580911401909115010F900F9055
:1039E0000F900F908052934010F02196DECFC0933D
:1039F00043068091540680FF09C08C2F8A508B3E6D
:103A000028F080917004806480937004C7BD8CE2BC
:103A100091E00E94FB18DF91CF910895EF92FF9201
:103A20001F93CF9310E080ED97E00E94D9187C019E
:103A3000CCE8133019F4CB3008F0C9E010E08091E5
:103A40005502909156028C5F934024F480911301AB
:103A500081500AC08091550290915602875094403F
:103A600034F0809113018F5F8093130101C011E046
:103A700080915302909154028C5F934024F4809182
:103A8000120181500AC080915302909154028750D4
:103A9000944034F0809112018F5F8093120101C035
:103AA0001F5F80915102909152028C5F934024F4E9
:103AB0008091110181500AC080915102909152026F
:103AC00087509440C4F0809111018F5F8093110161
:103AD00013C08BE294E09F938F9383EB94E19F93C9
:103AE0008F93E0915404F091550409950F900F9035
:103AF0000F900F905FC01F5F82E1809380028091E2
:103B00007A028E7F80937A0285EA8093BC0080914E
:103B100013018A3040F480917004816080937004B6
:103B20008AE08093130180911301863F40F08091D9
:103B3000700481608093700485EF809313018091FD
:103B400012018A3040F48091700482608093700486
:103B50008AE08093120180911201863F40F08091AB
:103B6000700482608093700485EF809312018091CD
:103B700011018A3040F48091700484608093700455
:103B80008AE08093110180911101863F40F080917D
:103B9000700484608093700485EF8093110180919C
:103BA0008002882339F0C7010E94E218882309F0B7
:103BB00090CFF5CF109210018FEC80937A00809116
:103BC00010018823E1F3CA3020F48AE090E00E94DB
:103BD000FB18C15009F02DCF86E490E00E94FB183D
:103BE000CF911F91FF90EF9008951F920F920FB603
:103BF0000F921124AF92BF92CF92DF92EF92FF9279
:103C00000F931F932F933F934F935F936F937F93E4
:103C10008F939F93AF93BF93EF93FF9380915E0237
:103C2000282F3327442755278F5F80935E02F901A1
:103C30002231310508F0AAC3EA5BFF4F0C94178EBE
:103C4000809178009091790046C0809178009091A1
:103C500079004AC180917800909179009093610237
:103C60008093600275C180918A0390918B032091AB
:103C7000780030917900821B930B909334068093E7
:103C80003306809133069091340690936B028093B3
:103C90006A027CC1809178009091790020918C0318
:103CA00030918D03821B930B9093420680934106C3
:103CB000809141069091420690936D0280936C0230
:103CC00067C38091640290916502209178003091E1
:103CD0007900820F931F909365028093640281E0C4
:103CE00058C38091620290916302209178003091D4
:103CF0007900820F931F909363028093620284E0A5
:103D000048C38091AD0683FF1AC080911E01909137
:103D10001F019C01220F331F280F391F409178008B
:103D2000509179008BE090E0489FB001499F700D61
:103D3000589F700D1124CB016EE170E00FC080918F
:103D40001E0190911F019C01220F331F280F391F64
:103D5000809178009091790063E070E00E947C8D02
:103D6000260F371F369527953695279530931F01D7
:103D700020931E0185E00DC3809178009091790019
:103D80004091860350918703841B950B90934C02BE
:103D900080934B0280914B0290914C02029704F168
:103DA00072E04E3E570784F420915F022B5F209310
:103DB0005F0225508091F9029091FA02845F914050
:103DC00018F4215F20935F0280915F02853684F1B1
:103DD0004F5F5F4F5093870340938603845626C0FE
:103DE00080914B0290914C028F5F9F4F0CF572E0D7
:103DF00047325707ECF020915F02255020935F0275
:103E00002B5F8091F9029091FA02845F914018F43F
:103E10002F5020935F0280915F028C394CF4415007
:103E2000504050938703409386038C5980935F02E0
:103E300081E080934A02809178009091790090937C
:103E40003A068093390680914B0290914C029C0176
:103E5000442737FD4095542F8091450390914603A8
:103E6000A0914703B0914803820F931FA41FB51F71
:103E70008093450390934603A0934703B093480370
:103E800020914503309146034091470350914803E8
:103E900057FF04C021503C4F4F4F5F4F0AE05595EC
:103EA0004795379527950A95D1F7809145039091CD
:103EB0004603A0914703B0914803821B930BA40BC8
:103EC000B50B8093450390934603A0934703B093AB
:103ED00048032EC180916202909163022091780084
:103EE00030917900820F931F909363028093620256
:103EF00010925D0250C2809102018A3071F480916B
:103F00007800909179002091600230916102820FD7
:103F1000931F01969695879517C040916002509126
:103F20006102843158F02091780030917900240F9B
:103F3000351F8FEF97E0821B930B06C080917800AE
:103F400090917900840F951F9093520280935102B3
:103F500086E01FC280918A0390918B0320917800A4
:103F600030917900821B930B909334068093330633
:103F7000809133069091340620916A0230916B0251
:103F8000820F931F9093500280934F0287E001C2EB
:103F9000809178009091790020918C0330918D036D
:103FA000821B930B909342068093410680914106B9
:103FB0009091420620916C0230916D02820F931F06
:103FC00090934E0280934D02E3C1209164023091A0
:103FD00065028091780090917900280F391F309305
:103FE000650220936402809102018A3019F4220F45
:103FF000331F04C0220F331F220F331F309365027B
:10400000209364022091640230916502C90137FD5A
:104010000796A3E095958795AA95E1F790935602A8
:10402000809355028091660290916702820F931FE0
:1040300097FD019695958795909367028093660208
:104040002091960330919703821B930B90931D014F
:1040500080931C0120915B0230915C0280911C01D5
:1040600090911D01280F391F37FF02C02F5F3F4F6E
:104070003595279530935C0220935B0230CE2091DA
:104080006202309163028091780090917900280F4C
:10409000391F3093630220936202809102018A30BB
:1040A00019F4220F331F04C0220F331F220F331FB6
:1040B0003093630220936202209162023091630286
:1040C000C90137FD079663E0959587956A95E1F7F5
:1040D00090935402809353028091680290916902F8
:1040E000820F931F97FD019695958795909369028E
:1040F000809368022091940330919503821B930B67
:1041000090931B0180931A012091590230915A0219
:1041100080911A0190911B01280F391F37FF02C0AF
:104120002F5F3F4F3595279530935A0220935902C0
:1041300083E02FC110925E0281E080931001809194
:104140004102909142020196909342028093410273
:1041500080917800909179009093150180931401DB
:104160008091140190911501AA27BB27A0906E029F
:10417000B0906F02C0907002D0907102A80EB91E6C
:10418000CA1EDB1EA0926E02B0926F02C092700235
:10419000D0927102809172028F5F8093720282319D
:1041A00008F4F6C08091160190911701A0911801B2
:1041B000B09119017C018D0123E0EE0CFF1C001F62
:1041C000111F2A95D1F7E81AF90A0A0B1B0BEA0C02
:1041D000FB1C0C1D1D1D80914502992787FD9095A4
:1041E000A92FB92FBC01CD0126EC34E240E050E00C
:1041F0000E94518DDC01CB01E81AF90A0A0B1B0B56
:10420000D801C7010496A11DB11DB7FF05C0D80193
:10421000C7010B96A11DB11D13E0B595A795979504
:1042200087951A95D1F78093160190931701A09363
:104230001801B093190180913B0690913C067C01D6
:104240000027F7FC0095102F80911601909117011F
:10425000A0911801B0911901E81AF90A0A0B1B0B79
:10426000E0922503F092260300932703109328037E
:1042700020914602309147024091480250914902F4
:1042800057FF04C0215F3F4F4F4F5F4FF4E05595FC
:10429000479537952795FA95D1F7809146029091E9
:1042A0004702A0914802B0914902821B930BA40BD4
:1042B000B50B8093460290934702A0934802B093B7
:1042C00049028091460290914702A0914802B09124
:1042D00049028E0D9F1DA01FB11F8093460290932F
:1042E0004702A0934802B093490280914302909103
:1042F0004402AC01E5E0440F551FEA95E1F7481B85
:10430000590B8091460290914702A0914802B091CA
:104310004902B7FF03C00F96A11DB11D74E0B5950A
:10432000A795979587957A95D1F720912503309198
:104330002603281B390B63E0220F331F6A95E1F730
:10434000240F351F37FF02C0215E3F4F45E03595F2
:1043500027954A95E1F73093440220934302D60112
:10436000C501D7FE03C00196A11DB11DB595A79546
:104370009795879580936E0290936F02A093700239
:10438000B093710289E08093720202C010925E02C3
:1043900082E080935D0280915D0280937C00809139
:1043A0005E02882319F08FEC80937A00FF91EF91E1
:1043B000BF91AF919F918F917F916F915F914F913D
:1043C0003F912F911F910F91FF90EF90DF90CF9031
:1043D000BF90AF900F900FBE0F901F90189590E276
:1043E000E1E2F1E08FE49193815087FFFCCF0895E3
:1043F00090917502E1E2F1E0E90FF11D80839F5F8A
:10440000909375020895EF92FF920F931F93CF93AD
:10441000DF932091730220FF0AC0809174028823E9
:1044200011F0815002C0809120018093740221FF1D
:104430000CC09091740280912001981719F4109289
:10444000740203C09F5F90937402822F992780FFAC
:1044500004C081FF02C0109274020E94EF2180917B
:104460007402282F332758EFE52E51E2F52EC09124
:104470005404D09155048A3098F481E180937502F8
:104480003F932F9382E694E09F938F93FF92EF9256
:10449000FE0109952DB73EB72A5F3F4F2DBF11C0D2
:1044A00080E1809375023F932F9387E694E09F937A
:1044B0008F93FF92EF92FE0109958DB79EB70696F6
:1044C0008DBF20917402822F9927AA27BB27FC0158
:1044D000429710F00C94B42CE85AFF4F48EFE42EAA
:1044E00041E2F42EC0915404D09155040C94178EDF
:1044F000109275028CE694E09F938F9308EF11E27F
:10450000FF92EF92FE01099584E1809375020F906E
:104510000F900F900F9081E690E09F938F9384E52A
:1045200090E09F938F931F921F92809102016AE007
:104530000E94708D892F99279F938F9380910201FC
:104540000E94708D99279F938F938CE794E09F939F
:104550008F93FF92EF92E0915404F09155040995E6
:1045600088E2809375022DB73EB7225F3F4F2DBF83
:104570008CEB96E09F938F930E941B3099279F931B
:104580008F9381E994E09F938F93FF92EF92E09154
:104590005404F091550409958DB79EB708968DBFC8
:1045A00090917004992351F08CE380937502892FC8
:1045B00099279F938F938FE994E081C690917B0216
:1045C000992371F08CE380937502892F99279F932B
:1045D0008F9386EB94E09F938F931F930F9391C0DB
:1045E0008091710484FF07C08CE3809375028BEC8B
:1045F00094E00C94462C809192019091930106973F
:1046000010F00C94BD2C8CE38093750288ED94E03F
:104610000C94462C8091540638EFE32E31E2F32EB1
:10462000C0915404D091550480FF74C0109275025B
:104630008091250390912603A0912703B091280330
:10464000BC01CD0125E030E040E050E00E94C58D86
:104650003F932F9385EE94E09F938F93FF92EF9279
:10466000FE01099584E1809375022DB73EB72A5F5C
:104670003F4F2DBF8091210390912203A0912303EE
:10468000B0912403BC01CD0125E030E040E050E0D2
:104690000E94C58D3F932F9382EF94E09F938F9359
:1046A000FF92EF92E0915404F0915504099588E24D
:1046B000809375028DB79EB706968DBF80911401C9
:1046C000909115019F938F938FEF94E09F938F9319
:1046D000FF92EF92E0915404F091550409958CE318
:1046E000809375022DB73EB72A5F3F4F2DBF87B528
:1046F00099279F938F938CE095E09F938F93FF92E0
:10470000EF92E0915404F091550409958DB79EB74E
:10471000069633C71092750289E195E09F938F93B7
:10472000FF92EF92FE01099584E1809375020F904C
:104730000F900F900F9088E295E09F938F93FF92D8
:10474000EF92E0915404F0915504099588E280932A
:1047500075020F900F900F900F9081E395E09F935B
:104760008F93FF92EF92E0915404F09155040995D4
:104770008CE3809375020F900F900F900F9080E460
:1047800095E09F938F93FF92EF920C944A2C109296
:10479000750289E495E09F938F9308EF11E2FF92F1
:1047A000EF92FE01099584E1809375020F900F90BE
:1047B0000F900F908091810390918203A0918303C9
:1047C000B0918403B7FF04C081509C4FAF4FBF4FDF
:1047D0002AE0B595A795979587952A95D1F7BF9328
:1047E000AF939F938F9386E595E09F938F931F934D
:1047F0000F93E0915404F0915504099588E2809359
:1048000075022DB73EB7285F3F4F2DBF80917903CA
:1048100090917A03A0917B03B0917C03B7FF04C011
:1048200081509C4FAF4FBF4FCAE0B595A795979564
:104830008795CA95D1F7BF93AF939F938F9385E6E2
:1048400095E09F938F931F930F93E0915404F09101
:10485000550409958CE3809375028DB79EB7089631
:104860008DBF8091DE019091DF019F938F9384E74C
:1048700095E09F938F931F930F93E0915404F091D1
:10488000550409952DB73EB72A5F3F4F11C71092C7
:10489000750280917607909177079F938F9380910F
:1048A0007407909175079F938F9383E895E09F938A
:1048B0008F93FF92EF92FE01099584E18093750238
:1048C0008DB79EB708968DBF80917A0790917B0730
:1048D0009F938F9380917807909179079F938F93FF
:1048E00083E995E09F938F93FF92EF92E0915404B8
:1048F000F0915504099588E2809375022DB73EB773
:10490000285F3F4F2DBF80917E0790917F079F9337
:104910008F9380917C0790917D079F938F9383EA7B
:1049200095E09F938F93FF92EF92E0915404F09162
:10493000550409958CE3809375028DB79EB7089650
:104940008DBF80918207909183079F938F93809171
:104950008007909181079F938F9383EB95E0A2C08E
:104960001092750280914906E82FFF27EE0FFF1F76
:10497000EE58F84F808191819F938F9380914806E4
:10498000E82FFF27EE0FFF1FEE58F84F808191812F
:104990009F938F9383EC95E09F938F93FF92EF9279
:1049A000FE01099584E1809375028DB79EB7089644
:1049B0008DBF80914B06E82FFF27EE0FFF1FEE58AB
:1049C000F84F808191819F938F9380914A06E82FC1
:1049D000FF27EE0FFF1FEE58F84F80819181885816
:1049E0009F4F9F938F9383ED95E09F938F93FF92BB
:1049F000EF92E0915404F0915504099588E2809378
:104A000075022DB73EB7285F3F4F2DBF80914D06F1
:104A1000E82FFF27EE0FFF1FEE58F84F808191819E
:104A200081589F4F9F938F9380914C06E82FFF27CB
:104A3000EE0FFF1FEE58F84F8081918181589F4FF4
:104A40009F938F9383EE95E09F938F93FF92EF92C6
:104A5000E0915404F091550409958CE3809375021C
:104A60008DB79EB708968DBF80914F06E82FFF2720
:104A7000EE0FFF1FEE58F84F8081918181589F4FB4
:104A80009F938F9380914E06E82FFF27EE0FFF1F15
:104A9000EE58F84F8081918181589F4F9F938F935B
:104AA00083EF95E09F938F93FF92EF92E0915404F0
:104AB000F091550409952DB73EB7285F3F4FF8C5D3
:104AC0001092750283E096E09F938F9308EF11E2B6
:104AD000FF92EF92FE010995809102010F900F90D5
:104AE0000F900F908A3009F09DC084E18093750289
:104AF00080919603909197039C0197FF02C0295FD4
:104B00003F4F287F821B930B9F938F938091960337
:104B10009091970397FD0796A3E095958795AA95A1
:104B2000E1F79F938F93209196033091970337FF7E
:104B300002C0295F3F4FF3E035952795FA95E1F7DD
:104B40008091550290915602821B930B9F938F93F5
:104B500081E196E09F938F931F930F93E09154040C
:104B6000F0915504099588E2809375028DB79EB740
:104B70000A968DBF80919403909195039C0197FFB5
:104B800002C0295F3F4F287F821B930B9F938F9317
:104B9000809194039091950397FD0796E3E0959596
:104BA0008795EA95E1F79F938F9320919403309135
:104BB000950337FF02C0295F3F4F73E03595279576
:104BC0007A95E1F78091530290915402821B930BE6
:104BD0009F938F9382E296E09F938F931F930F93FF
:104BE000E0915404F091550409958CE3809375028B
:104BF0002DB73EB7265F3F4F2DBF80919203909116
:104C000093039F938F9380919203909193032091AC
:104C1000510230915202821B930B9F938F9383E337
:104C200096E0A7C38B3019F0843108F4ADC084E15D
:104C30008093750280919603909197039C0197FF52
:104C400002C0215F3F4F207F821B930B97FD01968F
:104C5000959587959F938F93809196039091970355
:104C600097FD0F9654E0959587955A95E1F79F9398
:104C70008F93209196033091970337FF02C0295FED
:104C80003F4F43E0359527954A95E1F780915502CE
:104C900090915602821B930B9F938F9381E496E031
:104CA0009F938F931F930F93E0915404F0915504B9
:104CB000099588E2809375022DB73EB7265F3F4F76
:104CC0002DBF80919403909195039C0197FF02C0A2
:104CD000215F3F4F207F821B930B97FD0196959597
:104CE00087959F938F93809194039091950397FD5F
:104CF0000F96C4E095958795CA95E1F79F938F939A
:104D0000209194033091950337FF02C0295F3F4FF4
:104D1000B3E035952795BA95E1F7809153029091CC
:104D20005402821B930B9F938F9383E596E09F938E
:104D30008F931F930F93E0915404F09155040995BC
:104D40008CE3809375028DB79EB70A968DBF8091D4
:104D500092039091930397FD0196959587959F9364
:104D60008F938091920390919303209151023091FF
:104D70005202821B930B9F938F9385E696E09F933D
:104D80008F931F930F9392CE8D3009F0F6C584E177
:104D9000809375028091130199279F938F9380913F
:104DA00096039091970397FD0F96F4E0959587955C
:104DB000FA95E1F79F938F93209196033091970393
:104DC00037FF02C0295F3F4FE3E035952795EA950D
:104DD000E1F78091550290915602821B930B9F93AD
:104DE0008F9384E796E09F938F931F930F93E091A7
:104DF0005404F0915504099588E2809375028DB7AB
:104E00009EB70A968DBF8091120199279F938F9329
:104E1000809194039091950397FD0F9674E095957A
:104E200087957A95E1F79F938F9320919403309122
:104E3000950337FF02C0295F3F4F63E03595279503
:104E40006A95E1F78091530290915402821B930B73
:104E50009F938F9388E896E09F938F931F930F9370
:104E6000E0915404F091550409958CE38093750208
:104E70002DB73EB7265F3F4F2DBF80911101992777
:104E80009F938F93809192039091930397FD019646
:104E9000959587959F938F9380919203909193031B
:104EA0002091510230915202821B930B9F938F935A
:104EB0008CE996E09F938F931F930F93E091540496
:104EC000F091550409958DB79EB70A9656C3109276
:104ED000750280EB96E09F938F93FF92EF92FE0115
:104EE000099584E1809375020F900F900F900F90B9
:104EF00080918C0390918D039F938F9380914D02AD
:104F000090914E029F938F938DEB96E09F938F939A
:104F1000FF92EF92E0915404F0915504099588E2D4
:104F2000809375022DB73EB7285F3F4F2DBF80910C
:104F30008A0390918B039F938F9380914F0290915E
:104F400050029F938F938CEC96E09F938F93FF92E8
:104F5000EF92E0915404F091550409958CE380930D
:104F600075028DB79EB708968DBF8091860390918C
:104F700087039F938F9380914B0290914C029F9354
:104F80008F938BED96E08ECD1092750280911E016D
:104F900090911F016AE070E00E94908D9F938F9323
:104FA00080911E0190911F016AE070E00E94908D37
:104FB0007F936F938AEE96E09F938F93FF92EF9289
:104FC000FE01099584E1809375028DB79EB708961E
:104FD0008DBF8091CB089091CC086AE070E00E9470
:104FE0007C8D9F938F938091CB089091CC086AE041
:104FF00070E00E947C8D7F936F938EEF96E09F937D
:105000008F93FF92EF92E0915404F091550409952B
:1050100088E2809375022DB73EB7285F3F4F2DBFC2
:105020008091CD089091CE089F938F9382E197E075
:105030009F938F93FF92EF92E0915404F091550467
:1050400009958CE3809375028DB79EB706968DBF48
:105050008091CF089091D0089F938F9382E297E040
:105060002EC11092750284E397E09F938F93FF9275
:10507000EF92FE01099584E1809375020F900F90E5
:105080000F900F9080917207909173079F938F9369
:105090008DE397E09F938F93FF92EF92E0915404FA
:1050A000F0915504099588E2809375028DB79EB7FB
:1050B00006968DBF8091330399279F938F938DE43C
:1050C00097E09F938F93FF92EF92E0915404F091B9
:1050D000550409958CE3809375022DB73EB72A5F7E
:1050E0003F4F2DBF80917107992701979F938F9311
:1050F0008DE597E002CB109275028DE697E09F93C5
:105100008F93FF92EF92FE01099584E180937502DF
:105110000F900F900F900F90809141039091420358
:105120009F938F9385E797E09F938F93FF92EF92E2
:10513000E0915404F0915504099588E2809375023A
:105140002DB73EB72A5F3F4F2DBF8091DE01909172
:10515000DF019F938F9383E897E09F938F93FF9254
:10516000EF92E0915404F091550409958CE38093FB
:1051700075028DB79EB706968DBF809143039091BF
:1051800044039F938F9381E997E099C01092750231
:105190008091340399279F938F938FE997E09F9392
:1051A0008F93FF92EF92FE01099584E1809375023F
:1051B0008DB79EB706968DBF8091350399279F9333
:1051C0008F938BEA97E09F938F93FF92EF92E091FA
:1051D0005404F0915504099588E2809375022DB727
:1051E0003EB72A5F3F4F2DBF8091360399279F938B
:1051F0008F9387EB97E09F938F93FF92EF92E091CD
:105200005404F091550409958CE3809375028DB791
:105210009EB706968DBF8091370399279F938F93F2
:1052200083EC97E04CC01092750280913803992767
:105230009F938F938FEC97E09F938F93FF92EF92C2
:10524000FE01099584E1809375028DB79EB706969D
:105250008DBF8091390399279F938F938BED97E0B2
:105260009F938F93FF92EF92E0915404F091550435
:10527000099588E2809375022DB73EB72A5F3F4FAC
:105280002DBF80913A0399279F938F9387EE97E0E4
:105290009F938F93FF92EF92E0915404F091550405
:1052A00009958CE3809375028DB79EB706968DBFE6
:1052B00080913B0399279F938F9383EF97E09F9370
:1052C0008F93FF92EF92D9CA109275028FEF97E0F9
:1052D0009F938F9308EF11E2FF92EF92FE010995E1
:1052E00084E1809375020F900F900F900F90809142
:1052F000C10199279F938F9387E098E09F938F93A5
:10530000FF92EF92E0915404F0915504099588E2E0
:10531000809375028DB79EB706968DBF80912C0243
:1053200090912D0297FD0396959587959595879574
:105330009F938F9385E198E09F938F931F930F9393
:10534000E0915404F091550409958CE38093750223
:105350002DB73EB72A5F3F4F2DBF80917706992723
:105360009F938F938091760699279F938F9383E2E3
:1053700098E09F938F931F930F93E0915404F091C3
:10538000550409958DB79EB70896F7C0109275021F
:1053900081E398E09F938F93FF92EF92FE0109952E
:1053A00084E1809375020F900F900F900F90809181
:1053B0009104992787FD90959F938F9380919004F6
:1053C000992787FD90959F938F9381E498E09F9311
:1053D0008F93FF92EF92E0915404F0915504099558
:1053E00088E2809375022DB73EB7285F3F4F2DBFEF
:1053F00080919204992787FD90959F938F93809138
:10540000930499279F938F9381E598E09F938F93BF
:10541000FF92EF92E0915404F091550409958CE3CA
:10542000809375028DB79EB708968DBF80919704C3
:1054300099279F938F9380919404992787FD909546
:105440009F938F9381E698E02DCB1092750281E7B0
:1054500098E09F938F93FF92EF92FE01099584E16C
:10546000809375020F900F900F900F9080912C07F2
:1054700099278F7790709F938F9380912407992716
:105480008F7790709F938F9380911C0799278F77C8
:1054900090709F938F938091140799278F779070C6
:1054A0009F938F9381E898E09F938F93FF92EF9261
:1054B000E0915404F0915504099588E280937502B7
:1054C0008DB79EB70C968DBF80914C0799278F772B
:1054D00090709F938F938091440799278F77907056
:1054E0009F938F9380913C0799278F7790709F931C
:1054F0008F938091340799278F7790709F938F9324
:1055000082E998E09F938F93FF92EF92E091540489
:10551000F091550409958CE3809375022DB73EB741
:10552000245F3F4F2DBF80916C0799278F77907034
:105530009F938F938091640799278F7790709F93A3
:105540008F9380915C0799278F7790709F938F93AB
:105550008091540799278F7790709F938F9383EA58
:1055600098E09F938F93FF92EF92E0915404F09113
:10557000550409958DB79EB70C968DBFFEC110924C
:10558000750284EB98E09F938F93FF92EF92FE0158
:10559000099584E1809375020F900F900F900F9002
:1055A00080913007992787FD90959F938F938091E5
:1055B0002807992787FD90959F938F9380912007C7
:1055C000992787FD90959F938F938091180799272E
:1055D00087FD90959F938F9383EC98E09F938F9393
:1055E000FF92EF92E0915404F0915504099588E2FE
:1055F000809375022DB73EB7245F3F4F2DBF80913A
:105600005007992787FD90959F938F938091480726
:10561000992787FD90959F938F93809140079927B5
:1056200087FD90959F938F9380913807992787FDE9
:1056300090959F938F9384ED98E09F938F93FF9223
:10564000EF92E0915404F091550409958CE3809316
:1056500075028DB79EB70C968DBF80917007992704
:1056600087FD90959F938F9380916807992787FD79
:1056700090959F938F9380916007992787FD9095D0
:105680009F938F9380915807992787FD90959F93BB
:105690008F9385EE98E09F938F93FF92EF92E09126
:1056A0005404F091550409952DB73EB7245F3F4F40
:1056B0002DBF63C11092750286EF98E09F938F9380
:1056C00008EF11E2FF92EF92FE01099584E18093C9
:1056D00075020F900F900F900F9080912C07881FEC
:1056E0008827881F97E0899FC00111248D969F937A
:1056F0008F9380912407881F8827881F96E0899FB1
:10570000C00111248D969F938F9380911C07881F51
:105710008827881F95E0899FC00111248D969F934B
:105720008F9380911407881F8827881F9927880FD7
:10573000991F880F991F8D969F938F9385E099E00D
:105740009F938F93FF92EF92E0915404F091550450
:10575000099588E2809375028DB79EB70C968DBF30
:1057600080914C07881F8827881F9BE0899FC00174
:1057700011248D969F938F9380914407881F8827CB
:10578000881F9AE0899FC00111248D969F938F9363
:1057900080913C07881F8827881F99E0899FC00156
:1057A00011248D969F938F9380913407881F8827AB
:1057B000881F992723E0880F991F2A95E1F78D9676
:1057C0009F938F9389E199E09F938F93FF92EF923C
:1057D000E0915404F091550409958CE3809375028F
:1057E0002DB73EB7245F3F4F2DBF80915407881FD0
:1057F0008827881F9CE0899FC00111248D969F9364
:105800008F938DE299E09F938F93FF92EF92E091B7
:105810005404F0915504099580915C072DB73EB76B
:105820002A5F3F4F2DBF87FF12C080E4809375022F
:105830008EE399E09F938F93FF92EF92E09154044F
:10584000F091550409950F900F900F900F90809153
:10585000640787FF12C084E48093750281E499E0B5
:105860009F938F931F930F93E0915404F0915504ED
:1058700009950F900F900F900F9080916C0787FF04
:105880007CC088E48093750284E499E09F938F93B1
:105890001F930F93E0915404F091550409950F90D4
:1058A0000F900F900F9069C01092750287E499E0F5
:1058B0009F938F93FF92EF92FE01099584E180936D
:1058C00075020F900F900F900F90809102029091AF
:1058D00003029F938F9385E599E09F938F93FF92A7
:1058E000EF92E0915404F0915504099588E2809379
:1058F00075028DB79EB706968DBF80910402909178
:1059000005029F938F9382E699E09F938F93FF9276
:10591000EF92E0915404F0915504099589E4809345
:1059200075022DB73EB72A5F3F4F2DBF8FE699E036
:105930009F938F93FF92EF92E0915404F09155045E
:105940000995809173020F900F900F900F9083FF35
:1059500014C0109205021092040260E070E08EE024
:1059600090E00E94C92E09C080912001281719F4E7
:105970002150209320011092740210927302E6E0ED
:10598000CDB7DEB70C94088EF999FECF92BD81BDDC
:10599000F89A80B599270895F999FECF1FBA92BD5C
:1059A00081BD60BD0FB6F894FA9AF99A0FBE0895BA
:1059B0004AEA20E030E02617370740F4FC018191E5
:1059C000480F2F5F3F4F26173707C8F3842F9927BB
:1059D0000895EAEA40E050E04617570778F49C0142
:1059E000F999FECF32BD21BDF89A80B5E80F4F5F1F
:1059F0005F4F2F5F3F4F4617570790F38E2F992722
:105A0000089581E080934A0682E08093490683E00E
:105A10008093480684E080934B0685E080934C0693
:105A200086E080934D0687E080934E0688E0809361
:105A30004F0689E0809350068AE0809351068BE000
:105A4000809352068CE080935306089595E59093D9
:105A5000470680910201843170F08AE080936706E6
:105A600010928B068BE1809363068EE48093880608
:105A7000809389060DC083E08093670680E280935F
:105A80008B068EE180936306909388069093890637
:105A90008AE68093540662E06093AD0674E07093EA
:105AA0006E061092AA061092A70648E0409361067F
:105AB00056EE5093620690E4909364063EE1309374
:105AC00055068FEF809357068FE0809358063093EA
:105AD000560610925A0640935B0690935C0610920D
:105AE0005D0680935906109270061092710610920E
:105AF00072061092730610928D0610928E06109206
:105B00008F061092900690E89093740622E32093FB
:105B100075066093AC068093760650937706709373
:105B20007C068DE780937F068093800680938106B4
:105B30009093780685E58093790686E480937A06CB
:105B40008CED80937B068CE380937D0610927E061D
:105B50008FE58093910683EF809393068AEA809382
:105B600095068093960684E180939206809394062E
:105B7000209382069AE590938306209384061092E0
:105B8000AB068EEF8093970624E6209398069093B9
:105B9000990690939A0690939B068BE480939C06BB
:105BA00080939D0680939E0610929F0686E08093C8
:105BB000A0064093A1069093A2063093A30685EF1A
:105BC0008093A4062093A5066093A6061092A806CB
:105BD0001092A90681E280936B068DE280936C0699
:105BE00090936D060895CF93DF930E94262D8EE04B
:105BF00080935E0620E120935F063CE030936006D0
:105C000090E59093650686E9809366069093680612
:105C10008093690686E080936A0680E280936F062F
:105C20008AE5809385069093860681E080938706B7
:105C300020938A0684E680938C06AEEAB6E0E1E71C
:105C4000F1E0ED01019009923A95E1F763E770E028
:105C5000CD01875690400E94D82C8093BA06DF91E0
:105C6000CF910895CF93DF930E94262D8AE08093F1
:105C70005E0680E180935F0626E0209360069AE549
:105C80009093650688E780936606909368068093F4
:105C9000690620936A0620E220936F06909385069A
:105CA00080E5809386068CE38093870620938A069E
:105CB0008BE480938C06AEEAB6E08CE0E8E7F1E096
:105CC000ED01019009928A95E1F763E770E0CD015B
:105CD000875690400E94D82C8093BA06DF91CF91CE
:105CE0000895CF93DF930E94262D88E080935E066F
:105CF00030E130935F0626E02093600694E69093AF
:105D0000650688E780936606909368068093690627
:105D100020936A0630936F068AE58093850680E5B6
:105D20008093860696E49093870680E280938A06A5
:105D300090938C06AEEAB6E08CE0E0E8F1E0ED018D
:105D4000019009928A95E1F763E770E0CD018756EB
:105D500090400E94D82C8093BA06DF91CF9108958D
:105D6000F999FECF92BD81BDF89A80B59927089523
:105D7000F999FECF1FBA92BD81BD60BD0FB6F894F0
:105D8000FA9AF99A0FBE089564EC7CE20E94DF8BC8
:105D900008954CEC5CE20E94198C0895EF92FF92FA
:105DA0000F931F93CF93C82F8150853008F0C3E025
:105DB00084E7C89F8001112480EFE82E8FEFF82E32
:105DC000E00EF11E63E770E0C7010E94E92C682F26
:105DD00098012D593F4F8FB39927AC0142705070F5
:105DE00081FDF9CF32BD21BDF89A80B5861711F03B
:105DF000CA0121C08FB399279C012270307081FDA8
:105E0000F9CFF2BCE1BCF89A80B5853511F0C90133
:105E100012C084E7C89FC0011124409724EC3CE2E3
:105E200044E750E0BC0187E496E00E94BA8B0E94F0
:105E30007F6B81E090E0CF911F910F91FF90EF90E9
:105E40000895282F863010F025E003C0882309F438
:105E500021E0F999FECF1FBA82E090E092BD81BDAA
:105E600020BD0FB6F894FA9AF99A0FBE0895CF9311
:105E7000C82F80914706853509F042C0C63010F022
:105E8000C5E003C0CC2309F43BC063E770E087E4BE
:105E900096E00E94D82C8093BA0684E7C89FC00180
:105EA00011242CEC3CE244E750E067E476E04097B4
:105EB0000E94F78B2CEC3CE24CE050E068E476E08A
:105EC00080E590E00E94F78B6CE070E088E496E05B
:105ED0000E94D82C282FF999FECF1FBA8CE590E0AC
:105EE00092BD81BD20BD0FB6F894FA9AF99A0FBE03
:105EF0008C2F0E94212F0E947F6B81E090E002C0D6
:105F000080E090E0CF9108956DE470E088EE93E03A
:105F10000E94E92C482F8FB399279C012270307082
:105F200081FDF9CF85E394E092BD81BDF89A80B5FB
:105F3000841779F48FB399279C012270307081FD0A
:105F4000F9CF88EE93E092BD81BDF89A80B581309B
:105F500011F0C901089524EC3CE24EE450E068EEF3
:105F600073E08BEB96E00E94BA8B81E090E008959D
:105F70008091BB068130A9F46DE470E08BEB96E074
:105F80000E94D82C809308072CEC3CE24EE450E0B1
:105F90006BEB76E088EE93E00E94F78B81E090E077
:105FA000089580E090E00895CF93DF9381E080939F
:105FB000BB06EBEBF6E08FE0158616861786108A97
:105FC0008150349687FFF8CF80E48093C806809391
:105FD000C9061092CA068093CB068093CC0690EC3B
:105FE0009093CD061092CE068093CF068093D00674
:105FF0001092D1069093D2069093D3068093D40644
:106000001092D5068093D6069093D706ACEBB6E0F7
:1060100087E0EAE8F1E0ED01019009928A95E1F765
:106020006DE470E0CD0101970E94D82C80930807A1
:10603000DF91CF910895F999FECF82E090E092BD73
:1060400081BDF89A80B5282F863078F023E0322F72
:10605000F999FECF1FBA82E090E092BD81BD30BDBC
:106060000FB6F894FA9AF99A0FBE822F99270895DD
:106070001F93CF93C82F162F863010F0C5E003C0B2
:10608000882309F4C1E08C2F99278230910541F0D3
:106090008330910544F4019731F40E94F32D05C03B
:1060A0000E94322E02C00E94712E1123E1F06CE09A
:1060B00070E080E590E00E94E92C282FF999FECF4E
:1060C0008CE590E092BD81BDF89A80B5821759F4B5
:1060D00024EC3CE24CE050E060E570E088E496E0BF
:1060E0000E94BA8B02C00E94012D8C2F0E94372F74
:1060F000CF911F910895DF92EF92FF920F931F931C
:10610000CF93FF24DF2CEF2C81E090E00E94B02E93
:10611000853539F031E0E32E65E581E090E00E94BD
:10612000B82E6CE070E080E590E00E94E92CC82F6A
:10613000F999FECF8CE590E092BD81BDF89A80B5CB
:106140008C1711F421E0D22EC1E001E010E0EE2026
:1061500029F48C2F0E94CE2E8823C1F591E0F92ED0
:106160001F930F9387E799E09F938F9383EB94E1BD
:106170009F938F93E0915404F091550409958DB746
:106180009EB706968DBF0230110549F00330110508
:106190004CF40130110531F40E94F32D05C00E942A
:1061A000322E02C00E94712EDD2059F024EC3CE218
:1061B0004CE050E060E570E088E496E00E94BA8B25
:1061C00002C00E94012D8C2F0E94372FCF5F0F5FDE
:1061D0001F4FC63008F4BBCFFF2019F083E00E94A8
:1061E000212F0E941B30C82F0E94CE2E8C2F992762
:1061F0009F938F938DE999E09F938F9303EB14E125
:106200001F930F93E0915404F091550409958DB7B5
:106210009EB706968DBFEE2021F40E94842F88231E
:1062200099F486EB99E09F938F931F930F93E091DE
:106230005404F091550409950E94D42F0E94B82F60
:106240000F900F900F900F901092460690E0E8ECA0
:10625000F6E0CFE08081349618160CF49F5FC150B1
:10626000C7FFF8CF90934606892F99279F938F9366
:106270008CEB96E09F938F9387ED99E09F938F939C
:106280001F930F93E0915404F091550409958DB735
:106290009EB708968DBF88EF99E09F938F931F93C9
:1062A0000F93E0915404F091550409950F900F90CD
:1062B0000F900F90CF911F910F91FF90EF90DF9073
:1062C0000895982F2FB7F8943998389A88B1836039
:1062D00088B98091B9008C7F8093B9008AE280935D
:1062E000B8001092800210927E0210927D029923D3
:1062F00079F0E1E1F7E08BE01082118212821382E3
:1063000014821582168217828150389687FFF4CF47
:1063100078942FBF08951092800284E98093BC0086
:1063200080E88093BC001092BD001092BA001092D9
:10633000BB001092B9001092B80010927C0280E06D
:106340000E9461311092BB0085E88093BC0080916F
:106350007A02826080937A0208951F920F920FB69C
:106360000F9211242F933F934F935F938F939F939B
:10637000EF93FF9380918002282F332744275527DE
:106380008F5F80938002F9012731310508F0C2C286
:10639000E659FF4F0C94178E81E080937C0209C070
:1063A00080917E028C3090F480917E028F5F80938A
:1063B0007E0280917E02E82FFF27EE0FFF1FEE0F77
:1063C000FF1FE554F94F8585181654F780917E021A
:1063D0008C3070F0109279021092780210927E0246
:1063E00085E08093800280917D02880F8D5A04C0E1
:1063F00080917E02880F8E5A8093BB0085E87FC211
:1064000080917E02E82FFF2783E0EE0FFF1F8A9521
:10641000E1F7EF5EF84F81818093BB0085E88093C0
:10642000BC0080917E02E82FFF27EE0FFF1FEE0FCA
:10643000FF1FEE0FFF1FEF5EF84F808180FF91C0BE
:1064400080917E02E82FFF27EE0FFF1FEE0FFF1F48
:10645000EE0FFF1FEF5EF84F8281882329F08091B5
:106460004606873008F46CC28091780290917902D8
:10647000892B09F065C28091760290917702892B71
:1064800009F05EC26EC080917E0221E030E002C061
:10649000220F331F8A95E2F780917602909177025E
:1064A00028233923232B79F080917E02E82FFF27C0
:1064B000EE0FFF1FEE0FFF1FEE0FFF1FEF5EF84FF7
:1064C00080E184830DC080917E02E82FFF27EE0FCC
:1064D000FF1FEE0FFF1FEE0FFF1FEF5EF84F14823E
:1064E00080917E02E82FFF2753E0EE0FFF1F5A95A1
:1064F000E1F7EF5EF84F8481282F332743E0220F26
:10650000331F4A95E1F780917E02E82FFF2793E041
:10651000EE0FFF1F9A95E1F7EF5EF84F82818770CB
:10652000822B8093BB0085E88093BC0020917E0283
:1065300081E090E002C0880F991F2A95E2F7209130
:1065400078023091790282239323892B51F089E0DC
:1065500097E0909384028093830288E08093850281
:10656000EFC184E089C1E0918302F09184028191BE
:106570008093BB0085E88093BC00F0938402E09395
:10658000830280918502815080938502882309F4DB
:10659000D7C183E071C18091B900803351F58091FA
:1065A0008102882329F480917E028F5F809381028B
:1065B00080917E02E82FFF2783E0EE0FFF1F8A9570
:1065C000E1F7EF5EF84F838199278F7790708F37CF
:1065D00091057CF480917E02E82FFF27EE0FFF1FCC
:1065E000EE0FFF1FEE0FFF1FEF5EF84F83818F5FEF
:1065F00083831092800284E98093BC008AE090E05B
:10660000909393018093920180917E028F5F80939B
:106610007E02109280026DC18091B9008034C9F170
:1066200080917D02E82FFF27EE0FFF1FEE0FFF1F67
:10663000EE0FFF1FEF5EF84F83818F77838380918A
:106640007D028F5F80937D0280917D028C30A0F06F
:1066500010927D021092770210927602809182024F
:106660008F5F809382028C3038F01092820280918A
:106670007A028D7F80937A0280917A028160809382
:106680007A021092800284E98093BC0010927C020E
:1066900073C080917D02E82FFF27EE0FFF1FEE0FE2
:1066A000FF1FEE0FFF1FEF5EF84F8381806883832B
:1066B00080917D02E82FFF27EE0FFF1FEE0FFF1FD7
:1066C000EE0FFF1FEF5EF84F808180FF2FC080919B
:1066D0007D02E82FFF2753E0EE0FFF1F5A95E1F7E9
:1066E000EF5EF84F84819927009751F04097D9F5D4
:1066F00089E097E0909384028093830288E031C020
:1067000080917D02992743E0880F991F4A95E1F710
:106710008A5E984F909384028093830290917D02C9
:10672000809182029817E1F483E01BC080917D0282
:10673000992733E0880F991F3A95E1F78A5E984FC1
:10674000909384028093830280917A0281FD06C037
:1067500090917D0280918202981711F482E001C02D
:1067600081E08093850280918502813011F485E873
:1067700001C085EC8093BC008091810280937B02F4
:1067800010928102DDC0E0918302F0918402809139
:10679000BB00808380918302909184020196909344
:1067A00084028093830280918502815080938502C8
:1067B000823010F085EC5DC0813011F485E859C05D
:1067C00080917A0281FF2DC08091F80280FD1DC06A
:1067D00080917D02E82FFF2723E0EE0FFF1F2A950F
:1067E000E1F7EF5EF84F86818A3F79F480917D0270
:1067F000E82FFF2793E0EE0FFF1F9A95E1F7EF5E7A
:10680000F84F8081816080830CC080917D02E82FE9
:10681000FF2783E0EE0FFF1F8A95E1F7EF5EF84F49
:10682000108280917D028F5F80937D0280917D0236
:106830008C30A0F010927D021092770210927602B6
:10684000809182028F5F809382028C3038F01092A8
:10685000820280917A028D7F80937A021092800268
:1068600084E98093BC0080917A02816080937A02EF
:1068700065C08093BC0086E08093800261C088E997
:10688000BBCD80917F02880F805FB6CD80917F0263
:1068900099278130910561F0823091051CF4892B94
:1068A00021F04EC0029739F04BC080911301A4CD66
:1068B00080911201A1CD809111019ECD80E89CCDE7
:1068C0001092800284E98093BC0010927C028AE0DE
:1068D00090E0909393018093920180917F028230A7
:1068E00088F480917F028F5F80937F0282E18093A2
:1068F000800280917A028E7F80937A0285EA80936B
:10690000BC001EC010927F0280917A028160809349
:106910007A0216C01092800284E98093BC008091B4
:106920007A02816080937A028AE090E090939301EA
:106930008093920110927E0210927D0210927C024E
:10694000FF91EF919F918F915F914F913F912F9187
:106950000F900FBE0F901F9018951F93CF93DF934A
:10696000182F80912A03882321F480911102882313
:1069700019F081E090E097C01D3008F092C011231B
:10698000B1F0E12FFF2723E0EE0FFF1F2A95E1F77B
:10699000EF5EF84F35978081359688230CF081C0E3
:1069A0003897808180FD03C083E090E07CC08091B7
:1069B0000907823019F084E090E075C067E070E06C
:1069C00089E097E00E94D82C90911007891719F060
:1069D00085E090E068C080ED97E00E94D918EC0156
:1069E00080917A0280FD05C0CE010E94E2188823C2
:1069F000B9F3112319F48FEF90E00BC0212F332747
:106A00002150304081E090E002C0880F991F2A9504
:106A1000E2F79093790280937802A1E0B0E0E1E19F
:106A2000F7E040E050E06BE0CD01042E02C0880F9B
:106A3000991F0A94E2F7209178023091790282231B
:106A40009323892B11F01182128261504F5F5F4FA7
:106A5000389667FFE9CF10927E02109280028091F3
:106A60007A028E7F80937A0285EA8093BC008091BF
:106A70007A0280FD05C0CE010E94E2188823B9F396
:106A80008091780290917902892B29F0CE010E94A1
:106A9000E218882311F3809178029091790200978F
:106AA00011F082E090E0DF91CF911F9108950F9354
:106AB0001F93CF93DF93982F80912A03882321F48B
:106AC00080911102882319F081E090E092C09D30FE
:106AD000A0F4992319F486E090E08BC0C92FDD273C
:106AE000FE0133E0EE0FFF1F3A95E1F7EF5EF84F3E
:106AF00035978081359687FD03C082E090E079C0AC
:106B00003897808180FD03C083E090E072C080ED03
:106B100097E00E94D9188C0180917A0280FD05C00F
:106B2000C8010E94E2188823B9F3219721E030E0E0
:106B3000C90102C0880F991FCA95E2F790937702A6
:106B400080937602D901E1E1F7E040E050E06BE0AC
:106B5000CD01042E02C0880F991F0A94E2F72091FC
:106B600076023091770282239323892B11F01182D0
:106B7000128261504F5F5F4F389667FFE9CF1092E6
:106B80007D021092090710921007109280028091E6
:106B90007A028E7F80937A0285EA8093BC0080918E
:106BA0007A0280FD05C0C8010E94E2188823B9F36B
:106BB0008091760290917702892B29F0C8010E947A
:106BC000E218882311F380910907823019F084E0DC
:106BD00090E00FC067E070E089E097E00E94D82C59
:106BE00090911007891719F085E090E002C080E0CD
:106BF00090E0DF91CF911F910F91089589E1A6EA6E
:106C0000B7E0E2E7F7E011821082329611961C920B
:106C10001E921296815087FFF6CF80918C0790913B
:106C20008D078F57904090938D0780938C078091AC
:106C30008E0790918F078F57904090938F07809386
:106C40008E0780919007909191078F579040909375
:106C500091078093900780919207909193078F57A7
:106C60009040909393078093920710929303109211
:106C7000920310929503109294031092970310922E
:106C8000960308951F920F920FB60F9211240F933F
:106C90001F932F933F934F935F936F937F938F93A4
:106CA0009F93AF93BF93CF93DF93EF93FF93809125
:106CB000AD0682FDCFC04091860050918700809143
:106CC000870290918802481B590B80918600909111
:106CD00087009093880280938702CA018D54944064
:106CE000A0918902B0918A02835F9A4178F48091E1
:106CF000890280937107149714F01092940181E037
:106D000090E090938A028093890207C2AD30B1056A
:106D10000CF003C2CA018B5F9040845B914008F085
:106D200074C0425D5140FD01EA0FFB1FEE58F84F61
:106D300080819181FA01E81BF90BCF01F7FF03C0B5
:106D4000909581959F4F06975CF480913303883C22
:106D500020F480913303865F01C088EC8093330375
:106D6000FD01EA0FFB1FEE58F84F808191819C01D5
:106D7000220F331F280F391F240F351F37FF02C082
:106D80002D5F3F4FE901D595C795D595C795CA01A8
:106D900001968C179D0714F4219706C0415050406E
:106DA000C417D5070CF4219680913303833CE0F09F
:106DB0008D010A0F1B1FF801EE58F84F8081918159
:106DC0009E01281B390BC90163E070E00E94908D81
:106DD000CB01880F991F860F971F0A55184FD801AE
:106DE00011969C938E9307C0AA0FBB1FAA55B84F4C
:106DF00011961C921E92E0918902F0918A02EE0F88
:106E0000FF1FEE58F84FD183C08320918902309143
:106E10008A022F5F3F4F30938A022093890280912C
:106E20000201843108F079C12530310511F45D9AF1
:106E300001C05D988091890290918A028630910507
:106E400011F45C9A01C05C98079711F45B9A65C1D4
:106E50005B9863C1409186005091870080918B02BE
:106E600090918C02481B590B80918600909187006D
:106E700090938C0280938B02CA018D549440609150
:106E8000F502835F9A4108F07AC060938602809190
:106E90008602843008F453C0909171078091860275
:106EA000981709F04CC05091F6025B3008F43FC0CF
:106EB000109294011092F50240E05F31C0F0E42F8F
:106EC000FF27EE0FFF1F9F012F533D4FDF01AE58ED
:106ED000B84F8D919C91D9018D939C93DF01AA5558
:106EE000B84F8D919C91E552FD4F91838083E42FA3
:106EF000FF27EE0FFF1F9F012E58384FDF01A357CA
:106F0000BD4F8D919C91D90111969C938E93DF0179
:106F1000A955BD4F8D919C91EA55F84F918380837F
:106F2000842F8F5F482F8D3040F28093F50280913F
:106F3000F6028F3FB9F08F5F8093F60213C0809105
:106F4000F602853620F08AE08093F60202C01092A5
:106F5000F602809102018A3011F0843110F0289AF3
:106F600001C0289881E08093F50280912A0388234C
:106F700009F0D3C08091860280937107CEC06D3036
:106F800008F0A3C0CA018B5F9040845B914008F079
:106F90007EC0425D5140E62FFF27EE0FFF1FE357F3
:106FA000FD4F80819181FA01E81BF90BCF01059615
:106FB0000B97B0F48091F6028A3120F08091330370
:106FC000865F05C08B3028F0809133038E5F8093FD
:106FD000330380913303893C18F088EC80933303AA
:106FE000E62FFF27EE0FFF1FE357FD4F80819181B2
:106FF0009C01220F331F280F391F240F351F37FF25
:1070000002C02D5F3F4FE901D595C795D595C7952E
:10701000CA0101968C179D0714F4219706C04150B0
:107020005040C417D5070CF42196809133038E3B52
:10703000D8F0E62FFF27EE0FFF1FDF01A357BD4F4C
:107040008D919C919E01281B390BC90163E070E072
:107050000E94908DCB01880F991F860F971FE955CD
:10706000FD4F9183808308C0E62FFF27EE0FFF1F9F
:10707000E955FD4F118210828091F502E82FFF271C
:10708000EE0FFF1FE357FD4FD183C08309C08091EE
:1070900002018A3011F0843110F0289A01C028983A
:1070A00080910201843188F48091F502853011F4D9
:1070B0005D9A05C05D98863011F45C9A05C05C98B5
:1070C000873011F45B9A01C05B988091F50284319E
:1070D00020F48F5F8093F50220C08431F1F4809119
:1070E00002018A3011F0843110F0289A01C02898EA
:1070F0008EE18093F5022CE0C6EAD7E0A1ECB2E085
:10710000E2E7F7E08D919D91918380833296198219
:1071100018822296215027FFF5CFFF91EF91DF9142
:10712000CF91BF91AF919F918F917F916F915F911F
:107130004F913F912F911F910F910F900FBE0F9084
:107140001F901895EF92FF920F931F938091630603
:107150009927880F991F880F991F7C010027F7FC3A
:107160000095102F8091810390918203A091830359
:10717000B0918403BC01CD01A80197010E94C58D87
:107180003093F3052093F2058091790390917A036F
:10719000A0917B03B0917C03BC01CD01A8019701B4
:1071A0000E94C58D3093F5052093F4058091370832
:1071B0009091380897FD03969595879595958795B5
:1071C0009093F7058093F6058091490890914A08BD
:1071D00097FD039695958795959587959093F905D5
:1071E0008093F8058091920390919303209151022E
:1071F00030915202821B930B9093FB058093FA050A
:107200008091250390912603A0912703B091280334
:10721000BC01CD0125E030E040E050E00E94C58D8A
:107220003093FD052093FC0580914B0290914C0218
:107230009093FF058093FE058091DE019091DF0120
:10724000909303068093020680911E0190911F0186
:1072500090930506809304068091330399279093B9
:107260000706809306068091450890914608A091F4
:107270004708B091480820919601309197014091BC
:10728000980150919901BC01CD010E94C58D3093A8
:1072900009062093080680911207992790930B0600
:1072A00080930A0680911A07992790930D06809380
:1072B0000C0680912207992790930F0680930E0663
:1072C00080912A0799279093110680931006809148
:1072D00032079927909313068093120680913A07FC
:1072E0009927909315068093140680911C03992783
:1072F00090931706809316068091420799279093E2
:1073000025068093240680914A07992790932706A3
:107310008093260680912C0290912D0290931B065B
:1073200080931A068091CB089091CC0890931F0609
:1073300080931E068091CF089091D00890932106EB
:10734000809320068091210390912203A091230332
:10735000B0912403BC01CD0125E030E040E050E0D5
:107360000E94C58D3093230620932206809143030B
:107370009091440390932906809328068091D10828
:10738000992790932D0680932C0680911604909156
:10739000170490932F0680932E06809114049091E9
:1073A00015049093310680933006809170048823F1
:1073B00021F480917104882321F08091F10581608E
:1073C00003C08091F1058E7F8093F1051F910F918D
:1073D000FF90EF9008951F93CF93DF93182FEB0149
:1073E00080912A038823A1F411501F3F89F0D09384
:1073F0003302C09332028091320290913302892B82
:10740000D1F7CE018C0F9D1F0E94EE18115078F716
:10741000DF91CF911F910895CF93DF938091020167
:107420008D3011F40E940E1D10927A008091550249
:10743000909156029093F5078093F4078091530240
:10744000909154029093E4078093E3078091510256
:107450009091520290933F0880933E0820914D02F4
:1074600030914E02C901880F991F880F991F820F12
:10747000931F820F931F90933808809337082091B1
:107480004F0230915002C901880F991F880F991F30
:10749000820F931F820F931F90934A08809349088D
:1074A0008FEC80937A00A4E3B3E0CCE4D6E097E0DD
:1074B0008991E82FFF27EE0FFF1FEE58F84F01903C
:1074C000F081E02DE158FF4F1E161F061CF0E0E092
:1074D000F0E005C0EF3FF10514F0EFEFF0E08C9124
:1074E000282F3327E217F30714F4815004C02E1716
:1074F0003F0714F48F5F8C939150119697FFD8CF6C
:10750000809188069927AA27BB27BC01CD0124ECCE
:1075100039E040E050E00E94518DDC01CB018093C6
:10752000D6019093D701A093D801B093D90180914F
:1075300089069927AA27BB27BC01CD010E94518D3E
:10754000DC01CB018093D2019093D301A093D401AD
:10755000B093D501DF91CF910895A0E0B0E0E3EBC7
:10756000FAE30C94E68D882EC0E0D0E07E016E0137
:1075700010927004469AD0938D03C0938C03D093DD
:107580008B03C0938A03D0938703C0938603D09361
:107590009703C0939603D0939503C0939403D0931D
:1075A0009303C09392031092BE011092BD011092FA
:1075B00045020E940C3A84E690E00E94FB180E946B
:1075C0000C3A8091540680FF10C080911401909174
:1075D0001501875B934038F4809114019091150157
:1075E0008E5E924010F40E948C1C0FE18AE090E0C5
:1075F0000E94FB188091510290915202C80FD91F2E
:107600008091550290915602E80EF91E8091530226
:1076100090915402C80ED91E015007FFE7CF970181
:10762000205F3F4F369527953695279530939703E2
:1076300020939603C60140969695879596958795D3
:1076400090939503809394036096F5E0D695C79543
:10765000FA95E1F7D0939303C0939203909391032B
:107660008093900330938F0320938E03882009F436
:1076700041C0809137089091380897FF03C09095DA
:1076800081959F4F6CE070E00E94908D9B017093FC
:107690008D0360938C038091490890914A0897FF6D
:1076A00003C0909581959F4F6CE070E00E94908D93
:1076B00070938B0360938A038091390690913A0608
:1076C0009093870380938603B90184E090E00E9441
:1076D000C92E60918A0370918B0386E090E00E942E
:1076E000C92E609186037091870388E090E00E9424
:1076F000C92E65C084E090E00E94C42E90938D0353
:1077000080938C0386E090E00E94C42E90938B03BC
:1077100080938A0388E090E00E94C42E9C0190939D
:1077200087038093860380918C0390918D03815011
:10773000984050F480918A0390918B038150984037
:1077400018F421503440D8F18CEF99E09F938F9337
:1077500083EB94E19F938F93E0915404F09155044F
:107760000995809137089091380897FF03C090954C
:1077700081959F4F6CE070E00E94908D70938D0317
:1077800060938C038091490890914A0897FF03C049
:10779000909581959F4F6CE070E00E94908D709362
:1077A0008B0360938A038091390690913A069093F7
:1077B0008703809386030F900F900F900F90109285
:1077C000F5071092F4071092E4071092E307109265
:1077D0003F0810923E0884E690E00E94FB188091DA
:1077E0004D0290914E029C01220F331F220F331F36
:1077F000280F391F280F391F309338082093370876
:1078000080914F02909150028C01000F111F000FC8
:10781000111F080F191F080F191F10934A08009312
:10782000490880916306C82EDD24EE24FF244427F6
:1078300037FD4095542FC701B6010E94518D4B0171
:107840005C01609381037093820380938303909320
:1078500084039801442737FD4095542FC701B60192
:107860000E94518DDC01CB018093790390937A03C0
:10787000A0937B03B0937C0380925D0390925E03A0
:10788000A0925F03B09260038093550390935603D8
:10789000A0935703B09358031092510310925203D0
:1078A0001092530310925403809116019091170186
:1078B000A0911801B091190190933C0680933B066A
:1078C0001092440210924302109245031092460314
:1078D00010924703109248038091DE019091DF01DE
:1078E000909344038093430384E690E09093DB01FC
:1078F0008093DA010E948E6682E390E090933302D7
:1079000080933202809188069927AA27BB27BC0161
:10791000CD0124EC39E040E050E00E94518DDC01C3
:10792000CB018856954CAF4FBF4F8093D6019093B3
:10793000D701A093D801B093D901809189069927E6
:10794000AA27BB27BC01CD010E94518DDC01CB01D0
:107950008856954CAF4FBF4F8093D2019093D3017F
:10796000A093D401B093D50110929B0110929A017B
:107970008091DE019091DF01AA2797FDA095BA2F93
:107980002091960130919701409198015091990171
:10799000BC01CD010E94518DDC01CB0180934508D3
:1079A00090934608A0934708B093480810923E036E
:1079B00010923D0381E0809301010E947F6B8091D2
:1079C000F80284608093F8028FEF8093C6081092CB
:1079D000C70880E28093C808C4E3D3E0ACE4B6E013
:1079E00007E08D91E82FFF27EE0FFF1FEE58F84FAD
:1079F0008081918181588993015007FFF2CF84E6FD
:107A00008093330380913002882311F0469A579A6D
:107A1000809196039091970380569940815C9B4298
:107A200028F08091700481608093700480919403A9
:107A30009091950380569940815C9B4228F08091FB
:107A400070048260809370048091920390919303FC
:107A50008C5291408957954028F080917004846041
:107A60008093700480918C0390918D038C5291408F
:107A7000835C914028F0809170048860809370044A
:107A800080918A0390918B038C529140835C91404A
:107A900028F0809170048061809370048091860347
:107AA00090918703805092408355914028F08091B7
:107AB000700480628093700486E48093D101ECE0CE
:107AC000CDB7DEB70C94028EA3E1B0E0EAE6FDE3A9
:107AD0000C94E08D80919203909193032091510238
:107AE00030915202821B930B90933F0880933E0883
:107AF00080915B0290915C0297FD07969C0113E0D8
:107B0000359527951A95E1F73093F5072093F407FB
:107B10008091590290915A0297FD0796B3E095958E
:107B20008795BA95E1F79093E4078093E307309344
:107B30000108209300089093F9078093F80780913B
:107B4000370890913808AC01440F551F480F591F52
:107B500020914D0230914E02C901880F991F880F64
:107B6000991F820F931F820F931F480F591F57FFB2
:107B700002C04D5F5F4F559547955595479550937A
:107B80003808409337088091490890914A08AC0121
:107B9000440F551F480F591F20914F02309150023A
:107BA000C901880F991F880F991F820F931F820F99
:107BB000931F480F591F57FF02C04D5F5F4F5595E8
:107BC00047955595479550934A0840934908209109
:107BD0004D0230914E02C901880F991F880F991FDD
:107BE000820F931F820F931F9C01442737FD4095FE
:107BF000542F8091710390917203A0917303B091FF
:107C00007403820F931FA41FB51F80937103909379
:107C10007203A0937303B093740320914F023091C9
:107C20005002C901880F991F880F991F820F931F57
:107C3000820F931F9C01442737FD4095542F80915C
:107C40006D0390916E03A0916F03B0917003820F4A
:107C5000931FA41FB51F80936D0390936E03A09391
:107C60006F03B093700380910C0890910D082091E0
:107C70004D0230914E02820F931F90930D08809316
:107C80000C08809141089091420820914F02309158
:107C90005002820F931F9093420880934108809175
:107CA00088039091890301969093890380938803B8
:107CB0008091390690913A0620918603309187038E
:107CC000821B930B9C01442737FD4095542F8091D4
:107CD000690390916A03A0916B03B0916C03820FCA
:107CE000931FA41FB51F8093690390936A03A09309
:107CF0006B03B0936C038FEC80937A0010921001A9
:107D00002091590330915A0340915B0350915C03D9
:107D100029873A874B875C8729543B46414050402E
:107D20002CF028E43BE641E050E00DC089859A85BF
:107D3000AB85BC85885B9449AE4FBF4F4CF428EBB4
:107D400034E94EEF5FEF2D833E834F83588708C0A1
:107D500089859A85AB85BC858D839E83AF83B887E3
:107D60002091610330916203409163035091640359
:107D70002D873E874F87588B29543B4641405040C2
:107D80002CF028E43BE641E050E00DC08D859E8557
:107D9000AF85B889885B9449AE4FBF4F4CF428EB50
:107DA00034E94EEF5FEF29833A834B835C8308C04D
:107DB0008D859E85AF85B88989839A83AB83BC8383
:107DC000A0913E08B0913F08BB8BAA8BFD01CF016B
:107DD000AA2797FDA095BA2FA0905103B090520307
:107DE000C0905303D0905403A80EB91ECA1EDB1EC8
:107DF000A0925103B0925203C0925303D092540305
:107E0000E0904508F0904608009147081091480816
:107E1000E80EF91E0A1F1B1FE0924508F092460863
:107E20000093470810934808F0911303F98BFF2340
:107E300009F098C180911203882309F093C18091C1
:107E4000540686FF8FC18091E3079091E407AA272B
:107E500097FDA095BA2FBC01CD0129813A814B81B4
:107E60005C810E94518D9B01AC0197FF04C02150A1
:107E7000384F4F4F5F4FBBE0559547953795279546
:107E8000BA95D1F78091BD01682E77248824992472
:107E9000CA01B901A40193010E94518DDC01CB01FB
:107EA0008093AF039093B003A093B103B093B20358
:107EB000B7FF04C08150904FAF4FBF4F1C012D0141
:107EC000ACE05594479437942794AA95D1F7209223
:107ED000AF033092B0034092B1035092B20380914D
:107EE000F4079091F507AA2797FDA095BA2FBC013A
:107EF000CD012D813E814F8158850E94518D97FF84
:107F000004C06150784F8F4F9F4FFBE09595879548
:107F100077956795FA95D1F7A40193010E94518D49
:107F2000DC01CB018093B3039093B403A093B5031A
:107F3000B093B603B7FF04C08150904FAF4FBF4F0F
:107F40009C01AD01ECE05595479537952795EA954D
:107F5000D1F72093B3033093B4034093B503509308
:107F6000B6038091AF039091B0039093DB078093A9
:107F7000DA078091B3039091B4039093DF07809365
:107F8000DE0722193309440955092093B3033093BE
:107F9000B4034093B5035093B603E20EF31E041FDF
:107FA000151FE0924508F092460800934708109389
:107FB00048088091BC018823B1F457FF04C02F5FAB
:107FC0003F4F4F4F5F4F5595479537952795A21ACD
:107FD000B30AC40AD50AA0925103B0925203C092C8
:107FE0005303D09254032A893B8979010027F7FC77
:107FF0000095102F8091B3039091B403A091B50325
:10800000B091B603E80EF91E0A1F1B1FC801B70185
:1080100029813A814B815C810E94518D9B01AC0189
:1080200097FF04C02150384F4F4F5F4F6BE055957D
:108030004795379527956A95D1F78091BE01A82E6F
:10804000BB24CC24DD24CA01B901A60195010E94FC
:10805000518DDC01CB018093A7039093A803A093DB
:10806000A903B093AA03B7FF04C08150904FAF4F4C
:10807000BF4F3C014D013CE0959487947794679401
:108080003A95D1F76092A7037092A8038092A90352
:108090009092AA03C801B7012D813E814F81588576
:1080A0000E94518D97FF04C06150784F8F4F9F4FB2
:1080B0002BE095958795779567952A95D1F7A60139
:1080C00095010E94518DDC01CB018093AB0390930D
:1080D000AC03A093AD03B093AE03B7FF04C08150CF
:1080E000904FAF4FBF4FAC01BD018CE075956795C8
:1080F000579547958A95D1F74093AB035093AC03BE
:108100006093AD037093AE032A893B8937FF03C0A8
:10811000309521953F4F21343105E4F1D401C3015D
:1081200097FE07C0B095A095909581959F4FAF4F52
:10813000BF4F81389105A105B10584F4DB01CA0167
:1081400077FF07C0B095A095909581959F4FAF4F51
:10815000BF4F81389105A105B105E4F081E080931E
:108160003F0318C01092DF071092DE071092DB0762
:108170001092DA071092AB031092AC031092AD0389
:108180001092AE031092A7031092A8031092A903B5
:108190001092AA038091AB039091AC03A091AD0320
:1081A000B091AE03BC01CD0124E630E040E050E0E8
:1081B0000E94C58DE090A703F090A803E21AF30A8D
:1081C000F092F307E092F2078091A7039091A80341
:1081D000A091A903B091AA03BC01CD0124E630E02F
:1081E00040E050E00E94C58DDA01C9012091AB0347
:1081F0003091AC038C01021B130B1093E707009323
:10820000E6078091960190919701A0919801B09115
:108210009901BC01CD0128E631E040E050E00E9428
:10822000518D209145083091460840914708509162
:108230004808261737074807590764F0261B370BED
:10824000480B590B20934508309346084093470844
:1082500050934808209145083091460840914708BE
:108260005091480857FF0CC0260F371F481F591F51
:108270002093450830934608409347085093480898
:108280006091E3077091E4076E0D7F1D9B01442709
:1082900037FD4095542F8091550390915603A0913E
:1082A0005703B0915803820F931FA41FB51F8093EB
:1082B000550390935603A0935703B09358038091AE
:1082C000180390911903681B790BCB01AA2797FD1E
:1082D000A095BA2F29853A854B855C85820F931F1F
:1082E000A41FB51F8093590390935A03A0935B0377
:1082F000B0935C03C090D201D090D301E090D40140
:10830000F090D501C816D906EA06FB06C4F488EA3F
:1083100091E6A0E0B0E08C199D09AE09BF098093F9
:10832000590390935A03A0935B03B0935C0380932B
:10833000550390935603A0935703B09358032227F5
:108340003327A9012C193D094E095F098091590372
:1083500090915A03A0915B03B0915C03821793073D
:10836000A407B507B4F4D701C601885A9146A040C6
:10837000B0408093590390935A03A0935B03B0934A
:108380005C038093550390935603A0935703B093D7
:1083900058036091F4077091F507600F711F9B01FE
:1083A000442737FD4095542F80915D0390915E03E3
:1083B000A0915F03B0916003820F931FA41FB51FAC
:1083C00080935D0390935E03A0935F03B09360037B
:1083D0008091160390911703681B790BCB01AA2794
:1083E00097FDA095BA2F2D853E854F855889820F20
:1083F000931FA41FB51F8093610390936203A09302
:108400006303B0936403E090D601F090D70100912C
:10841000D8011091D901E816F9060A071B07C4F420
:1084200088EA91E6A0E0B0E08E199F09A00BB10B9D
:108430008093610390936203A0936303B0936403FA
:1084400080935D0390935E03A0935F03B0936003FA
:1084500022273327A9012E193F09400B510B809188
:10846000610390916203A0916303B091640382174A
:108470009307A407B507B4F4D801C701885A9146F9
:10848000A040B0408093610390936203A093630384
:10849000B093640380935D0390935E03A0935F03A6
:1084A000B09360038091510390915203A0915303C4
:1084B000B09154038093650390936603A093670380
:1084C000B09368038091610390916203A09163036C
:1084D000B09164038093810390938203A0938303FC
:1084E000B09384038091590390915A03A0915B0348
:1084F000B0915C038093790390937A03A0937B03FC
:10850000B0937C0380915D0390915E03A0915F0323
:10851000B091600380937D0390937E03A0937F03CB
:10852000B09380038091550390915603A091570317
:10853000B09158038093750390937603A0937703CB
:10854000B093780380911C0190911D0197FD0796CF
:1085500003E0959587950A95E1F79093F507809349
:10856000F40780911A0190911B0197FD079613E083
:10857000959587951A95E1F79093E4078093E30723
:1085800080915502909156020F9734F488E19CEF48
:108590009093F5078093F4078091550290915602CD
:1085A000079734F480E398EF9093F5078093F407EE
:1085B000209102012A30A9F480915502909156022F
:1085C000835F934034F088EE93E09093F5078093B7
:1085D000F40780915502909156028A5F9340DCF037
:1085E00014C08091550290915602815D974034F0FD
:1085F00088EE93E09093F5078093F40780915502FD
:1086000090915602805E974034F080ED97E0909311
:10861000F5078093F40780915302909154020F97CD
:1086200034F488E19CEF9093E4078093E307809112
:10863000530290915402079734F480E398EF90939B
:10864000E4078093E3072A30A9F4809153029091C4
:108650005402835F934034F088EE93E09093E407F4
:108660008093E30780915302909154028A5F934074
:10867000DCF014C08091530290915402815D9740C8
:1086800034F088EE93E09093E4078093E3078091C1
:10869000530290915402805E974034F080ED97E051
:1086A0009093E4078093E3076091C801662309F47F
:1086B000AFC040911C0150911D018091B703909172
:1086C000B803481B590B5093BE034093BD03209140
:1086D0001C0130911D01280F391F37FF02C02F5F89
:1086E0003F4F359527953093B8032093B703413812
:1086F00051051CF080E890E005C040585F4F34F40D
:1087000080E89FEF9093BE038093BD0340911A01D0
:1087100050911B018091B9039091BA03481B590BEA
:108720005093BC034093BB0320911A0130911B016D
:10873000280F391F37FF02C02F5F3F4F3595279510
:108740003093BA032093B903413851051CF080E8F7
:1087500090E005C040585F4F34F480E89FEF90935D
:10876000BC038093BB03462F55278091BD03909196
:10877000BE03849FB001859F700D949F700D1124DE
:108780009B0177FF02C0215F3F4FF4E035952795AD
:10879000FA95E1F78091F4079091F507820F931F06
:1087A0009093F5078093F4078091BB039091BC03ED
:1087B000849FD001859FB00D949FB00D1124AD0111
:1087C0009D01B7FF02C0215F3F4FE4E0359527953B
:1087D000EA95E1F78091E3079091E407820F931FF8
:1087E0009093E4078093E30780911C0190911D0111
:1087F000860F971F90931D0180931C0180911A0191
:1088000090911B01840F951F90931B0180931A0177
:108810000091F8071091F9078091DA079091DB0732
:10882000101611065CF59C0197FF04C02227332720
:10883000281B390BC901AA2797FDA095BA2F2091B3
:10884000BC01332744275527BC01CD010E94518D1F
:108850009B01AC0197FF04C0215C3F4F4F4F5F4F1E
:1088600076E055954795379527957A95D1F780917C
:10887000F2079091F307820F931F27C097FF03C061
:10888000909581959F4FAA2797FDA095BA2F20918B
:10889000BC01332744275527BC01CD010E94518DCF
:1088A0009B01AC0197FF04C0215C3F4F4F4F5F4FCE
:1088B00066E055954795379527956A95D1F780914C
:1088C000F2079091F307821B930B9093F307809329
:1088D000F207E0900008F09001088091DE07909187
:1088E000DF071E141F045CF59C0197FF04C02227BC
:1088F0003327281B390BC901AA2797FDA095BA2F4A
:108900002091BC01332744275527BC01CD010E948B
:10891000518D9B01AC0197FF04C0215C3F4F4F4F2D
:108920005F4F96E055954795379527959A95D1F7DE
:108930008091E6079091E707820F931F27C097FF6A
:1089400003C0909581959F4FAA2797FDA095BA2FB8
:108950002091BC01332744275527BC01CD010E943B
:10896000518D9B01AC0197FF04C0215C3F4F4F4FDD
:108970005F4F86E055954795379527958A95D1F7AE
:108980008091E6079091E707821B930B9093E7078E
:108990008093E6078091540687FF44C0B989BB23C2
:1089A00009F040C0809112038823E1F5E1E0EE1662
:1089B000E1E0FE064CF08091F4079091F5078E0DF2
:1089C0009F1D805091400DC0F0E0EF16FFEFFF06B5
:1089D00064F48091F4079091F5078E0D9F1D8050EF
:1089E0009F4F9093F5078093F40721E00130120721
:1089F0004CF08091E3079091E407800F911F805025
:108A000091400CC03FEF0030130764F48091E307FE
:108A10009091E407800F911F80509F4F9093E4073F
:108A20008093E307E2E1CD5E0C94FC8D80912A03F4
:108A3000882301F58091F8028C7F8093F802A5E7E6
:108A4000B4E0E1E1F7E09BE080911102882309F4B2
:108A50008C938D91818312829150389697FFF4CF39
:108A600080911102882359F08091110281508093E6
:108A7000110205C08091F80281608093F802809114
:108A80007C02882319F010927C02089580937E0264
:108A90008093800280917A028E7F80937A0285EAA9
:108AA0008093BC000895CF93DF93A4E3B3E0CCE4BC
:108AB000D6E057E08991E82FFF27EE0FFF1FEE5811
:108AC000F84F0190F081E02DE158FF4FEF3FF105A5
:108AD00021F01CF0EFEFF0E004C0F7FF02C0E0E08F
:108AE000F0E04C91242F3327E217F307A9F0CF01D0
:108AF000821B930B97FD0396959587959595879582
:108B0000242F280F2C93822F9927E817F90714F4A4
:108B1000215001C02F5F2C935150119657FFCACF9F
:108B200080915606883F38F0EFEFF0E0E81BF1093E
:108B3000EC5CFC4F80818093CE018091CE01882334
:108B400029F0843618F084E68093CE01809158068F
:108B5000883F38F0EFEFF0E0E81BF109EC5CFC4FE8
:108B600080818093CC018091CC01882329F08436C8
:108B700018F084E68093CC0180916506883F38F038
:108B8000EFEFF0E0E81BF109EC5CFC4F8081809393
:108B9000C7018091C7018B3010F48AE002C08F3F7B
:108BA00011F48093C70180919206883F38F0EFEF6F
:108BB000F0E0E81BF109EC5CFC4F808180930E082B
:108BC00080910E08823010F481E002C08F3F11F4D2
:108BD00080930E0880919406883F38F0EFEFF0E024
:108BE000E81BF109EC5CFC4F808180933A0880918E
:108BF0003A08823010F481E002C08F3F11F4809374
:108C00003A0880917F06883F38F0EFEFF0E0E81BEC
:108C1000F109EC5CFC4F808180930908809180060B
:108C2000883F38F0EFEFF0E0E81BF109EC5CFC4F17
:108C300080818093E00780918106883F38F0EFEFD4
:108C4000F0E0E81BF109EC5CFC4F80818093140894
:108C500090915706983F18F49093CD0109C0EFEF1B
:108C6000F0E0E91BF109EC5CFC4F80818093CD01C1
:108C7000983F18F49093CD0109C0EFEFF0E0E91BA5
:108C8000F109EC5CFC4F80818093CD0180915A0604
:108C9000883F38F0EFEFF0E0E81BF109EC5CFC4FA7
:108CA00080818093CB0180915C06883F38F0EFEFA4
:108CB000F0E0E81BF109EC5CFC4F80818093C90176
:108CC00080916406883F38F0EFEFF0E0E81BF1098F
:108CD000EC5CFC4F80818093CA0180916606883FDE
:108CE00038F0EFEFF0E0E81BF109EC5CFC4F80811D
:108CF0008093C60180916706883F38F0EFEFF0E07F
:108D0000E81BF109EC5CFC4F80818093C8018091E5
:108D10006806883F38F0EFEFF0E0E81BF109EC5C03
:108D2000FC4F80818093C50180916906883F38F0AF
:108D3000EFEFF0E0E81BF109EC5CFC4F80818093E1
:108D4000C40180916F06883F38F0EFEFF0E0E81B38
:108D5000F109EC5CFC4F80818093C2018091700628
:108D6000883F38F0EFEFF0E0E81BF109EC5CFC4FD6
:108D7000808180930D0380917106883F38F0EFEF7A
:108D8000F0E0E81BF109EC5CFC4F808180930C0360
:108D900080917206883F38F0EFEFF0E0E81BF109B0
:108DA000EC5CFC4F808180930B0380917306883FBD
:108DB00038F0EFEFF0E0E81BF109EC5CFC4F80814C
:108DC00080930A0380918D06883F38F0EFEFF0E042
:108DD000E81BF109EC5CFC4F8081809309038091D2
:108DE0008E06883F38F0EFEFF0E0E81BF109EC5C0D
:108DF000FC4F80818093080380918F06883F38F074
:108E0000EFEFF0E0E81BF109EC5CFC4F8081809310
:108E1000070380919006883F38F0EFEFF0E0E81B01
:108E2000F109EC5CFC4F808180930603809174060D
:108E3000883F38F0EFEFF0E0E81BF109EC5CFC4F05
:108E400080818093C10180917806883F38F0EFEFF0
:108E5000F0E0E81BF109EC5CFC4F80818093C001DD
:108E600080918206883F38F0EFEFF0E0E81BF109CF
:108E7000EC5CFC4F80818093BF0180918506883F28
:108E800038F0EFEFF0E0E81BF109EC5CFC4F80817B
:108E90008093BE0180918606883F38F0EFEFF0E0C6
:108EA000E81BF109EC5CFC4F80818093BD0180914F
:108EB0008706883F38F0EFEFF0E0E81BF109EC5C43
:108EC000FC4F80818093BC0180918C06883F38F0F4
:108ED000EFEFF0E0E81BF109EC5CFC4F8081809340
:108EE000BB018091A706883F38F0EFEFF0E0E81B68
:108EF000F109EC5CFC4F808180934C088091C201A9
:108F0000282F33272F5F3F4F8CE398E2B9010E944F
:108F1000908D7093D0016093CF0180916206809311
:108F20003B08809161068093FA079091A9069333DC
:108F3000E8F181E080930503983F58F0EFEFF0E00F
:108F4000E91BF109EC5CFC4F8081823310F4109234
:108F500005038091D10120910503821799F0833098
:108F600070F4222319F08CED95E002C088EC90E0BB
:108F700090933302809332022093D10103C0815039
:108F80008093D10180918D0890918E0897FF08C041
:108F900080910503882321F080917004806803C0CC
:108FA000809170048F778093700405C01092050340
:108FB0008AE08093D10180918D0890918E0897FF6F
:108FC0001DC080912A038823C9F08091050388235E
:108FD000A9F080910801909109018F5F9F4F71F472
:108FE00088E99AE3909333028093320280E094EA16
:108FF0009093090180930801109205038091050365
:10900000882369F08091F70281608093F702809154
:10901000BE01823D48F4825E8093BE0105C080910E
:10902000F7028E7F8093F702DF91CF910895A9E137
:10903000B0E0EDE1F8E40C94E08D0E94643D3091E5
:1090400002013C3010F4299A01C02998E0902B03CA
:10905000F0902C03FA82E9828091FA0799270A9608
:10906000E816F90614F49A838983809133038436D1
:1090700008F05CC08091D3039091D403009731F045
:1090800001979093D4038093D30307C010922A03CF
:109090008091F8028F7E8093F8023A3011F03431DB
:1090A00010F0289A01C028988091F9029091FA0254
:1090B000895E9340C0F180916C06282F33273A8354
:1090C00029838091F80280618093F802809148069C
:1090D000A82FBB27AA0FBB1FFD01EA55F84F11822D
:1090E000108280914906282F3327220F331FC90190
:1090F0008A55984FFC0111821082AE58B84F1196D4
:109100001C921E922E58384FD90111961C921E9215
:1091100080914B06E82FFF27EE0FFF1FEE58F84F08
:1091200011821082D4C210922A03D1C280913303DB
:109130008D3808F4CCC28091F8028F7E8093F802BB
:1091400090916D0682E3989FC00111249093D403FF
:109150008093D303E981FA81B9978CF080912A0337
:10916000882369F08091F9029091FA02FFEF8F3F16
:109170009F0729F001969093FA028093F90280915B
:10918000F9029091FA028F3F910509F008F51092CB
:109190004D0310924E0310924F0310925003109201
:1091A000490310924A0310924B0310924C03109201
:1091B000BF031092C0031092C1031092C203109219
:1091C000510310925203109253031092540305C09E
:1091D0008091F80282608093F80280914A06E82F1D
:1091E000FF27EE0FFF1FEE58F84F808191818135E8
:1091F00091050CF452C120912A03222309F04DC19C
:1092000080914B06E82FFF27EE0FFF1FEE58F84F17
:10921000808191818C3491050CF417C18091D50324
:109220008F5F8093D503893C08F437C13C3010F43C
:10923000299801C0299A10922A031092D5031092FE
:10924000FA021092F90230914806E32FFF27EE0F41
:10925000FF1FEE58F84F8081918187349105B4F457
:1092600080914906E82FFF27EE0FFF1FEE58F84FB9
:10927000808191810190F081E02DF7FF03C0F0958E
:10928000E195FF4FE734F1050CF478C041E02091FF
:109290004906A22FBB27AA0FBB1FAE58B84F8D910E
:1092A0009C9111978734910544F0E32FFF27EE0F2F
:1092B000FF1FEE58F84F808191818D919C918734EA
:1092C000910574F080914806E82FFF27EE0FFF1FED
:1092D000EE58F84F80819181873491050CF042E07F
:1092E000E22FFF27EE0FFF1FEE58F84F808191818C
:1092F0008634910574F480914806E82FFF27EE0F1D
:10930000FF1FEE58F84F80819181873491050CF052
:1093100043E0E22FFF27EE0FFF1FEE58F84F80814A
:1093200091818A5B9F4F74F480914806E82FFF2754
:10933000EE0FFF1FEE58F84F808191818734910521
:109340000CF044E0E22FFF27EE0FFF1FEE58F84F1E
:10935000808191818A5B9F4F74F480914806E82F49
:10936000FF27EE0FFF1FEE58F84F80819181863462
:1093700091050CF445E0842F0E94212F809149062D
:10938000E82FFF27EE0FFF1FEE58F84F80819181E5
:109390000190F081E02DF7FF03C0F095E195FF4FBC
:1093A0007E97BCF480914806E82FFF27EE0FFF1F41
:1093B000EE58F84F808191818A5B9F4F54F481E091
:1093C00080938B0488EE93E0909333028093320273
:1093D00064C00E941B300E94CE2E80E00E94C00814
:1093E00080916E060E94EA898091540680FF10C029
:1093F0008091140190911501875B934038F480911E
:109400001401909115018E5E924010F40E948C1C04
:109410001092300280E00E94AD3A81E080939A037E
:1094200080933002579A0E941B3068E770E00E94D8
:10943000EB3985E68093FE010E941B309AE0899FFC
:10944000C00111248093FC0128C080819181855B3B
:109450009F4F0CF58091D5038F5F8093D503893C96
:10946000E0F03C3010F4299801C0299A10922A03A8
:109470001092D5031092FA021092F90281E00E9434
:10948000AD3A81E080939A030E941B3068E770E058
:109490000E94EB3902C02093D50380914A06E82F41
:1094A000FF27EE0FFF1FEE58F84F808191818B5AF6
:1094B0009F4F0CF00CC130912A03E0914B063323EF
:1094C00009F0DAC0FF27EE0FFF1FEE58F84F80813A
:1094D0009181855B9F4F0CF0CCC02091AA06E22FB2
:1094E000FF27EE0FFF1FEE58F84F80819181855BBB
:1094F0009F4F1CF0222309F0BCC08091D6038F5FE0
:109500008093D603893C08F4E2C03093D60380915F
:109510007004882309F0A6C080919A03882309F477
:10952000A1C080912004882309F09CC081E090E0D4
:109530009093FA028093F90281E080932A031092BB
:10954000BF031092C0031092C1031092C203109285
:1095500051031092520310925303109254038091BE
:109560006306E82EFF240027112780913708909189
:1095700038089C01442737FD4095542FC801B70196
:109580000E94518DDC01CB018093610390936203B3
:10959000A0936303B09364038091490890914A08B3
:1095A0009C01442737FD4095542FC801B7010E9404
:1095B000518DDC01CB018093590390935A03A09302
:1095C0005B03B0935C038091810390918203A0912F
:1095D0008303B091840380935D0390935E03A09313
:1095E0005F03B09360038091790390917A03A09117
:1095F0007B03B0917C038093550390935603A09313
:109600005703B093580310924D0310924E031092DB
:109610004F03109250031092490310924A03109284
:109620004B0310924C038091F80288608093F802FB
:109630009091A8068FE0989F900111248091DE01FF
:109640009091DF01820F931F68E671E00E94908D78
:1096500097FD0196959587958093850384E6809381
:10966000D80335C08CED95E090933302809332029D
:109670002EC01092D6032BC0FF27EE0FFF1FEE580F
:10968000F84F808191818C349105FCF02091AA06DD
:10969000E22FFF27EE0FFF1FEE58F84F80819181D8
:1096A000855B9F4F14F0222381F48091D7038F5F55
:1096B0008093D703893C58F010922A031092D70365
:1096C0001092FA021092F90202C01092D703809110
:1096D0009401815080939401809194018F3F21F0F7
:1096E0008091F80284FF72C30E9453458091E10388
:1096F0009091E2039C01220F331F280F391FC09065
:109700004806AC2DBB27AA0FBB1FFD01EE58F84F32
:10971000B0905E064B2D552780819181849FF0018A
:10972000859FF00D949FF00D11242E0F3F1F37FFE2
:1097300002C02D5F3F4FB901759567957595679587
:10974000AA55B84F80915F06082F11278D919C91E3
:10975000809F7001819FF00C909FF00C11246E0D82
:109760007F1D7093E2036093E1038091E303909186
:10977000E4039C01220F331F280F391FD0904906A4
:10978000AD2DBB27AA0FBB1FFD01EE58F84F8081FE
:109790009181849FF001859FF00D949FF00D11241D
:1097A0002E0F3F1F37FF02C02D5F3F4FA901559578
:1097B000479555954795AA55B84F8D919C91809F97
:1097C0007001819FF00C909FF00C11244E0D5F1DD5
:1097D0005093E4034093E30380910503882309F445
:1097E00048C0CB0177FD0396DC01B595A795B595EB
:1097F000A795CA0157FD0396FC01F595E795F595E8
:10980000E7958091F301682F772767FD70956A9F30
:1098100090016B9F300D7A9F300D112480912204AE
:10982000482F552747FD50954E9FC0014F9F900DE3
:109830005E9F900D1124280F391F37FF02C0295F4A
:109840003F4F03E0359527950A95E1F730933203B2
:10985000209331036E9F90016F9F300D7E9F300DDE
:1098600011244A9FC0014B9F900D5A9F900D1124C7
:109870003FC08091A806E82FFF27E456FE4F86815F
:109880008093F301908190932204A82FBB27A7FD1A
:10989000B095A69F9001A79F300DB69F300D112463
:1098A000E92FFF27E7FDF095E49FC001E59F900DAC
:1098B000F49F900D1124280F391F37FF02C0295F34
:1098C0003F4F13E0359527951A95E1F73093320312
:1098D00020933103A49F9001A59F300DB49F300DBC
:1098E0001124E69FC001E79F900DF69F900D112473
:1098F000281B390B37FF02C0295F3F4FF3E0359536
:109900002795FA95E1F73093300320932F03809148
:109910004B06E82FFF27EE0FFF1FEE58F84F808110
:109920009181909581959F4F90932E0380932D0365
:109930008530910514F0049705C00FEF8C3F900718
:1099400034F4049690932E0380932D0304C0109258
:109950002E0310922D0380911604909117042091EC
:10996000120430911304820F931F00913103109160
:109970003203081B190B10933203009331038091BB
:109980001404909115042091100430911104820F59
:10999000931F80902F0390903003881A990A909219
:1099A000300380922F0380914A06E82FFF27EE0FA5
:1099B000FF1FEE58F84FE080F18028E730E0E20E1C
:1099C000F31EF0922C03E0922B038091C70199279C
:1099D000AA2797FDA095BA2FBC01CD010E94C58C86
:1099E000DC01CB0120E030E040E251E4BC01CD01DC
:1099F0000E94338CDC01CB01BC01CD010E94978C0D
:109A0000DC01CB01809343088091C6018093160846
:109A10008091C5019927AA2797FDA095BA2FBC016F
:109A2000CD010E94C58CDC01CB0120E030E040E29A
:109A300051E4BC01CD010E94338CDC01CB01BC019F
:109A4000CD010E94978CDC01CB018093EC078091C3
:109A5000C401809302088091970480FF59C08091CF
:109A60004C08813808F454C080919004992787FDF0
:109A700090952B2D3327829FA001839F500D929F9D
:109A8000500D1124040F151F10933203009331035E
:109A900080919104992787FD9095829FB001839FC3
:109AA000700D929F700D1124860E971E90923003B8
:109AB00080922F0380919204282F332727FD309521
:109AC00080912D0390912E03820F931F90932E036C
:109AD00080932D0380919404282F332727FD309500
:109AE000809159069927289FD001299FB00D389F52
:109AF000B00D1124B0939B01A0939A01809193041F
:109B000099278E159F0524F490932C0380932B03A3
:109B100080912B0390912C0397FF04C010922C038B
:109B200010922B038091540682FF02C010921608F7
:109B30004091310350913203CA0157FD03969C01B5
:109B4000359527953595279537FF03C03095219595
:109B50003F4F8091FD029091FE0282179307B4F46B
:109B6000CA0157FF03C0909581959F4F97FD0396BB
:109B700095958795959587959093FE028093FD0224
:109B80008536910544F084E690E001C001979093FA
:109B9000FE028093FD0240912F0350913003CA01D1
:109BA00057FD03969C01359527953595279537FFE9
:109BB00003C0309521953F4F8091FB029091FC02AC
:109BC00082179307B4F4CA0157FF03C0909581959B
:109BD0009F4F97FD039695958795959587959093BB
:109BE000FC028093FB028536910544F084E690E008
:109BF00001C001979093FC028093FB028091F802D0
:109C000084FF08C01092FE021092FD021092FC0226
:109C10001092FB02ED2DFF27EE0FFF1FEE58F84FBD
:109C200040918306242F332780819181281739079B
:109C300044F48091AB0682FF04C081E0809311035D
:109C400013C0ED2DFF27EE0FFF1FEE58F84F842FA6
:109C5000992720918406821B910920813181281740
:109C6000390714F41092110340914906E42FFF279D
:109C7000EE0FFF1FEE58F84F50918306852F99275E
:109C800022273327281B390B808191818217930764
:109C900044F48091AB0683FF04C081E080931003FD
:109CA00016C080911003882391F0E42FFF27EE0F58
:109CB000FF1FEE58F84F809184069927851B910964
:109CC000208131818217930714F410921003EC2D38
:109CD000FF27EE0FFF1FEE58F84F40918306242F09
:109CE0003327808191812817390744F48091AB068E
:109CF00080FF04C081E080930E0317C080910E03A3
:109D0000882399F0EC2DFF27EE0FFF1FEE58F84F38
:109D1000842F992720918406821B9109208131810B
:109D20002817390714F410920E0340914806E42FC7
:109D3000FF27EE0FFF1FEE58F84F50918306852F37
:109D4000992722273327281B390B8081918182177D
:109D5000930744F48091AB0681FF04C081E08093B7
:109D60000F0316C080910F03882391F0E42FFF2783
:109D7000EE0FFF1FEE58F84F809184069927851B40
:109D80009109208131818217930714F410920F03F7
:109D900080911103882319F480911003811181E0CF
:109DA0008093120380910E03882321F480910F0386
:109DB000882351F081E080931303109212031092D4
:109DC00011031092100302C08093130380911203B9
:109DD000882321F480911303882369F080918206FF
:109DE0009927E981FA818E179F0714F49A83898352
:109DF00081E080933F038091F80284FF1AC01092A3
:109E00002E0310922D031092320310923103109200
:109E1000300310922F039AE59093430888E78093CC
:109E200016089093EC078093020810921203109288
:109E300013038091050890910608A0910708B0913E
:109E4000080820918103309182034091830350914F
:109E50008403820F931FA41FB51F8093050890935E
:109E60000608A0930708B093080880910F08909106
:109E70001008A0911108B091120820907903309039
:109E80007A0340907B0350907C03820D931DA41DA8
:109E9000B51D80930F0890931008A0931108B093FC
:109EA00012088091FC079091FD07A091FE07B091E8
:109EB000FF07E0907D03F0907E0300917F031091F7
:109EC0008003EB82FC820D831E838E0D9F1DA01FDD
:109ED000B11F8093FC079093FD07A093FE07B093FA
:109EE000FF078091ED079091EE07A091EF07B091E9
:109EF000F007E0907503F0907603009177031091DE
:109F00007803EF82F88609871A878E0D9F1DA01FA0
:109F1000B11F8093ED079093EE07A093EF07B093E6
:109F2000F007F0901303FB86FF2029F480911203C1
:109F3000882309F460C0109271031092720310928A
:109F400073031092740310926D0310926E031092BB
:109F50006F03109270031092050810920608109279
:109F600007081092080810920F081092100810921B
:109F70001108109212081092FC071092FD0710921F
:109F8000FE071092FF071092ED071092EE07109255
:109F9000EF071092F0078091610390916203A09106
:109FA0006303B091640380935D0390935E03A09379
:109FB0005F03B09360038091590390915A03A0917D
:109FC0005B03B0915C038093550390935603A09379
:109FD0005703B0935803109242021092410210921C
:109FE00017031092160310921903109218030B8591
:109FF000002309F0F9C180911203882309F0F4C10C
:10A000008091390690913A06815092402CF48091CB
:10A010002A03882309F4E8C16091C6086C87A090E0
:10A0200063068091370890913808998F888FA091A6
:10A030004908B0914A08BB8BAA8B16160CF0DDC0FC
:10A04000BB24CC24DD24CA01B901A60195010E94DC
:10A05000C58D79018A01E88DF98DCF01AA2797FD79
:10A06000A095BA2FE81AF90A0A0B1B0BC201B1011D
:10A07000A60195010E94C58D59016A012A893B8973
:10A08000C901AA2797FDA095BA2FA81AB90ACA0A2A
:10A09000DB0A3C85232E332427FC3094432C532C9D
:10A0A000C801B701A20191010E94518D97FF04C020
:10A0B00061507E4F8F4F9F4F3B014C0109E09594BB
:10A0C0008794779467940A95D1F7C601B501A201E8
:10A0D00091010E94518D97FF04C061507E4F8F4FB8
:10A0E0009F4F5B016C0119E0D594C794B794A79476
:10A0F0001A95D1F74C854093DC018091FD02909137
:10A10000FE02813491053CF48091FB029091FC02A7
:10A1100081349105D4F0D401C30197FE03C00196A8
:10A12000A11DB11D3C014D019594879477946794CE
:10A13000D601C501D7FE03C00196A11DB11D5C016A
:10A140006D01D594C794B794A79480914B06E82FDE
:10A15000FF27EE0FFF1FEE58F84F8081918101908D
:10A16000F081E02DF7FF03C0F095E195FF4F7A975E
:10A17000A4F0C401B30123E030E040E050E00E94CD
:10A18000C58D39014A01C601B50123E030E040E048
:10A1900050E00E94C58D59016A018091C808282F9E
:10A1A000332727FD3095432F532F261537054805B4
:10A1B000590514F439014A01992787FD9095909526
:10A1C00081959F4FAA2797FDA095BA2F681679060B
:10A1D0008A069B0614F43C014D012A153B054C05EB
:10A1E0005D0514F459016A01A816B906CA06DB0612
:10A1F0000CF0D2C05C016D01CFC0EA2CFF24002717
:10A200001127CA01B901A80197010E94C58D390122
:10A210004A01688D798DCB01AA2797FDA095BA2FA9
:10A22000681A790A8A0A9B0AC201B101A80197013A
:10A230000E94C58D59016A01EA89FB89CF01AA27CD
:10A2400097FDA095BA2FA81AB90ACA0ADB0AD40149
:10A25000C30197FE03C00F96A11DB11D3C014D0126
:10A26000F4E09594879477946794FA95D1F7D601A2
:10A27000C501D7FE03C00F96A11DB11D5C016D0184
:10A28000E4E0D594C794B794A794EA95D1F7809168
:10A29000FD029091FE02813491053CF48091FB0215
:10A2A0009091FC0281349105A4F0C401B30123E034
:10A2B00030E040E050E00E94C58D39014A01C601FE
:10A2C000B50123E030E040E050E00E94C58D590127
:10A2D0006A0180914B06E82FFF27EE0FFF1FEE5813
:10A2E000F84F808191810190F081E02DF7FF03C04C
:10A2F000F095E195FF4F7A97A4F0C401B30123E0F4
:10A3000030E040E050E00E94C58D39014A01C601AD
:10A31000B50123E030E040E050E00E94C58D5901D6
:10A320006A0189E18093DC01F1E26F167104810416
:10A3300091042CF070E2672E712C812C912C00EE90
:10A3400060160FEF70060FEF80060FEF900644F4D3
:10A3500060EE662E6FEF762E6FEF862E6FEF962EE5
:10A3600011E2A116B104C104D1042CF050E2A52ED3
:10A37000B12CC12CD12C20EEA2162FEFB2062FEF5C
:10A38000C2062FEFD20644F440EEA42E4FEFB42EB7
:10A390004FEFC42E4FEFD42E809161039091620352
:10A3A000A0916303B091640386199709A809B909BC
:10A3B0008093610390936203A0936303B09364035B
:10A3C0008091590390915A03A0915B03B0915C0373
:10A3D0008A199B09AC09BD098093590390935A03CC
:10A3E000A0935B03B0935C03809141029091420281
:10A3F0008F3F910509F008F4C4C53B85332309F06C
:10A400004EC580911203882309F049C580913F030E
:10A41000882309F044C540918B064D87442309F4F5
:10A420003EC58091050890910608A0910708B0915B
:10A430000808B7FF04C081509F4FAF4FBF4FE92EB0
:10A44000FA2E0B2F112707FD1A95E0920508F092BE
:10A450000608009307081093080880910F08909150
:10A460001008A0911108B0911208B7FF04C08150E4
:10A470009F4FAF4FBF4F892F9A2FAB2FBB27A7FD01
:10A48000BA958E879F87A88BB98B80930F0890937E
:10A490001008A0931108B093120880916306A82EAB
:10A4A000BB24CC24DD2420917103309172034091B0
:10A4B000730350917403C601B5010E94518D97FF3B
:10A4C00004C061507F4F8F4F9F4F672E782E892E8B
:10A4D000992487FC9A94609271037092720380921F
:10A4E00073039092740320916D0330916E03409139
:10A4F0006F0350917003C601B5010E94518D97FF03
:10A5000004C061507F4F8F4F9F4F272E382E492E0A
:10A51000552447FC5A9420926D0330926E0340926A
:10A520006F03509270038091690390916A03A09128
:10A530006B03B0916C03B7FF04C081509F4FAF4FC6
:10A54000BF4F892F9A2FAB2FBB27A7FDBA958093BA
:10A55000690390936A03A0936B03B0936C03D801D3
:10A56000C70186199709A809B9098093CB0390936D
:10A57000CC03A093CD03B093CE0320918A06E22EA4
:10A58000FF2400271127BC01CD01A80197010E94DB
:10A59000C58D59016A012093D9033093DA034093A2
:10A5A000DB035093DC038E859F85A889B9898219C6
:10A5B0009309A409B5098093CF039093D003A09386
:10A5C000D103B093D203BC01CD01A80197010E9431
:10A5D000C58D2093DD033093DE034093DF0350935A
:10A5E000E003D601C501D7FE04C081509F4FAF4F95
:10A5F000BF4F892F9A2FAB2FBB27A7FDBA959093FA
:10A6000017038093160357FF04C021503F4F4F4F4D
:10A610005F4FBB2757FDBA95A52F942F832F90939B
:10A620001903809318038091FD029091FE028134FA
:10A630009105DCF48091FB029091FC02813491053C
:10A64000A4F480914B06E82FFF27EE0FFF1FEE5872
:10A65000F84F808191810190F081E02DF7FF03C0D8
:10A66000F095E195FF4F7A97E4F08091C6088F3F0F
:10A67000C1F4809116039091170397FD019695956B
:10A6800087959093170380931603809118039091F8
:10A69000190397FD019695958795909319038093DB
:10A6A00018038091FC079091FD07A091FE07B091DF
:10A6B000FF07B7FF04C081509F4FAF4FBF4F892F97
:10A6C0009A2FAB2FBB27A7FDBA958093FC079093D9
:10A6D000FD07A093FE07B093FF078091ED079091CF
:10A6E000EE07A091EF07B091F007B7FF04C08150CB
:10A6F0009F4FAF4FBF4F892F9A2FAB2FBB27A7FD7F
:10A70000BA958093ED079093EE07A093EF07B0936F
:10A71000F0078091810390918203A0918303B0910F
:10A7200084032B813C814D815E81281B390B4A0BB0
:10A730005B0B2093C3033093C4034093C503509332
:10A74000C6038091790390917A03A0917B03B09125
:10A750007C03EF80F88409851A85E81AF90A0A0B48
:10A760001B0BE092C703F092C8030093C903109338
:10A77000CA032093CB033093CC034093CD03509373
:10A78000CE03E092CF03F092D0030093D103109355
:10A79000D20380915D0390915E03A0915F03B0911D
:10A7A0006003821B930BA40BB50B80935D03909306
:10A7B0005E03A0935F03B093600380915503909173
:10A7C0005603A0915703B09158038E199F09A00B0F
:10A7D000B10B8093550390935603A0935703B09306
:10A7E00058035D855523E1F020913D0330913E03F0
:10A7F000213831054CF0809192039091930301969A
:10A80000909393038093920320583F4F4CF4809190
:10A8100092039091930301979093930380939203F3
:10A8200010923E0310923D0381E090E09093E60386
:10A830008093E503E090CB03F090CC030091CD032F
:10A840001091CE03D801C70117FF07C088279927A9
:10A85000DC018E199F09A00BB10B81509240A040E2
:10A86000B04034F084E090E09093E6038093E503F9
:10A870008091EB039091EC03A091ED03B091EE0376
:10A88000209105083091060840910708509108086A
:10A89000821B930BA40BB50B815E914BAF4FBF4F47
:10A8A0008F539C49A040B04028F08091C70889315F
:10A8B0000CF4FFC0F1E0EF16F0E1FF06F0E00F0747
:10A8C000F0E01F070CF473C08091E703882309F4BC
:10A8D0006AC0D801C70117FF07C088279927DC0184
:10A8E0008E199F09A00BB10B9C01AD01B7FF04C0ED
:10A8F00021503E4F4F4F5F4FF9E0559547953795A3
:10A900002795FA95D1F78091E5039091E603820FA0
:10A91000931F9093E6038093E503D801C70117FFC7
:10A9200003C00796A11DB11DE3E0B595A7959795C6
:10A930008795EA95D1F78093D9039093DA03A09392
:10A94000DB03B093DC0389589341A040B04064F02E
:10A9500088E893E1A0E0B0E08093D9039093DA0314
:10A96000A093DB03B093DC032091D9033091DA0389
:10A970004091DB035091DC0357FF04C021503F4F4F
:10A980004F4F5F4F232F342F452F552747FD5A95A3
:10A990008091160390911703820F931F90931703D2
:10A9A0008093160306C081E08093E70302C01092F3
:10A9B000E70330E0E31630EFF3063FEF03073FEF26
:10A9C00013070CF073C08091E803882309F46AC070
:10A9D000D801C70117FF07C088279927DC018E1906
:10A9E0009F09A00BB10B9C01AD01B7FF04C0215022
:10A9F0003E4F4F4F5F4F69E05595479537952795E7
:10AA00006A95D1F78091E5039091E603820F931F39
:10AA10009093E6038093E503D801C70117FF03C0B5
:10AA20000796A11DB11D23E0B595A795979587952C
:10AA30002A95D1F78093D9039093DA03A093DB038F
:10AA4000B093DC0388579C4EAF4FBF4F64F488E748
:10AA50009CEEAFEFBFEF8093D9039093DA03A093FE
:10AA6000DB03B093DC032091D9033091DA034091EA
:10AA7000DB035091DC0357FF04C021503F4F4F4F81
:10AA80005F4F232F342F452F552747FD5A9580912F
:10AA9000160390911703820F931F909317038093CF
:10AAA000160311C081E08093E8030DC01092E80303
:10AAB0000AC01092E6031092E50384E690E09093BA
:10AAC000DB018093DA015D85252F33278091E50333
:10AAD0009091E6032817390724F43093E603209376
:10AAE000E5031091C708112379F0212F332727FDA3
:10AAF00030958091E5039091E6032817390724F4F7
:10AB00003093E6032093E5034091CB035091CC03AF
:10AB10006091CD037091CE034138510561057105F7
:10AB200074F080919603909197032091E503309102
:10AB3000E603820F931F90939703809396034058E8
:10AB40005F4F6F4F7F4F74F48091960390919703FE
:10AB50002091E5033091E603821B930B90939703BA
:10AB60008093960381E090E09093E6038093E50361
:10AB7000C090CF03D090D003E090D103F090D203E7
:10AB8000D701C601F7FE07C088279927DC018C1979
:10AB90009D09AE09BF0981509240A040B04034F0F9
:10ABA00084E090E09093E6038093E5038091EF03C7
:10ABB0009091F003A091F103B091F20320910F085E
:10ABC000309110084091110850911208821B930B8C
:10ABD000A40BB50B815E914BAF4FBF4F8F539C4978
:10ABE000A040B04018F019310CF4FFC001E0C016CD
:10ABF00000E1D00600E0E00600E0F0060CF473C0CF
:10AC00008091E903882309F46AC0D701C601F7FEE1
:10AC100007C088279927DC018C199D09AE09BF0957
:10AC20009C01AD01B7FF04C021503E4F4F4F5F4F15
:10AC300009E055954795379527950A95D1F7809165
:10AC4000E5039091E603820F931F9093E6038093B0
:10AC5000E503D701C601F7FE03C00796A11DB11D8C
:10AC600013E0B595A795979587951A95D1F7809399
:10AC7000DD039093DE03A093DF03B093E0038958D4
:10AC80009341A040B04064F088E893E1A0E0B0E0D8
:10AC90008093DD039093DE03A093DF03B093E00382
:10ACA0002091DD033091DE034091DF035091E003FA
:10ACB00057FF04C021503F4F4F4F5F4F232F342F7A
:10ACC000452F552747FD5A958091180390911903F8
:10ACD000820F931F909319038093180306C081E09D
:10ACE0008093E90302C01092E90320E0C21620EF2E
:10ACF000D2062FEFE2062FEFF2060CF073C0809120
:10AD0000EA03882309F46AC0D701C601F7FE07C029
:10AD100088279927DC018C199D09AE09BF099C0180
:10AD2000AD01B7FF04C021503E4F4F4F5F4FE9E0E8
:10AD30005595479537952795EA95D1F78091E50385
:10AD40009091E603820F931F9093E6038093E503AF
:10AD5000D701C601F7FE03C00796A11DB11D73E020
:10AD6000B595A795979587957A95D1F78093DD034B
:10AD70009093DE03A093DF03B093E00388579C4ECB
:10AD8000AF4FBF4F64F488E79CEEAFEFBFEF809307
:10AD9000DD039093DE03A093DF03B093E0032091E3
:10ADA000DD033091DE034091DF035091E00357FF54
:10ADB00004C021503F4F4F4F5F4F232F342F452F5B
:10ADC000552747FD5A958091180390911903820FDA
:10ADD000931F909319038093180311C081E080930F
:10ADE000EA030DC01092EA030AC01092E603109223
:10ADF000E50384E690E09093DB018093DA014D85D2
:10AE0000242F33278091E5039091E6032817390713
:10AE100024F43093E6032093E5038091C708882348
:10AE200079F0282F332727FD30958091E503909105
:10AE3000E6032817390724F43093E6032093E5034B
:10AE40004091CF035091D0036091D1037091D20310
:10AE5000413851056105710574F08091940390911A
:10AE600095032091E5033091E603820F931F9093A1
:10AE700095038093940340585F4F6F4F7F4FCCF4FE
:10AE800080919403909195032091E5033091E6031E
:10AE9000821B930B90939503809394030AC01092A6
:10AEA00019031092180310921703109216031092B0
:10AEB0003F0380911608882341F4109219031092E1
:10AEC00018031092170310921603809105089091B1
:10AED0000608A0910708B09108088093EB039093AF
:10AEE000EC03A093ED03B093EE0380910F089091D3
:10AEF0001008A0911108B09112088093EF0390936D
:10AF0000F003A093F103B093F20310927103109237
:10AF10007203109273031092740310926D031092D7
:10AF20006E0310926F0310927003109269031092D7
:10AF30006A0310926B0310926C0310920508109232
:10AF40000608109207081092080810920F08109235
:10AF5000100810921108109212081092FC0710921B
:10AF6000FD071092FE071092FF071092ED07109256
:10AF7000EE071092EF071092F00710924202109223
:10AF80004102E0902D03F0902E03C701F7FE04C0AC
:10AF9000882799278E199F0904973CF080915406C1
:10AFA00084FD03C082E38093D80310916006A12E34
:10AFB000BB24CC24DD24B701882777FD8095982F0A
:10AFC0009701F7FE04C0222733272E193F09442793
:10AFD00037FD4095542F0E94518D9B01AC01C60155
:10AFE000B5010E94518D97FF04C061507E4F8F4F75
:10AFF0009F4F59E095958795779567955A95D1F725
:10B000009B01812F99278E9DD0018F9DB00D9E9D14
:10B01000B00D1124CD01B7FD0396959587959595B3
:10B020008795280F391F80911A0390911B03280FD1
:10B03000391F442737FD4095542F2093BF03309389
:10B04000C0034093C1035093C20380915103909178
:10B050005203A0915303B0915403821B930BA40B92
:10B06000B50B8093510390935203A0935303B09375
:10B0700054038155934CA040B04064F080E593ECBC
:10B08000A0E0B0E08093510390935203A093530348
:10B09000B09354038091510390915203A0915303B4
:10B0A000B0915403805B9C43AF4FBF4F64F480EB7F
:10B0B0009CE3AFEFBFEF8093510390935203A093B3
:10B0C0005303B0935403C090DE01D090DF01D7FC4E
:10B0D00049C18091540683FF45C18091DD018150B3
:10B0E0008093DD01882309F041C18DE08093DD016B
:10B0F0008091810390918203A0918303B091840396
:10B10000B7FF04C081509E4FAF4FBF4F09E0B595C8
:10B11000A795979587950A95D1F72C0197FF04C0BD
:10B1200050944194510853948091790390917A03FB
:10B13000A0917B03B0917C03B7FF04C081509E4F68
:10B14000AF4FBF4F19E0B595A795979587951A957D
:10B15000D1F79C0197FF03C0309521953F4F4216D0
:10B1600053060CF42901B20157FE02C06D5F7F4FF8
:10B170003B0175946794759467940894611C711CE5
:10B18000ACE1EA2EA2E0FA2ECE0CDF1C76010027FD
:10B19000F7FC0095102F24EE3DEFC20ED31E8091D8
:10B1A000450890914608A0914708B09148088090C2
:10B1B000960190909701A0909801B0909901BC01E0
:10B1C000CD01A50194010E94C58DE21AF30A040B7A
:10B1D000150BC801B70128E631E040E050E00E94BD
:10B1E000C58DDC01CB018C01045B10408091DA013C
:10B1F0009091DB01009731F001979093DB018093F0
:10B20000DA0134C039E14316510484F580913D03DD
:10B2100090913E03800F911F90933E0380933D03D6
:10B220008091D803882311F181508093D80388231B
:10B23000E9F4C601AA2797FDA095BA2FBC01CD015C
:10B24000A50194010E94518DDC01CB01809345083A
:10B2500090934608A0934708B0934808BC01CD01DD
:10B260000E94C58D30934403209343038091DA01FB
:10B270009091DB01892B39F58091DC019927089F9A
:10B28000A001099F500D189F500D1124CA01B30150
:10B290000E94908D9B01442737FD4095542F80914B
:10B2A000450890914608A0914708B0914808820F40
:10B2B000931FA41FB51F8093450890934608A09341
:10B2C0004708B09348088091D803882309F04AC002
:10B2D00080914303909144037C010027F7FC009583
:10B2E000102F8091450890914608A0914708B09191
:10B2F0004808BC01CD01A50194010E94C58DE21A48
:10B30000F30A040B150B6CE172E080E090E0E60EAE
:10B31000F71E081F191FC801B70128E631E040E0F9
:10B3200050E00E94C58DDC01CB019C01245B3040C4
:10B330008091CA0186959927289FD001299FB00D39
:10B34000389FB00D11249D01B7FF02C0215F3F4F10
:10B35000F4E035952795FA95E1F730931B03209398
:10B360001A0304C010921B0310921A0380913F032A
:10B37000882381F01092490310924A0310924B03E4
:10B3800010924C0310924D0310924E0310924F03F3
:10B3900010925003F0901303FF20F1F480911608EF
:10B3A000282F3327442755278091810390918203CA
:10B3B000A0918303B0918403BC01CD010E94518D03
:10B3C000DC01CB01BC01CD0128EF3AE240E050E0C6
:10B3D0000E94C58D390102C066247724E0901203D3
:10B3E000EE20F1F480911608282F332744275527A3
:10B3F0008091790390917A03A0917B03B0917C03B3
:10B40000BC01CD010E94518DDC01CB01BC01CD01FD
:10B4100028EF3AE240E050E00E94C58D290102C0C9
:10B42000442455248091E6079091E707893C9105D3
:10B430001CF088EC90E005C088539F4F34F488E3FB
:10B440009FEF9093E7078093E6078091F207909132
:10B45000F307893C91051CF088EC90E005C0885307
:10B460009F4F34F488E39FEF9093F3078093F207A4
:10B470008091F4079091F507AA2797FDA095BA2F20
:10B4800020914308A22EBB24CC24DD24BC01CD0195
:10B49000A60195010E94518D9B01AC018091E607A8
:10B4A0009091E707AA2797FDA095BA2FE7E0880FAC
:10B4B000991FAA1FBB1FEA95D1F7280F391F4A1FF2
:10B4C0005B1F57FF04C0215C3F4F4F4F5F4F76E03B
:10B4D00055954795379527957A95D1F78301020FB2
:10B4E000131F1093F5070093F4078091E3079091E1
:10B4F000E407AA2797FDA095BA2FBC01CD01A601AC
:10B5000095010E94518D9B01AC018091F2079091B1
:10B51000F307AA2797FDA095BA2F67E0880F991F18
:10B52000AA1FBB1F6A95D1F7280F391F4A1F5B1F3F
:10B5300057FF04C0215C3F4F4F4F5F4F96E055953A
:10B540004795379527959A95D1F74201820E931E1C
:10B550009092E4078092E30780913E0890913F0823
:10B56000880F991FAA2797FDA095BA2F2091EC0765
:10B57000332744275527BC01CD010E94518D5B0123
:10B580006C0197FF08C02FE330E040E050E0A20ECE
:10B59000B31EC41ED51E86E0D594C794B794A79455
:10B5A0008A95D1F780910208282F33274427552701
:10B5B0008091650390916603A0916703B091680341
:10B5C000BC01CD010E94518DDC01CB01BC01CD013C
:10B5D00020EF35E540E050E00E94C58DB501620FD7
:10B5E000731F70933F0860933E080150104134F080
:10B5F00080E090E19093F5078093F4078091F40741
:10B600009091F5078050904F34F480E090EF909344
:10B61000F5078093F40751E0851650E1950634F064
:10B6200080E090E19093E4078093E3078091E30743
:10B630009091E4078050904F34F480E090EF909325
:10B64000E4078093E3076150704134F080E090E1BB
:10B6500090933F0880933E0880913E0890913F0868
:10B660008050904F34F480E090EF90933F088093A7
:10B670003E0880910001482F552780911E0190912E
:10B680001F014817590794F420911E0130911F01A2
:10B6900009811A81049FC001059F900D149F900D90
:10B6A0001124B9010E947C8D7A83698329813A81B2
:10B6B000220F331F220F331F3A83298340915406F0
:10B6C00040FF92C7EE2009F08FC7FF2009F08CC71A
:10B6D000AA24BB24450180911403909115039093F3
:10B6E0001D0680931C062091980330919903211523
:10B6F000310509F03FC080911401909115018959DD
:10B70000934058F087B5803F20F4809145028150E6
:10B7100011C081E08093FE034EC08091140190918E
:10B7200015018436910508F587B58031D0F08091F8
:10B7300045028F5F809345029FE0890290011124AA
:10B7400080914306821B87BD8CE291E09093330287
:10B75000809332028EE591E0909399038093980351
:10B760002AC081E08093FD0326C0F092FD03F09291
:10B77000FE0321C08091250390912603A091270309
:10B78000B091280314E0880F991FAA1FBB1F1A95B8
:10B79000D1F78093460290934702A0934802B0935A
:10B7A0004902B0924402A0924302215030403093AB
:10B7B0009903209398032091CD0141FF24C02233A7
:10B7C000D8F48091E80181508093E8018F3FD9F54A
:10B7D000109240038091250390912603A0912703A6
:10B7E000B09128038093210390932203A093230315
:10B7F000B093240381E004C081E08093400388EC8F
:10B800008093E80120C080919A0190919B01820F62
:10B81000911D209159063327829FA001839F500DCF
:10B82000929F500D1124CA01AA2797FDA095BA2F07
:10B830008093210390932203A0932303B0932403C6
:10B8400081E0809340038091810390918203A091D5
:10B850008303B0918403E0909601F09097010091EA
:10B86000980110919901BC01CD01A80197010E9496
:10B87000C58D59016A018091790390917A03A09155
:10B880007B03B0917C03BC01CD01A80197010E940C
:10B89000C58DB901C5010E9498838C01CC9714F025
:10B8A0000CE310E0C8010E94806E8C0180E280935E
:10B8B000950180914003882309F408C58091F8021E
:10B8C00099279C012071307084FD00C58091F7029A
:10B8D00082608093F7027091AD0670FD04C0809184
:10B8E000540681FD0CC0C980DA803093F4032093A4
:10B8F000F3038091F802806C8093F80255C2809126
:10B90000F80281FF27C24091E4015091E501CA018C
:10B910000F9620912B0330912C0382179307BCF5CF
:10B920006091FD03662399F58091F80287FF15C0A9
:10B930008091F8028F778093F8028091250390918F
:10B940002603A0912703B0912803809321039093AD
:10B950002203A0932303B09324038091F802806410
:10B960008093F802241B350B2F50304037FF03C063
:10B97000309521953F4F8091F3039091F403820F0E
:10B98000931F9093F4038093F3038BE23BC0CA01AF
:10B990000F9728173907DCF56091FE036623B9F588
:10B9A0008091F80286FF15C08091F8028F7B80930A
:10B9B000F8028091250390912603A0912703B0916E
:10B9C00028038093210390932203A0932303B09331
:10B9D00024038091F80280688093F802241B350BC1
:10B9E000215F3F4F37FF03C0309521953F4F809136
:10B9F000F3039091F403821B930B9093F4038093D1
:10BA0000F3038DE2809395016093FF03BFC08DE344
:10BA10008093950160911C03662391F120911D0391
:10BA200030911E0340911F03509120038091210308
:10BA300090912203A0912303B091240382179307CE
:10BA4000A407B507ECF48091F80280648093F802B3
:10BA50008091F3039091F403860F911D9093F4036A
:10BA60008093F3038AE08093FF038EE58093950132
:10BA70008091F80287FF8AC08091F8028F7734C0E6
:10BA8000662309F444C020911D0330911E034091A8
:10BA90001F03509120038091210390912203A091D4
:10BAA0002303B0912403281739074A075B077CF565
:10BAB0008091F80280688093F8028091F30390915E
:10BAC000F403861B91099093F4038093F30386EFAC
:10BAD0008093FF0386E7809395018091F80286FFAB
:10BAE00055C08091F8028F7B8093F80280912503E6
:10BAF00090912603A0912703B091280380932103FE
:10BB000090932203A0932303B09324033FC080911A
:10BB1000F802807CD9F18091FF03882389F4809119
:10BB2000250390912603A0912703B09128038093C9
:10BB3000210390932203A0932303B093240302C014
:10BB40001092FF038091F8028F738093F802109295
:10BB5000F4031092F30371FF06C084EF91E0909319
:10BB600033028093320280912903882379F48091F3
:10BB7000250390912603A0912703B0912803C39732
:10BB8000A105B1051CF081E0809329032091F30306
:10BB90003091F403C90137FF04C088279927821B1D
:10BBA000930B815092400CF4BEC04091FF0344239C
:10BBB000E9F080911D0390911E03209121033091A3
:10BBC0002203821B930B0996439748F480911D032F
:10BBD00090911E03A0911F03B091200327C0242F32
:10BBE000332727FD3095432F532F14C080915906DA
:10BBF0009927289FB001299F700D389F700D11243F
:10BC0000CB0160E075E00E94908D9B01442737FDD9
:10BC10004095542F8091210390912203A0912303FA
:10BC2000B0912403820F931FA41FB51F809321039B
:10BC300090932203A0932303B09324031092F40360
:10BC40001092F303C0902503D0902603E0902703C1
:10BC5000F0902803D701C60180509440A040B04026
:10BC6000209121033091220340912303509124031A
:10BC700082179307A407B5075CF4D701C60180506B
:10BC80009C4FAF4FBF4F281739074A075B0744F057
:10BC90008093210390932203A0932303B093240362
:10BCA0008091AD0681FF06C084E690E09093330258
:10BCB0008093320280915D068823A9F580911C0350
:10BCC000882389F5409114035091150357FF02C052
:10BCD0004D5F5F4F559547955595479580911E014E
:10BCE00090911F01209100013327489FD001499F67
:10BCF000B00D589FB00D1124CD01B9010E94908D57
:10BD00007093E5016093E401663471051CF486E4E8
:10BD100090E005C06739710534F086E990E09093B2
:10BD2000E5018093E4018091980390919903892B18
:10BD3000B9F18091250390912603A0912703B0913A
:10BD400028038093210390932203A0932303B093AD
:10BD5000240326C08091250390912603A0912703F8
:10BD6000B091280380599140A040B04080932103B6
:10BD700090932203A0932303B093240380915D0644
:10BD8000882311F0992702C088E790E09093E5019D
:10BD90008093E401E981FA81F0931503E0931403A1
:10BDA000C0901403D09015032091250330912603F1
:10BDB00040912703509128032C8B3D8B4E8B5F8B3A
:10BDC00020912103309122034091230350912403B9
:10BDD0006C897D898E899F892617370748075907FF
:10BDE00024F08091AD0680FDBDC2809198039091B2
:10BDF0009903892B39F0C0901403D0901503AA241D
:10BE0000BB24D9C08C899D89AE89BF89821B930BC5
:10BE1000A40BB50B8093C3039093C403A093C503F5
:10BE2000B093C603823070E897077FEFA7077FEFD4
:10BE3000B7072CF481E090E8AFEFBFEF09C08F5F48
:10BE40009F47A040B04064F08FEF9FE7A0E0B0E0D4
:10BE50008093C3039093C403A093C503B093C60318
:10BE6000A090C303B090C4038091CC01282F332746
:10BE7000442755278091C3039091C403A091C50323
:10BE8000B091C603BC01CD010E94518D97FF04C043
:10BE9000615E7F4F8F4F9F4FA5E095958795779572
:10BEA0006795AA95D1F76093C3037093C4038093F9
:10BEB000C5039093C6036530FEEF7F07FFEF8F0742
:10BEC000FFEF9F072CF484E09EEFAFEFBFEF09C0B8
:10BED000605074408040904064F080E094E0A0E0C6
:10BEE000B0E08093C3039093C403A093C503B093C1
:10BEF000C6038090C3039090C40320914302309105
:10BF0000440237FF02C0295F3F4FF3E03595279584
:10BF1000FA95E1F74FEF223834071CF421E83FEFA0
:10BF200005C02038310514F020E830E0C901AA2707
:10BF300097FDA095BA2F2091CE013327442755278E
:10BF4000BC01CD010E94518D97FF04C06D5F7F4FF2
:10BF50008F4F9F4FE2E09595879577956795EA9586
:10BF6000D1F79B015FEF613075071CF420E03FEFD4
:10BF700006C06F3F710519F014F020E031E08091A8
:10BF8000F802807C49F0C90137FD03969C01359584
:10BF90002795359527950DC08091AD0680FF09C086
:10BFA000C90137FD07969C0143E0359527954A95D1
:10BFB000E1F7820E931E2091CB01222309F454C095
:10BFC0006091450370914603809147039091480327
:10BFD00097FF04C061587F4F8F4F9F4F37E0959573
:10BFE0008795779567953A95D1F733274427552755
:10BFF0000E94518D97FF04C0615E7F4F8F4F9F4F0E
:10C00000B5E09595879577956795BA95D1F7609343
:10C01000C3037093C4038093C5039093C603613830
:10C02000AFEF7A07AFEF8A07AFEF9A072CF480E8FB
:10C030009FEFAFEFBFEF0AC06F3F7105810591051C
:10C0400069F064F080E091E0A0E0B0E08093C30389
:10C050009093C403A093C503B093C6038091C30318
:10C060009091C403880E991E8091C901282F33270F
:10C070008091CA08992787FD9095289FF001299FF4
:10C08000F00D389FF00D11249F01F7FF02C02158D9
:10C090003F4F220F232F221F330BFFEF21383F0783
:10C0A0001CF420E83FEF06C02F3F310519F014F0D3
:10C0B00020E031E0820E931EC401AA2797FDA095CF
:10C0C000BA2FE0901403F09015039701442737FD31
:10C0D0004095542FBC01CD010E94518D97FF04C0A3
:10C0E00061507E4F8F4F9F4FF9E0959587957795DB
:10C0F0006795FA95D1F7C61AD70A8091F303909104
:10C10000F403892B09F060C01E141F040CF05CC0FE
:10C110009501B7FE03C0309521953F4F2D33310572
:10C1200040F48091F7039091F8038C159D0574F508
:10C1300026C02C533040E5E036952795EA95E1F787
:10C140002031310510F02FE030E04091F70350919D
:10C15000F8031A141B04E4F480E190E0821B930BB3
:10C16000489F9001499F300D589F300D112474E075
:10C17000369527957A95E1F72C153D0520F58091A8
:10C18000E6019091E701C816D906F4F06C011CC0D5
:10C19000205F3F4F8091E6019091E701829FB001BF
:10C1A000839F700D929F700D11249B0164E0369562
:10C1B00027956A95E1F74C155D0514F06A0104C0F6
:10C1C000C216D30608F06901C601AA2797FDA095FB
:10C1D000BA2F2DE0880F991FAA1FBB1F2A95D1F7F0
:10C1E0009801442737FD4095542FBC01CD010E9492
:10C1F000C58D2093C7033093C8034093C903509360
:10C20000CA03C090C703D090C8038091F5039091F2
:10C21000F6039C01220F331F280F391F2C0D3D1DE3
:10C2200037FF02C02D5F3F4FA901559547955595A2
:10C2300047955093F6034093F50380915506282FB8
:10C240003327220F331F220F331F241735076CF4B7
:10C2500080913B08282F3327220F331F220F331FD3
:10C26000205530404217530724F03093F6032093B3
:10C27000F5038091AD0680FF14C08091F503909185
:10C28000F603A981BA818A179B0724F0B093F603BD
:10C29000A093F503E091F503F091F603FA83E983A7
:10C2A00061C029813A812E193F0937FF02C02D5FF5
:10C2B0003F4F3595279535952795E090F503F090FC
:10C2C000F603E20EF31EFA82E9824CC080915D060D
:10C2D000882301F5609114037091150377FF02C064
:10C2E0006D5F7F4F759567957595679540911E01B8
:10C2F00050911F0180910001282F3327649FC001B6
:10C30000659F900D749F900D1124B9010E94908D2E
:10C31000CB0101C099279093E5018093E4018091BE
:10C32000E4019091E501873491051CF486E490E0E6
:10C3300005C08639910534F086E990E09093E501D7
:10C340008093E40129813A813093F6032093F50329
:10C350008091F802806C8093F8028091F7028D7FC3
:10C360008093F7028091F80299279C012270307027
:10C3700081FF2BC18091F9039091FA03A091FB03F7
:10C38000B091FC030097A105B10521F0809129032C
:10C390008130B1F449815A81CA01AA2797FDA0953D
:10C3A000BA2F2EE0880F991FAA1FBB1F2A95D1F71D
:10C3B0008093F9039093FA03A093FB03B093FC03DB
:10C3C00080912903813019F482E0809329036981E7
:10C3D0007A81CB01AA2797FDA095BA2F980144270F
:10C3E00037FD4095542FBC01CD010E94518DDC01D9
:10C3F000CB018093C7039093C803A093C903B09364
:10C40000CA03B7FF04C08150904EAF4FBF4F7C01AD
:10C410008D01FDE015950795F794E794FA95D1F70E
:10C42000E092C703F092C8030093C9031093CA03B4
:10C430006091F9027091FA028FE0603A780750F546
:10C440008091F9039091FA03A091FB03B091FC0352
:10C450009C01AD01EAE05695479537952795EA95F9
:10C46000D1F7821B930BA40BB50BA8019701F4E045
:10C47000220F331F441F551FFA95D1F7820F931FC8
:10C48000A41FB51F8093F9039093FA03A093FB03B5
:10C49000B093FC0360547F4118F58091F9039091AB
:10C4A000FA03A091FB03B091FC039C01AD01ECE009
:10C4B0005695479537952795EA95D1F7821B930BAB
:10C4C000A40BB50BA801970172E0220F331F441F84
:10C4D000551F7A95D1F7820F931FA41FB51F38C03F
:10C4E00080914302909144028091430290914402D2
:10C4F00097FF03C0909581959F4F8436910584F5F1
:10C5000080912503909126032091210330912203ED
:10C51000821B930B81509F4F8F5F914008F5809154
:10C52000F9039091FA03A091FB03B091FC039C01E5
:10C53000AD016EE056954795379527956A95D1F7E9
:10C54000821B930BA40BB50B8E0D9F1DA01FB11F5B
:10C550008093F9039093FA03A093FB03B093FC0339
:10C560008091F9039091FA03A091FB03B091FC0331
:10C570001EE0B695A795979587951A95D1F7909354
:10C5800015038093140340915B06442399F05527CB
:10C590009C01BA010E94908DC901861B970B909354
:10C5A000F8038093F703260F371F3093E70120939A
:10C5B000E6011FC01092F8031092F7038FEF93E08B
:10C5C0009093E7018093E60114C010922903109222
:10C5D000F9031092FA031092FB031092FC033093BC
:10C5E00015032093140305C08091F802806C80939A
:10C5F000F8022090FA07222D3327220F331F220F33
:10C60000331F285D3F4FE981FA812E173F0714F051
:10C610003A83298330903B08832D9927880F991FEF
:10C62000880F991F80559040E980FA808E159F05EC
:10C6300014F49A83898380917B02882321F480916A
:10C64000D1088F3FA1F08091F9029091FA020297F0
:10C65000C09768F409811A811016110644F481E02C
:10C6600090E09093FA028093F9023A83298329811A
:10C670003A8130930106209300068091BF03909188
:10C68000C003A091C103B091C203F2E0880F991FCB
:10C69000AA1FBB1FFA95D1F700913E0810913F08E1
:10C6A000081B190B213A31058CF0C90137FD0196A1
:10C6B00095958795801791070CF48C01909581953D
:10C6C0009F4F081719076CF48C010BC00135110539
:10C6D00014F000E510E03FEF003B130714F400EB0B
:10C6E0001FEF232D3327220F331F220F331FC901C2
:10C6F00049815A81841B950B801791070CF48C019A
:10C7000069817A81621B730B061717070CF48B0182
:10C710008091F4079091F507609131037091320395
:10C72000861B970B9093040880930308D0901608FB
:10C7300020914D0330914E0340914F03509150038F
:10C74000DD2041F0661A770AC301AA2797FDA0955C
:10C75000BA2F04C0AA2797FDA095BA2F280F391F1A
:10C760004A1F5B1F20934D0330934E0340934F03AA
:10C770005093500380914D0390914E03A0914F032D
:10C78000B091500381509A4FA040B04064F080E0D7
:10C790009AEFA0E0B0E080934D0390934E03A093F6
:10C7A0004F03B093500380914D0390914E03A0919D
:10C7B0004F03B091500380509640AF4FBF4F64F489
:10C7C00080E096E0AFEFBFEF80934D0390934E0370
:10C7D000A0934F03B0935003C0906A0620910308C2
:10C7E00030910408F8E0FC1598F08C2D9927829F71
:10C7F0007001839FF00C929FF00C1124C701F7FC8D
:10C8000007967C0163E0F594E7946A95E1F712C01E
:10C810008C2D86959927829FA001839F500D929F12
:10C82000500D1124CA0157FD03967C01F594E7943D
:10C83000F594E794A090CF01B090D00195014427E2
:10C8400037FD4095542F80914D0390914E03A09158
:10C850004F03B0915003BC01CD010E94C58DE20E83
:10C86000F31E9090BB01692D77278827992798019F
:10C8700017FF04C022273327201B310B37FF02C0CC
:10C880002F5F3F4F35952795A981BA812A0F3B1F0E
:10C89000442737FD4095542F0E94518D97FF04C0C7
:10C8A000615C7F4F8F4F9F4F26E0959587957795D9
:10C8B00067952A95D1F79B016E157F050CF47B01D6
:10C8C000309521953F4FE216F3060CF479018091E3
:10C8D000E3079091E40760912F0370913003861B6A
:10C8E000970B9093E2078093E107209149033091E1
:10C8F0004A0340914B0350914C03DD2041F0461A0E
:10C90000570AC201AA2797FDA095BA2F04C0AA27EB
:10C9100097FDA095BA2F280F391F4A1F5B1F209340
:10C92000490330934A0340934B0350934C03809147
:10C93000490390914A03A0914B03B0914C0381505D
:10C940009A4FA040B04064F080E09AEFA0E0B0E0E1
:10C950008093490390934A03A0934B03B0934C03F5
:10C960008091490390914A03A0914B03B0914C03ED
:10C9700080509640AF4FBF4F64F480E096E0AFEF39
:10C98000BFEF8093490390934A03A0934B03B09366
:10C990004C032091E1073091E20748E04C1598F0F4
:10C9A0008C2D9927829FB001839F700D929F700DEF
:10C9B0001124CB0177FD07966C01B3E0D594C794A1
:10C9C000BA95E1F712C0C6948C2D9927829FD001A9
:10C9D000839FB00D929FB00D1124CD01B7FD03963A
:10C9E0006C01D594C794D594C7949501442737FD1D
:10C9F0004095542F8091490390914A03A0914B0395
:10CA0000B0914C03BC01CD010E94C58DC20ED31E56
:10CA1000692D772788279927980117FF04C02227B7
:10CA20003327201B310B37FF02C02F5F3F4F359557
:10CA30002795E981FA812E0F3F1F442737FD409546
:10CA4000542F0E94518D97FF04C0615C7F4F8F4F20
:10CA50009F4FE6E09595879577956795EA95D1F78D
:10CA60009B016C157D050CF46B01309521953F4FB2
:10CA7000C216D3060CF469014090070361E1862ECB
:10CA800067E0962E58ECA52E56E0B52E4BE0542EBE
:10CA900039E1632E38E0732ED5012C9112160CF07B
:10CAA00027C1203429F4E981FA81F98FE88F1FC06A
:10CAB00049815A81CA01AA2797FDA095BA2F332729
:10CAC00027FD3095432F532FBC01CD010E94518D7E
:10CAD00097FF04C0615C7F4F8F4F9F4F26E0959575
:10CAE0008795779567952A95D1F7798F688FF501A6
:10CAF0002181203439F4288D398D2E0D3F1D398F39
:10CB0000288F2AC0203C39F4488D598D4E195F0971
:10CB1000598F488F21C0C701AA2797FDA095BA2F2A
:10CB2000332727FD3095432F532FBC01CD010E94A1
:10CB3000518D97FF04C0615C7F4F8F4F9F4FB6E0D0
:10CB40009595879577956795BA95D1F7A88DB98D05
:10CB5000A60FB71FB98FA88FF5012281203439F4B1
:10CB6000288D398D2C0D3D1D398F288F2AC0203CF2
:10CB700039F4488D598D4C195D09598F488F21C062
:10CB8000C601AA2797FDA095BA2F332727FD309518
:10CB9000432F532FBC01CD010E94518D97FF04C03C
:10CBA000615C7F4F8F4F9F4FA6E095958795779556
:10CBB0006795AA95D1F7A88DB98DA60FB71FB98F24
:10CBC000A88FF5012381203439F4288D398D200F69
:10CBD000311F398F288F2AC0203C39F4488D598D58
:10CBE000401B510B598F488F21C0C801AA2797FDC0
:10CBF000A095BA2F332727FD3095432F532FBC0123
:10CC0000CD010E94518D97FF04C0615C7F4F8F4F13
:10CC10009F4FF6E09595879577956795FA95D1F7AB
:10CC2000A88DB98DA60FB71FB98FA88FF30180818A
:10CC30009181288D398D8217930764F4B901680FAB
:10CC4000791F77FF02C06F5F7F4F75956795798F6A
:10CC5000688F1BC031E0341548F0488D598D440F62
:10CC6000551F481B590B598F488F0FC0242D332750
:10CC7000688D798D861B970BB9010E94908DA88DC8
:10CC8000B98DA60FB71FB98FA88F822D9927880F4E
:10CC9000991F880F991FE88DF98D8E179F075CF4F7
:10CCA000832D9927880F991F880F991F288D398DFB
:10CCB0002817390714F0998F888F888D998D97FDE3
:10CCC00003969595879595958795F4018183880FAF
:10CCD000991F880F991F288D398D281B390BC90181
:10CCE000880F8283E88DF98DD301ED93FC9303C007
:10CCF000F401118212825A9422E030E0620E731E17
:10CD000044E050E0A40EB51E68E070E0860E971E69
:10CD100057FEC2CEE2E1C75E0C94FC8D80910C04FC
:10CD200090910D04A0910E04B0910F04809304041F
:10CD300090930504A0930604B0930704809108041F
:10CD400090910904A0910A04B0910B04809300040F
:10CD500090930104A0930204B093030408951092E9
:10CD600017041092160410921504109214040895DA
:10CD700084B1806A84B93D9A82E58CBD1DBC459A18
:10CD800081E0809350088AEA8093610883E8809369
:10CD900062088AE080936308109265081092640824
:10CDA00010926708109266081092C90810928508C0
:10CDB000089530915008332309F085C00DB407FE63
:10CDC00082C084E080933102459A2EB5809123047D
:10CDD00099278130910589F0823091051CF4892BC7
:10CDE00021F03EC00297B9F03BC0309384082093F5
:10CDF00024042138A9F581E008C0253549F4809143
:10CE00002404820F8093240482E08093230428C0AA
:10CE10003093230425C080918408E82FFF27EA552A
:10CE2000F74F20838F5F8093840890912404803291
:10CE3000A0F0291769F480E2A6EAB8E0E6E8F8E095
:10CE40000D9001928A95E1F781E08093850802C0F8
:10CE5000309385081092230403C0920F909324040A
:10CE600020916008223208F028C045980000000098
:10CE700000000000000000000000000000000000B2
:10CE800000000000000000000000000000000000A2
:10CE9000000000000000000000000000E0915908C0
:10CEA000F0915A08E20FF11D80818EBD80918208B9
:10CEB0009081890F8093820803C081E0809350089D
:10CEC0002F5F209360080895EF92FF920F931F93B6
:10CED000809163069927880F991F880F991F7C01FD
:10CEE0000027F7FC0095102F809181039091820319
:10CEF000A0918303B0918403BC01CD01A8019701E7
:10CF00000E94C58D30936508209364088091790351
:10CF100090917A03A0917B03B0917C03BC01CD0179
:10CF2000A80197010E94C58D309367082093660879
:10CF30002091450830914608409147085091480893
:10CF4000DA01C90103E0880F991FAA1FBB1F0A95C8
:10CF5000D1F7820F931FA41FB51F820F931FA41F29
:10CF6000B51F209196013091970140919801509101
:10CF70009901BC01CD010E94C58D30936D082093AD
:10CF80006C0880919203909193032091510230910B
:10CF90005202821B930B9093730880937208E09166
:10CFA0008803F091890380910C0890910D08BF01CE
:10CFB0000E94908D9B01220F331F220F331F260FDB
:10CFC000371F260F371F37FF02C02D5F3F4F3595A4
:10CFD00027953595279530936908209368088091A7
:10CFE000410890914208BF010E94908D9B01220F41
:10CFF000331F220F331F260F371F260F371F37FF10
:10D0000002C02D5F3F4F3595279535952795309375
:10D010006B0820936A08109289031092880310927B
:10D020000D0810920C08109242081092410880914D
:10D03000630899278D30910509F46CC08E309105F5
:10D040005CF48B30910509F494C08C3091050CF0A0
:10D0500015C10A9761F0B3C18F30910509F487C1FA
:10D060008F3091050CF462C14097A9F1A8C180915D
:10D070000D038093760880910C038093770880914C
:10D080000B038093780880910A038093790880913C
:10D09000090380937A088091080380937B0880912C
:10D0A000070380937C088091060380937D0880911C
:10D0B000F80280937E088091F802837F8093F802C3
:10D0C0000E941B3080937F088091850380938008A5
:10D0D0008091F70228C18091CB089091CC08909361
:10D0E0007708809376088091CF089091D00890932C
:10D0F00079088093780880911E0190911F01809398
:10D100007A088091000180937B088091950180933B
:10D110007C0855C180919706809376088091980687
:10D1200080937708809199068093780880919A0679
:10D130008093790880919B0680937A0880919F065E
:10D1400080937B088091A00680937C088091A10643
:10D1500080937D088091A40680937E088091A2062A
:10D1600080937F088091A306809380088091A50614
:10D17000DAC0F89480914A06E82FFF27EE0FFF1FD0
:10D18000EE58F84F0190F081E02DE038F1051CF0E9
:10D19000EFE7F0E006C02FEFE138F20714F4E1E822
:10D1A000FFEFE093760880914B06E82FFF27EE0F04
:10D1B000FF1FEE58F84F0190F081E02DE038F105A7
:10D1C0001CF0EFE7F0E006C06FEFE138F60714F46B
:10D1D000E1E8FFEFE093770880914906E82FFF2709
:10D1E000EE0FFF1FEE58F84F0190F081E02DE03870
:10D1F000F1051CF0EFE7F0E006C08FEFE138F8072B
:10D2000014F4E1E8FFEFE093780880914806E82FF6
:10D21000FF27EE0FFF1FEE58F84F0190F081E02D31
:10D22000E038F1051CF0EFE7F0E006C02FEFE13841
:10D23000F20714F4E1E8FFEF7894E0937908809125
:10D24000340380937A088091350380937B08809122
:10D25000360380937C088091370380937D0880910A
:10D26000380380937E088091390380937F088091F2
:10D270003A038093800880913B0355C080918B04D2
:10D28000863018F010928B0485E0809376088091A8
:10D29000A606809377088091250390912603A0919C
:10D2A0002703B0912803BC01CD0125E030E040E028
:10D2B00050E00E94C58D30937908209378088091C2
:10D2C000210390912203A0912303B0912403BC0178
:10D2D000CD0125E030E040E050E00E94C58D309364
:10D2E0007B0820937A0880919C0680937C0880912B
:10D2F0009D0680937D0880919E0680937E08809194
:10D30000330380937F088091720790917307809315
:10D310008008809100069091010697FD03969595EF
:10D320008795959587958093810849C010927608D6
:10D3300084E5809377081092780883E180937908D8
:10D340008091020180937A088091700480937B0819
:10D350008091710480937C088091720480937D0891
:10D360008091730480937E088091740426C080911C
:10D370007C06809376088091AC0680937708809134
:10D38000C101809378088091750680937908809117
:10D39000760680937A088091770680937B08809147
:10D3A000C00180937C088091790680937D088091EC
:10D3B0007A0680937E0880917B0680937F08809117
:10D3C0008508882309F44DC18AEF8093F20181E03A
:10D3D0008093DD014091870850918808CA018150EF
:10D3E0009E4F8F5F9340B0F42091890830918A0856
:10D3F000C90181509E4F8F5F934060F48091540625
:10D4000085FF08C050931704409316043093150409
:10D410002093140480918F089091900890931904A0
:10D4200080931804809191089091920890931B0426
:10D4300080931A04809193089091940890931D040E
:10D4400080931C0480918D0890918E0821E089368C
:10D45000920724F49093DF018093DE018091DE0136
:10D460009091DF012091430330914403821B930B81
:10D47000845E9D4F68E671E00E94908D845B9040D1
:10D48000909342038093410320919708309198082C
:10D4900080913202909133028217930720F43093E7
:10D4A00033022093320280918608992788369105AD
:10D4B00009F460C08936910524F48736910531F06E
:10D4C000D8C08936910509F47CC0D3C080919908F1
:10D4D0008093C60880919A088093C80880919B0821
:10D4E0008093C70880919C088093C90880919D080B
:10D4F0008093CA0880919E088093F30180919F08D1
:10D5000080932204809105038823F9F02091A108DB
:10D510003091A20837FD19C0309344032093430390
:10D5200090917E06992389F08FE0989FC001112485
:10D53000281B390BC90188599E4F68E671E00E948B
:10D54000908D909344038093430320911E04309167
:10D550001F048091A3089091A408280F391F37FF5A
:10D5600002C02F5F3F4F3595279530931F042093BE
:10D570001E047FC08091990880935B0880919A086F
:10D5800080935C0880919B0880935D0880919C0843
:10D5900080935E0880919D0880935F088091F005DC
:10D5A00090919E08892B8093F00590919F0890930D
:10D5B00020048091F10583709C70892B8093F10584
:10D5C00058C0809199088093510880919A0880935F
:10D5D000520880919B088093530880919C08809307
:10D5E000540880919D0890919E08909356088093CE
:10D5F000550880919F089091A008909358088093B7
:10D6000057088091A108992787FD90959093A507C9
:10D610008093A4078091A20880931C038091A308A3
:10D620009091A4089C01442737FD4095542FDA01BE
:10D63000C90163E0880F991FAA1FBB1F6A95D1F724
:10D64000820F931FA41FB51F820F931FA41FB51F26
:10D6500080931D0390931E03A0931F03B093200398
:10D6600008C010921704109216041092150410921C
:10D6700014041F910F91FF90EF900895809150082E
:10D68000882309F43BC0459881E698E090935A08B6
:10D690008093590890912104E92FFF27E751FE4F0D
:10D6A0009F5F90932104808180936308993010F0EC
:10D6B00010922104109250080E94646781E08093C8
:10D6C00060080000000000000000000000000000F2
:10D6D000000000000000000000000000000000004A
:10D6E000000000000000000000000000000000003A
:10D6F000000080916108809382088EBD089587B1F3
:10D700008C6087B91092260480E88093F50110920E
:10D7100025048093F401089580912B048150809317
:10D720002B048F3F09F0FBC024E020932B04809151
:10D73000F802992780739070892B21F480917104ED
:10D7400080FF1CC080919506882349F080912E04AB
:10D75000882311F42093260481E080932E04809185
:10D7600096068823B9F080912F04882319F484E069
:10D770008093250481E080932F040CC010922E0426
:10D7800010922F048091910680932C04809193062F
:10D7900080932D0480912E04882309F040C080914D
:10D7A000AB06282F332724FF07C080912A03882344
:10D7B00019F425FD4DC04EC090919206983F50F04F
:10D7C00080910E088D3D30F080912C0488230CF45C
:10D7D0003FC040C0983F48F080910E088A3028F43E
:10D7E00080912C048823B4F133C0809126048150A9
:10D7F000809326048F3F79F580910E0881508093A5
:10D8000026048091F501813011F480E801C08695ED
:10D810008093F5018091F50190912C0417C08091BF
:10D8200026048150809326048F3FA9F489E08093D9
:10D8300026048091F501813011F480E801C08695BD
:10D840008093F5018091F50190919506892311F05F
:10D85000429A01C0429880912F04882309F043C066
:10D860008091AB06282F332724FF07C080912A031D
:10D87000882319F426FD50C034C090919406983F37
:10D8800050F080913A088D3D30F080912D0488232E
:10D890000CF442C026C0983F48F080913A088A3084
:10D8A00028F480912D048823E4F036C0809125046B
:10D8B0008150809325048F3F91F580913A088150E3
:10D8C000809325048091F401813011F480E801C037
:10D8D00086958093F4018091F40190912D04892321
:10D8E000D9F44398089580912504815080932504AC
:10D8F0008F3FA9F489E0809325048091F401813061
:10D9000011F480E801C086958093F4018091F401C0
:10D9100090919606892311F0439A089543980895AB
:10D920004FB724E130E0F8948091C9008F7780935D
:10D93000C9008091C9008F7B8093C9008091C90084
:10D940008F7D8093C9005A9A52985B9A539A832F7D
:10D9500099278093CD002093CC008091C8008260ED
:10D960008093C80080E18093C9008091CA008F77BE
:10D970008093CA008091CA008F7B8093CA008091F7
:10D98000CA008F7D8093CA008091CA008F7E8093E9
:10D99000CA008091CA00877F8093CA008091C90025
:10D9A0008B7F8093C9008091CA0084608093CA00F5
:10D9B0008091CA0082608093CA008091C80087FF6E
:10D9C00003C08091CE00F9CF8091C9008068809318
:10D9D000C9004FBF0895EF92FF920F931F93CF930B
:10D9E000DF93482F00E010E08091F601813061F470
:10D9F0001092F60184E48093300410923204109265
:10DA00003104109233042BC180913004882319F41F
:10DA100021E030E001C0980190913104992371F424
:10DA2000232B11F081E010C084E4809330049093A4
:10DA300032049093310490933304FAC0913069F426
:10DA4000232B09F0EBC082E08093310480913204F3
:10DA50008F5F8093320483E0E9C09230D1F4232BAE
:10DA600009F0DCC083E0809330044093330490914C
:10DA70003204923039F41092340447FF03C081E03D
:10DA80008093340483E0809331049F5F9093320449
:10DA9000CFC0933009F0C2C0232B09F0BFC09093D0
:10DAA000300482E080933104809132048F5F809350
:10DAB000320420913304822F9927782F6627842FF0
:10DAC0009927682B792B80916E06813049F4737009
:10DAD000CB018050924063E070E00E94908D17C0AF
:10DAE000823061F47770CB018050944066E070E042
:10DAF0000E94908D2695269526950BC073706856CA
:10DB00007140CB0177FD0196BC017595679526950F
:10DB10002695022F11270F7010700F5F1F4F0D30C9
:10DB2000110508F074C07801E00EF11EF701EE58FF
:10DB3000F84F808191819B01281B390BC90137FF68
:10DB400003C0909581959F4F069794F4809133037D
:10DB5000883C30F480913303865F8093330308C0A0
:10DB600088EC8093330380916F008F7D80936F00EA
:10DB7000F701EE58F84F808191819C01220F331FED
:10DB8000280F391F260F371F37FF02C02D5F3F4F69
:10DB9000E901D595C795D595C795CB0101968C1709
:10DBA0009D0714F4219706C061507040C617D7072F
:10DBB0000CF4219680913303843BD0F0F701EE58AA
:10DBC000F84F80819181FE01E81BF90BCF0163E0E2
:10DBD00070E00E94908DCB01880F991F860F971FD0
:10DBE00026EA37E0E20EF31EF7019183808307C037
:10DBF00026EA37E0E20EF31EF70111821082000FD1
:10DC0000111F0E58184FF801D183C08311C0023183
:10DC1000110570F081E08093F6010AC081E08093E5
:10DC2000F601109232041092340484E4809330049C
:10DC300080913204803198F080913404882331F44B
:10DC40008091F601882311F480939401109232049C
:10DC5000109234041092310484E480933004E6E09E
:10DC6000CDB7DEB70C94088ECF93FC0197FF05C0AB
:10DC7000CFEFF095E195FF4F01C0C1E028E631E01C
:10DC8000CF01B9010E94908DFC018B35910554F0B4
:10DC90008B5590408A35910538F484EB90E08E1BCB
:10DCA0009F0BFC0141E00DC0CF01855B90408A35A0
:10DCB000910518F4E45BF04003C02E1B3F0BF90103
:10DCC0004FEFEE0FFF1FEC5EF54F259134918C2F37
:10DCD000992787FD9095289FB001299F700D389F47
:10DCE000700D1124842F992787FD9095689FA001BE
:10DCF000699F500D789F500D1124CA01CF9108954E
:10DD00002AE530E0281B390BC9010E94346E0895C2
:10DD1000CF93DF9380E00E947E8580911E019091D9
:10DD20001F016AE070E00E94908D9F938F93809115
:10DD30001E0190911F016AE070E00E94908D7F9318
:10DD40006F9384E59BE09F938F93C1E7D5E8DF93C2
:10DD5000CF93E0915404F091550409952DB73EB747
:10DD6000285F3F4F2DBF8091F2018823B9F186E0F3
:10DD70000E947E8580915508909156086AE070E077
:10DD80000E947C8D7F936F938FED90E09F938F9394
:10DD90008091450890914608A0914708B0914808A5
:10DDA00020919601309197014091980150919901ED
:10DDB000BC01CD010E94C58D3F932F938DE59BE063
:10DDC0009F938F93DF93CF93E0915404F091550488
:10DDD00009958DB79EB70A968DBF12C086E00E9446
:10DDE0007E8589E69BE09F938F93DF93CF93E091AD
:10DDF0005404F091550409950F900F900F900F90D7
:10DE0000809120048823C1F086E00E947E85809165
:10DE1000200499279F938F9380E79BE09F938F9394
:10DE2000DF93CF93E0915404F091550409952DB7F9
:10DE30003EB72A5F3F4F2DBF80E10E947E858091D3
:10DE40000002909101026CE370E00E947C8D9F9330
:10DE50008F9380910002909101026CE370E00E9428
:10DE60007C8D7F936F938091CF089091D0089F9382
:10DE70008F938BE79BE09F938F93C1E7D5E8DF9368
:10DE8000CF93E0915404F091550409958091540684
:10DE90002DB73EB7265F3F4F2DBF80FF29C08AE1D7
:10DEA0000E947E858091950199279F938F93809101
:10DEB000250390912603A0912703B0912803BC016C
:10DEC000CD0124E630E040E050E00E94C58D3F9354
:10DED0002F9388E89BE09F938F93DF93CF93E091FC
:10DEE0005404F091550409958DB79EB708968DBFDF
:10DEF00020919A03222351F58091CF089091D00868
:10DF0000029720F5822F0E947E858FE89BE09F93E9
:10DF10008F93DF93CF93E0915404F09155040995CA
:10DF200080E10E947E850F900F900F900F9080EA05
:10DF30009BE09F938F93DF93CF93E0915404F091F4
:10DF4000550409950F900F900F900F9080910B033F
:10DF5000882391F08091F80285FD0EC08091950193
:10DF60008B3211F485E603C08D3231F484E780935F
:10DF7000FE018AE08093FC01DF91CF9108950F9319
:10DF80001F9380E00E947E8580913007992787FD4E
:10DF900090959F938F9380912807992787FD90955F
:10DFA0009F938F9380912007992787FD90959F934A
:10DFB0008F9380911807992787FD90959F938F9352
:10DFC00081EB9BE09F938F9301E715E81F930F93DD
:10DFD000E0915404F0915504099580E10E947E85FA
:10DFE0008DB79EB70C968DBF80915007992787FDFE
:10DFF00090959F938F9380914807992787FD9095DF
:10E000009F938F9380914007992787FD90959F93C9
:10E010008F9380913807992787FD90959F938F93D1
:10E0200082EC9BE09F938F931F930F93E091540496
:10E03000F091550409958DB79EB70C968DBF1F9131
:10E040000F910895CF93DF932091CB083091CC08A6
:10E0500080914E0490914F048217930720F43093DF
:10E060004F0420934E0480E00E947E8580911E0123
:10E0700090911F016AE070E00E94908D9F938F93B2
:10E0800080911E0190911F016AE070E00E94908DC6
:10E090007F936F9382ED9BE09F938F93C1E7D5E8C9
:10E0A000DF93CF93E0915404F091550409958DB717
:10E0B0009EB708968DBF80912A038823D1F48AE009
:10E0C0000E947E8580914E0490914F046AE070E03A
:10E0D0000E947C8D9F938F9380914E0490914F046A
:10E0E0006AE070E00E947C8D7F936F938BED9BE0E4
:10E0F00019C08AE00E947E858091CB089091CC085F
:10E100006AE070E00E947C8D9F938F938091CB0892
:10E110009091CC086AE070E00E947C8D7F936F93B1
:10E1200084EE9BE09F938F93DF93CF93E091540411
:10E13000F091550409958DB79EB708968DBF80E183
:10E140000E947E858091CF089091D0089F938F93F5
:10E150008091CD089091CE089F938F938DEE9BE098
:10E160009F938F93DF93CF93E0915404F0915504E4
:10E1700009958DB79EB708968DBFDF91CF91089511
:10E180000F931F93CF93DF938091F201C1E7D5E8FE
:10E19000882309F478C080E00E947E85809152082F
:10E1A00099279F938F938091540899279F938F93DA
:10E1B00089EF9BE09F938F938E01DF93CF93E09144
:10E1C0005404F091550409958DB79EB708968DBFFC
:10E1D00080915308833031F48CE00E947E8588E082
:10E1E0009CE005C08CE00E947E858DE09CE09F93C2
:10E1F0008F93DF93CF93E0915404F09155040995E8
:10E200000F900F900F900F908091510881FF12C0D6
:10E210008CE00E947E8582E19CE09F938F931F9308
:10E220000F93E0915404F091550409950F900F90CD
:10E230000F900F9080E10E947E858FED90E09F937C
:10E240008F9380915708909158089F938F93809156
:10E250005508909156086AE070E00E947C8D7F938B
:10E260006F9387E19CE09F938F9381E795E89F935D
:10E270008F93E0915404F091550409958DB79EB7A2
:10E280000A968DBF12C082E00E947E8587E29CE0E4
:10E290009F938F93DF93CF93E0915404F0915504B3
:10E2A00009950F900F900F900F90DF91CF911F91D4
:10E2B0000F9108951F93CF93DF93182F80913D08FE
:10E2C0008F5F80933D089091E001891710F11092C3
:10E2D0003D088091160780930B0880911E0780935C
:10E2E0003C088091260780930A0880912E0780932E
:10E2F0001808809136078093360880913E078093F6
:10E30000F607809146078093130880914E0780930B
:10E3100017089091160780915204891710F4909372
:10E32000520490911E0780915604891710F490931F
:10E3300056049091260780915004891710F4909309
:10E34000500490912E0780915104891710F49093F6
:10E3500051049091360780915304891710F49093DB
:10E36000530490913E0780914D04891710F49093C7
:10E370004D049091460780915704891710F49093AB
:10E38000570490914E0780915804891710F4909388
:10E39000580480912A03882301F5809152048093C8
:10E3A0000B088091560480933C0880915004809320
:10E3B0000A08809151048093180880915304809337
:10E3C000360880914D048093F6078091570480931E
:10E3D0001308809158048093170880E00E947E857E
:10E3E00080911808282F332780914606482F5527FB
:10E3F0008091A5039091A603BA010E947C8D261BF3
:10E40000370B3F932F9380910A08282F3327809151
:10E410004606482F55278091A5039091A603BA017F
:10E420000E947C8D261B370B3F932F9380913C08D5
:10E43000282F332780914606482F55278091A50322
:10E440009091A603BA010E947C8D261B370B3F9347
:10E450002F9380910B08282F332780914606482F51
:10E4600055278091A5039091A603BA010E947C8D47
:10E47000261B370B3F932F9384E39CE09F938F934E
:10E48000C1E7D5E8DF93CF93E0915404F0915504B0
:10E49000099580E10E947E852DB73EB7245F3F4FEE
:10E4A0002DBF80911308282F332780914606482FCF
:10E4B00055278091A5039091A603BA010E947C8DF7
:10E4C000261B370B3F932F9380911308282F332758
:10E4D00080914606482F55278091A5039091A60369
:10E4E000BA010E947C8D261B370B3F932F9380919E
:10E4F000F607282F332780914606482F552780910D
:10E50000A5039091A603BA010E947C8D261B370BB0
:10E510003F932F9380913608282F3327809146060A
:10E52000482F55278091A5039091A603BA010E9418
:10E530007C8D261B370B3F932F9385E49CE09F93A4
:10E540008F93DF93CF93E0915404F0915504099594
:10E55000809146062DB73EB7245F3F4F2DBF8430D4
:10E5600039F580E10E947E858091CB089091CC089E
:10E570006AE070E00E947C8D9F938F938091CB081E
:10E580009091CC086AE070E00E947C8D7F936F933D
:10E5900085E59CE09F938F93DF93CF93E0915404A4
:10E5A000F091550409958DB79EB708968DBF29C087
:10E5B000863039F588E10E947E858091CB08909164
:10E5C000CC086AE070E00E947C8D9F938F938091CD
:10E5D000CB089091CC086AE070E00E947C8D7F931C
:10E5E0006F9388E69CE09F938F93DF93CF93E091A6
:10E5F0005404F091550409952DB73EB7285F3F4F5D
:10E600002DBF1F3221F48091E0018F5F05C01F34C0
:10E6100029F48091E00181508093E001DF91CF9156
:10E620001F910895482F109215081092E507109237
:10E6300032081092A4038F3251F08F3441F0809150
:10E64000E1019091E2010197049708F03EC08091AA
:10E65000E1019091E2010197049770F04F3419F4B1
:10E6600081E090E004C04F3239F484E090E0909370
:10E67000E2018093E10140E02091E1013091E2016B
:10E680002130310519F48EE38093150822303105CD
:10E6900019F48EE38093E5072330310519F48EE3F6
:10E6A000809332082430310519F48EE38093A4035B
:10E6B0004F3819F42150304004C04F3131F42F5FEE
:10E6C0003F4F3093E2012093E101842F9927089571
:10E6D0000F931F9380E00E947E8580912C079927DD
:10E6E0008F7790709F938F938091240799278F77CE
:10E6F00090709F938F9380911C0799278F779070CC
:10E700009F938F938091140799278F7790709F9391
:10E710008F9382E79CE09F938F9301E715E81F9307
:10E720000F93E0915404F0915504099580E10E9403
:10E730007E858DB79EB70C968DBF80914C0799272B
:10E740008F7790709F938F938091440799278F774D
:10E7500090709F938F9380913C0799278F7790704B
:10E760009F938F938091340799278F7790709F9311
:10E770008F9382E89CE09F938F931F930F93E09178
:10E780005404F091550409958DB79EB70C968DBF32
:10E790001F910F9108956F927F928F929F92AF92E7
:10E7A000BF92CF92DF92EF92FF920F931F93A090B0
:10E7B0004D03B0904E03C0904F03D090500329E01A
:10E7C000D594C794B794A7942A95D1F7E0904903BC
:10E7D000F0904A0300914B0310914C0399E015957A
:10E7E0000795F794E7949A95D1F76090510370904C
:10E7F0005203809053039090540389E0959487943A
:10E80000779467948A95D1F780E00E947E85FF9285
:10E81000EF92BF92AF9282E99CE09F938F9301E7C2
:10E8200015E81F930F93E0915404F0915504099556
:10E8300080E10E947E858DB79EB708968DBF7F923E
:10E840006F9280EA9CE09F938F931F930F93E091C8
:10E850005404F091550409958DB79EB706968DBF67
:10E860001F910F91FF90EF90DF90CF90BF90AF90EE
:10E870009F908F907F906F90089580E00E947E859A
:10E8800080912B0390912C039F938F93809114037D
:10E890009091150397FD0396959587959595879586
:10E8A0009F938F9381EB9CE09F938F9381E795E8F3
:10E8B0009F938F93E0915404F091550409958DB77F
:10E8C0009EB708968DBF08950F931F93CF930E9414
:10E8D0001273C82F80E00E947E85809190079091EE
:10E8E000910781589F4F9F938F938091320899276A
:10E8F0009F938F9380918C0790918D0781589F4FA4
:10E900009F938F938091150899279F938F9382EC03
:10E910009CE09F938F9301E715E81F930F93E0917D
:10E920005404F0915504099580E10E947E852DB72D
:10E930003EB7245F3F4F2DBF809192079091930780
:10E9400081589F4F9F938F938091A40399279F9302
:10E950008F9380918E0790918F0781589F4F9F933F
:10E960008F938091E50799279F938F9385ED9CE086
:10E970009F938F931F930F93E0915404F09155044C
:10E98000099580E090E02DB73EB7245F3F4F2DBF43
:10E99000CF3211F481E090E040E050E02091E101BD
:10E9A0003091E2012130310509F4A9018423952336
:10E9B000892B49F080918C0790918D070196909357
:10E9C0008D0780938C0780E090E0CF3411F481E0D4
:10E9D00090E040E050E02130310509F4A9018423A2
:10E9E0009523892B49F080918C0790918D07019791
:10E9F00090938D0780938C0780E090E0CF3211F4E4
:10EA000081E090E040E050E02230310511F441E037
:10EA100050E084239523892B49F080918E079091B3
:10EA20008F07019690938F0780938E0780E090E088
:10EA3000CF3411F481E090E040E050E02230310525
:10EA400011F441E050E084239523892B49F0809113
:10EA50008E0790918F07019790938F0780938E0771
:10EA600080E090E0CF3211F481E090E040E050E0AF
:10EA70002330310511F441E050E084239523892BA4
:10EA800049F0809190079091910705969093910796
:10EA90008093900780E090E0CF3411F481E090E023
:10EAA00040E050E02330310511F441E050E0842390
:10EAB0009523892B49F080919007909191070597B4
:10EAC000909391078093900780E090E0CF3211F40B
:10EAD00081E090E040E050E02430310511F441E065
:10EAE00050E084239523892B49F0809192079091DF
:10EAF00093070A96909393078093920780E090E0A3
:10EB0000CF3411F481E090E040E050E02430310552
:10EB100011F441E050E084239523892B49F0809142
:10EB20009207909193070A97909393078093920787
:10EB3000CF911F910F910895CF93C82F1092FE018E
:10EB40008091AD0680FF14C080E00E947E8588EE33
:10EB50009CE09F938F9381E795E89F938F93E0913B
:10EB60005404F091550409950F900F900F900F9059
:10EB70008091AD0680FD14C080E10E947E8589EF02
:10EB80009CE09F938F9381E795E89F938F93E0910B
:10EB90005404F091550409950F900F900F900F9029
:10EBA000CF3221F48091AD06816006C0CF3431F4BC
:10EBB0008091AD068E7F82608093AD06CF910895DF
:10EBC0000F931F93CF93C82F0E94127380E00E946F
:10EBD0007E8580915A0699279F938F938091320862
:10EBE00099279F938F938091560699279F938F9390
:10EBF0008091150899279F938F938AE09DE09F93BA
:10EC00008F9301E715E81F930F93E0915404F0915F
:10EC10005504099580E10E947E852DB73EB7245F9B
:10EC20003F4F2DBF8091550699279F938F938091D9
:10EC3000A40399279F938F938091580699279F93B8
:10EC40008F938091E50799279F938F938CE19DE0A7
:10EC50009F938F931F930F93E0915404F091550469
:10EC6000099580E090E02DB73EB7245F3F4F2DBF60
:10EC7000CF3211F481E090E040E050E02091E101DA
:10EC80003091E2012130310509F4A9018423952353
:10EC9000892B29F0809156068F5F8093560680E07D
:10ECA00090E0CF3411F481E090E040E050E021307A
:10ECB000310509F4A90184239523892B29F080913A
:10ECC000560681508093560680E090E0CF3211F4D2
:10ECD00081E090E040E050E02230310511F441E065
:10ECE00050E084239523892B29F0809158068F5F6B
:10ECF0008093580680E090E0CF3411F481E090E0FA
:10ED000040E050E02230310511F441E050E084232E
:10ED10009523892B29F080915806815080935806BD
:10ED200080E090E0CF3211F481E090E040E050E0EC
:10ED30002330310511F441E050E084239523892BE1
:10ED400029F080915A068F5F80935A0680E090E008
:10ED5000CF3411F481E090E040E050E02330310501
:10ED600011F441E050E084239523892B29F0809110
:10ED70005A06815080935A0680E090E0CF3211F419
:10ED800081E090E040E050E02430310511F441E0B2
:10ED900050E084239523892B29F0809155068F5FBD
:10EDA0008093550680E090E0CF3411F481E090E04C
:10EDB00040E050E02430310511F441E050E084237C
:10EDC0009523892B29F08091550681508093550613
:10EDD000CF911F910F9108950F931F93CF930E948E
:10EDE0001273C82F80E00E947E8580915C0699276F
:10EDF0009F938F938091320899279F938F9380914F
:10EE00005B0699279F938F938091150899279F936D
:10EE10008F938EE29DE09F938F9301E715E81F93F8
:10EE20000F93E0915404F0915504099580E10E94FC
:10EE30007E852DB73EB7245F3F4F2DBF80916C0676
:10EE400099279F938F938091A40399279F938F93E2
:10EE50008091590699279F938F938091E507992771
:10EE60009F938F9380E49DE09F938F931F930F93C5
:10EE7000E0915404F0915504099580E090E02DB79D
:10EE80003EB7245F3F4F2DBFCF3211F481E090E0B9
:10EE900040E050E02091E1013091E2012130310564
:10EEA00009F4A90184239523892B29F080915B061D
:10EEB0008F5F80935B0680E090E0CF3411F481E0B7
:10EEC00090E040E050E02130310509F4A9018423AD
:10EED0009523892B29F080915B06815080935B06F6
:10EEE00080E090E0CF3211F481E090E040E050E02B
:10EEF0002230310511F441E050E084239523892B21
:10EF000029F0809159068F5F8093590680E090E048
:10EF1000CF3411F481E090E040E050E02230310540
:10EF200011F441E050E084239523892B29F080914E
:10EF3000590681508093590680E090E0CF3211F459
:10EF400081E090E040E050E02330310511F441E0F1
:10EF500050E084239523892B29F080915C068F5FF4
:10EF600080935C0680E090E0CF3411F481E090E083
:10EF700040E050E02330310511F441E050E08423BB
:10EF80009523892B29F080915C06815080935C0643
:10EF900080E090E0CF3211F481E090E040E050E07A
:10EFA0002430310511F441E050E084239523892B6E
:10EFB00029F080916C068F5F80936C0680E090E072
:10EFC000CF3411F481E090E040E050E0243031058E
:10EFD00011F441E050E084239523892B29F080919E
:10EFE0006C06815080936C06CF911F910F9108950C
:10EFF0000F931F93CF930E941273C82F80E00E943B
:10F000007E858091600699279F938F938091320827
:10F0100099279F938F9380915E0699279F938F9353
:10F020008091150899279F938F9382E59DE09F9388
:10F030008F9301E715E81F930F93E0915404F0912B
:10F040005504099580E10E947E852DB73EB7245F67
:10F050003F4F2DBF80918B0699279F938F9380916F
:10F06000A40399279F938F9380915F0699279F937D
:10F070008F938091E50799279F938F9385E69DE075
:10F080009F938F931F930F93E0915404F091550435
:10F09000099580E090E02DB73EB7245F3F4F2DBF2C
:10F0A000CF3211F481E090E040E050E02091E101A6
:10F0B0003091E2012130310509F4A901842395231F
:10F0C000892B29F080915E068F5F80935E0680E039
:10F0D00090E0CF3411F481E090E040E050E0213046
:10F0E000310509F4A90184239523892B29F0809106
:10F0F0005E06815080935E0680E090E0CF3211F48E
:10F1000081E090E040E050E02230310511F441E030
:10F1100050E084239523892B29F080915F068F5F2F
:10F1200080935F0680E090E0CF3411F481E090E0BE
:10F1300040E050E02230310511F441E050E08423FA
:10F140009523892B29F080915F06815080935F067B
:10F1500080E090E0CF3211F481E090E040E050E0B8
:10F160002330310511F441E050E084239523892BAD
:10F1700029F0809160068F5F8093600680E090E0C8
:10F18000CF3411F481E090E040E050E023303105CD
:10F1900011F441E050E084239523892B29F08091DC
:10F1A000600681508093600680E090E0CF3211F4D9
:10F1B00081E090E040E050E02430310511F441E07E
:10F1C00050E084239523892B29F080918B068F5F53
:10F1D00080938B0680E090E0CF3411F481E090E0E2
:10F1E00040E050E02430310511F441E050E0842348
:10F1F0009523892B29F080918B06815080938B0673
:10F20000CF911F910F9108950F931F93CF930E9459
:10F210001273C82F80E00E947E8580916606992730
:10F220009F938F938091320899279F938F9380911A
:10F23000650699279F938F938091150899279F932F
:10F240008F9388E79DE09F938F9301E715E81F93C5
:10F250000F93E0915404F0915504099580E10E94C8
:10F260007E852DB73EB7245F3F4F2DBF80916F063F
:10F2700099279F938F938091A40399279F938F93AE
:10F280008091670699279F938F938091E50799272F
:10F290009F938F938BE89DE09F938F931F930F9382
:10F2A000E0915404F0915504099580E090E02DB769
:10F2B0003EB7245F3F4F2DBFCF3211F481E090E085
:10F2C00040E050E02091E1013091E2012130310530
:10F2D00009F4A90184239523892B29F080916506DF
:10F2E0008F5F8093650680E090E0CF3411F481E079
:10F2F00090E040E050E02130310509F4A901842379
:10F300009523892B29F080916506815080936506AD
:10F3100080E090E0CF3211F481E090E040E050E0F6
:10F320002230310511F441E050E084239523892BEC
:10F3300029F0809167068F5F8093670680E090E0F8
:10F34000CF3411F481E090E040E050E0223031050C
:10F3500011F441E050E084239523892B29F080911A
:10F36000670681508093670680E090E0CF3211F409
:10F3700081E090E040E050E02330310511F441E0BD
:10F3800050E084239523892B29F0809166068F5FB6
:10F390008093660680E090E0CF3411F481E090E045
:10F3A00040E050E02330310511F441E050E0842387
:10F3B0009523892B29F080916606815080936606FB
:10F3C00080E090E0CF3211F481E090E040E050E046
:10F3D0002430310511F441E050E084239523892B3A
:10F3E00029F080916F068F5F80936F0680E090E038
:10F3F000CF3411F481E090E040E050E0243031055A
:10F4000011F441E050E084239523892B29F0809169
:10F410006F06815080936F06CF911F910F910895D1
:10F420000F931F93CF930E941273C82F80E00E9406
:10F430007E858091A30699279F938F9380913208B0
:10F4400099279F938F938091980699279F938F93E5
:10F450008091150899279F938F938EE99DE09F9344
:10F460008F9301E715E81F930F93E0915404F091F7
:10F470005504099580E10E947E852DB73EB7245F33
:10F480003F4F2DBF8091A50699279F938F93809121
:10F49000A40399279F938F938091A20699279F9306
:10F4A0008F938091E50799279F938F9381EB9DE040
:10F4B0009F938F931F930F93E0915404F091550401
:10F4C000099580E090E02DB73EB7245F3F4F2DBFF8
:10F4D000CF3211F481E090E040E050E02091E10172
:10F4E0003091E2012130310509F4A90184239523EB
:10F4F000892B29F0809198068F5F8093980680E091
:10F5000090E0CF3411F481E090E040E050E0213011
:10F51000310509F4A90184239523892B29F08091D1
:10F52000980681508093980680E090E0CF3211F4E5
:10F5300081E090E040E050E02230310511F441E0FC
:10F5400050E084239523892B29F08091A2068F5FB8
:10F550008093A20680E090E0CF3411F481E090E047
:10F5600040E050E02230310511F441E050E08423C6
:10F570009523892B29F08091A20681508093A206C1
:10F5800080E090E0CF3211F481E090E040E050E084
:10F590002330310511F441E050E084239523892B79
:10F5A00029F08091A3068F5F8093A30680E090E00E
:10F5B000CF3411F481E090E040E050E02330310599
:10F5C00011F441E050E084239523892B29F08091A8
:10F5D000A30681508093A30680E090E0CF3211F41F
:10F5E00081E090E040E050E02430310511F441E04A
:10F5F00050E084239523892B29F08091A5068F5F05
:10F600008093A50680E090E0CF3411F481E090E093
:10F6100040E050E02430310511F441E050E0842313
:10F620009523892B29F08091A50681508093A5060A
:10F63000CF911F910F9108950F931F93CF930E9425
:10F640001273C82F80E00E947E8580919B069927C7
:10F650009F938F938091320899279F938F938091E6
:10F66000990699279F938F938091150899279F93C7
:10F670008F9384EC9DE09F938F9301E715E81F9390
:10F680000F93E0915404F0915504099580E10E9494
:10F690007E852DB73EB7245F3F4F2DBF8091A403D9
:10F6A00099279F938F9380919A0699279F938F9381
:10F6B0008091E50799279F938F9385ED9DE09F9318
:10F6C0008F931F930F93E0915404F0915504099583
:10F6D00080E090E02DB73EB7265F3F4F2DBFCF3281
:10F6E00011F481E090E040E050E02091E1013091A0
:10F6F000E2012130310509F4A90184239523892BE6
:10F7000029F0809199068F5F8093990680E090E0C0
:10F71000CF3411F481E090E040E050E02130310539
:10F7200009F4A90184239523892B29F08091990656
:10F7300081508093990680E090E0CF3211F481E00F
:10F7400090E040E050E02230310511F441E050E01B
:10F7500084239523892B29F080919A068F5F8093CB
:10F760009A0680E090E0CF3411F481E090E040E030
:10F7700050E02230310511F441E050E0842395231C
:10F78000892B29F080919A06815080939A0680E017
:10F7900090E0CF3211F481E090E040E050E023307F
:10F7A000310511F441E050E084239523892B29F0A1
:10F7B00080919B068F5F80939B0680E090E0CF3422
:10F7C00011F481E090E040E050E02330310511F485
:10F7D00041E050E084239523892B29F080919B06FA
:10F7E000815080939B06CF911F910F910895FF92B6
:10F7F0000F931F93CF93F82EC091AB06CF7080E08C
:10F800000E947E8581EE9DE09F938F9301E715E82E
:10F810001F930F93E0915404F09155040995809142
:10F82000AB060F900F900F900F9082FF06C08CE3F5
:10F830000E94718580E00E9471858091AB0680FFF7
:10F8400006C08EE50E94718580E00E9471858091DE
:10F85000AB0681FF06C086E70E94718580E00E94AA
:10F8600071858091AB0683FF03C08EE30E94718592
:10F8700080E10E947E858C2F99279F938F9383EE42
:10F880009DE09F938F931F930F93E0915404F09109
:10F890005504099580E090E02DB73EB72A5F3F4FB1
:10F8A0002DBF3FE2F31611F481E090E020E030E05C
:10F8B000CF3010F421E030E082239323892B09F02C
:10F8C000CF5F80E090E02FE4F21611F481E090E049
:10F8D00020E030E0CC2311F021E030E082239323BC
:10F8E000892B09F0C1508091AB06807F8C2B8093CF
:10F8F000AB06CF911F910F91FF9008950F931F9327
:10F90000CF930E941273C82F80E00E947E85809161
:10F91000840699279F938F938091320899279F930C
:10F920008F938091820699279F938F9380911508DA
:10F9300099279F938F9385EF9DE09F938F9301E786
:10F9400015E81F930F93E0915404F0915504099525
:10F9500080E10E947E852DB73EB7245F3F4F2DBFCB
:10F960008091830699279F938F938091E50799272C
:10F970009F938F9388E09EE09F938F931F930F93A5
:10F98000E0915404F0915504099580E090E02DB782
:10F990003EB7285F3F4F2DBFCF3211F481E090E09A
:10F9A00040E050E02091E1013091E2012130310549
:10F9B00009F4A90184239523892B29F080918206DB
:10F9C0008F5F8093820680E090E0CF3411F481E075
:10F9D00090E040E050E02130310509F4A901842392
:10F9E0009523892B29F0809182068150809382068D
:10F9F00080E090E0CF3211F481E090E040E050E010
:10FA00002230310511F441E050E084239523892B05
:10FA100029F0809183068F5F8093830680E090E0D9
:10FA2000CF3411F481E090E040E050E02230310525
:10FA300011F441E050E084239523892B29F0809133
:10FA4000830681508093830680E090E0CF3211F4EA
:10FA500081E090E040E050E02330310511F441E0D6
:10FA600050E084239523892B29F0809184068F5FB1
:10FA70008093840680E090E0CF3411F481E090E040
:10FA800040E050E02330310511F441E050E08423A0
:10FA90009523892B29F080918406815080938406D8
:10FAA000CF911F910F9108950F931F93CF930E94B1
:10FAB0001273C82F80E00E947E8580918706992767
:10FAC0009F938F938091320899279F938F93809172
:10FAD000850699279F938F938091150899279F9367
:10FAE0008F9382E19EE09F938F9301E715E81F9328
:10FAF0000F93E0915404F0915504099580E10E9420
:10FB00007E852DB73EB7245F3F4F2DBF80918F0676
:10FB100099279F938F938091A40399279F938F9305
:10FB20008091860699279F938F938091E507992767
:10FB30009F938F9385E29EE09F938F931F930F93E4
:10FB4000E0915404F0915504099580E090E02DB7C0
:10FB50003EB7245F3F4F2DBFCF3211F481E090E0DC
:10FB600040E050E02091E1013091E2012130310587
:10FB700009F4A90184239523892B29F08091850616
:10FB80008F5F8093850680E090E0CF3411F481E0B0
:10FB900090E040E050E02130310509F4A9018423D0
:10FBA0009523892B29F080918506815080938506C5
:10FBB00080E090E0CF3211F481E090E040E050E04E
:10FBC0002230310511F441E050E084239523892B44
:10FBD00029F0809186068F5F8093860680E090E012
:10FBE000CF3411F481E090E040E050E02230310564
:10FBF00011F441E050E084239523892B29F0809172
:10FC0000860681508093860680E090E0CF3211F422
:10FC100081E090E040E050E02330310511F441E014
:10FC200050E084239523892B29F0809187068F5FEC
:10FC30008093870680E090E0CF3411F481E090E07B
:10FC400040E050E02330310511F441E050E08423DE
:10FC50009523892B29F08091870681508093870610
:10FC600080E090E0CF3211F481E090E040E050E09D
:10FC70002430310511F441E050E084239523892B91
:10FC800029F080918F068F5F80938F0680E090E04F
:10FC9000CF3411F481E090E040E050E024303105B1
:10FCA00011F441E050E084239523892B29F08091C1
:10FCB0008F06815080938F06CF911F910F910895E9
:10FCC0000F931F93CF930E941273C82F80E00E945E
:10FCD0007E8580916A0699279F938F938091320841
:10FCE00099279F938F938091680699279F938F936D
:10FCF0008091150899279F938F9388E39EE09F93A7
:10FD00008F9301E715E81F930F93E0915404F0914E
:10FD10005504099580E10E947E852DB73EB7245F8A
:10FD20003F4F2DBF80918C0699279F938F93809191
:10FD3000A40399279F938F938091690699279F9396
:10FD40008F938091E50799279F938F938BE49EE093
:10FD50009F938F931F930F93E0915404F091550458
:10FD6000099580E090E02DB73EB7245F3F4F2DBF4F
:10FD7000CF3211F481E090E020E030E04091E101E9
:10FD80005091E2014130510509F49A0182239323F5
:10FD9000892B29F0809168068F5F8093680680E048
:10FDA00090E0CF3411F481E090E020E030E0413089
:10FDB000510509F49A0182239323892B29F080911C
:10FDC000680681508093680680E090E0CF3211F49D
:10FDD00081E090E020E030E04230510511F421E074
:10FDE00030E082239323892B29F0809169068F5F6D
:10FDF0008093690680E090E0CF3411F481E090E0D8
:10FE000020E030E04230510511F421E030E082235F
:10FE10009323892B29F0809169068150809369068C
:10FE200020E030E0CF3211F421E030E080E090E0DB
:10FE30004330510511F481E090E08223932360E088
:10FE400070E020916A062F3010F461E070E08623A4
:10FE50009723892B19F02F5F20936A0620E030E06A
:10FE6000CF3411F421E030E080E090E043305105E0
:10FE700011F481E090E08223932360E070E0209110
:10FE80006A06222311F061E070E086239723892B14
:10FE900019F0215020936A0680E090E0CF3211F4EF
:10FEA00081E090E020E030E04430510511F421E0A1
:10FEB00030E082239323892B29F080918C068F5F79
:10FEC00080938C0680E090E0CF3411F481E090E0E4
:10FED00020E030E04430510511F421E030E082238D
:10FEE0009323892B29F080918C06815080938C0676
:10FEF000CF911F910F9108950F931F93CF930E945D
:10FF00001273C82F80E00E947E8580917806992721
:10FF10009F938F938091320899279F938F9380911D
:10FF2000740699279F938F938091150899279F9323
:10FF30008F938EE59EE09F938F9301E715E81F93C3
:10FF40000F93E0915404F0915504099580E10E94CB
:10FF50007E852DB73EB7245F3F4F2DBF8091790638
:10FF600099279F938F938091A40399279F938F93B1
:10FF70008091750699279F938F938091E507992724
:10FF80009F938F9381E79EE09F938F931F930F938F
:10FF9000E0915404F0915504099580E090E02DB76C
:10FFA0003EB7245F3F4F2DBFCF3211F481E090E088
:10FFB00040E050E02091E1013091E2012130310533
:10FFC00009F4A90184239523892B29F080917406D3
:10FFD0008F5F8093740680E090E0CF3411F481E06D
:10FFE00090E040E050E02130310509F4A90184237C
:10FFF0009523892B29F08091740681508093740693
:020000021000EC
:1000000080E090E0CF3211F481E090E040E050E0F9
:100010002230310511F441E050E084239523892BEF
:1000200029F0809175068F5F8093750680E090E0DF
:10003000CF3411F481E090E040E050E0223031050F
:1000400011F441E050E084239523892B29F080911D
:10005000750681508093750680E090E0CF3211F4F0
:1000600081E090E040E050E02330310511F441E0C0
:1000700050E084239523892B29F0809178068F5FA7
:100080008093780680E090E0CF3411F481E090E036
:1000900040E050E02330310511F441E050E084238A
:1000A0009523892B29F080917806815080937806DA
:1000B00080E090E0CF3211F481E090E040E050E049
:1000C0002430310511F441E050E084239523892B3D
:1000D00029F0809179068F5F8093790680E090E027
:1000E000CF3411F481E090E040E050E0243031055D
:1000F00011F441E050E084239523892B29F080916D
:100100007906815080937906CF911F910F910895C0
:100110000F931F93CF93C82F80EF8093110280E03D
:100120000E947E8580914D08E82FFF2743E0EE0F67
:10013000FF1F4A95E1F7EF5EF84F8581282F33279F
:1001400080914606482F55278091A5039091A603DC
:10015000BA010E947C8D261B370B3F932F9384E8B6
:100160009EE09F938F9301E715E81F930F93E09113
:100170005404F0915504099580E10E947E858DB765
:100180009EB706968DBF80914D08E82FFF27EB584C
:10019000FB4F808199279F938F9380914D089927DA
:1001A00001969F938F9385E99EE09F938F931F9372
:1001B0000F93E0915404F0915504099520E030E04C
:1001C0008DB79EB708968DBFCF3211F421E030E095
:1001D00040E050E08091E907843610F441E050E0BF
:1001E00024233523232B19F08E5F8093E90720E029
:1001F00030E0CF3411F421E030E040E050E0809175
:10020000E907882311F041E050E024233523232B14
:1002100019F082508093E90720E030E0CF3A11F4E2
:1002200021E030E040E050E080914D088F3010F444
:1002300041E050E024233523232B41F0E82FFF2712
:10024000EB58FB4F10828F5F80934D0820E030E029
:10025000CF3C11F421E030E040E050E080914D08C7
:10026000882311F041E050E024233523232B41F073
:10027000E82FFF27EB58FB4F1082815080934D08E9
:1002800080914D08E82FFF27EB58FB4F8091E9073D
:100290008083CF911F910F9108951F93CF93DF9388
:1002A000182F80E00E947E850E941B3099279F9323
:1002B0008F9386EA9EE09F938F93C1E7D5E8DF9303
:1002C000CF93E0915404F0915504099580E10E9488
:1002D0007E858DB79EB706968DBF8091E3019927E5
:1002E0009F938F9383EB9EE09F938F93DF93CF93A6
:1002F000E0915404F091550409958DB79EB7069688
:100300008DBF1F3959F580912A03882339F585E679
:100310008093FE010E941B309AE0899FC001112446
:100320008093FC018091E3010E94372F0E941B30D3
:1003300068E770E00E94EB398DE00E947E8586ECD4
:100340009EE09F938F93DF93CF93E0915404F091BD
:10035000550409950F900F900F900F9020E030E01A
:100360001F3211F421E030E040E050E08091E301E1
:10037000853010F441E050E024233523232B19F07D
:100380008F5F8093E30120E030E01F3411F421E01F
:1003900030E040E050E08091E301823010F041E035
:1003A00050E024233523232B19F081508093E3015F
:1003B000DF91CF911F910895CF93C82F20913504DD
:1003C0002093360499278F32910589F18033910566
:1003D0003CF48F30910509F43CC04F97C1F065C0E3
:1003E0008F34910561F18F38910509F05EC08091DD
:1003F000E1019091E2010197049708F456C086E06C
:10040000289FF0011124E653F54F84911FC080917D
:10041000E1019091E2010197049708F446C086E05B
:10042000289FF0011124E553F54F84910FC086E019
:10043000289FF0011124E453F54F849107C086E012
:10044000289FF0011124E353F54F849180933504E4
:100450002CC08091E1019091E201059779F486E04A
:10046000289FF0011124E553F54F849180933504C2
:1004700086E090E09093E2018093E1018091E101B8
:100480009091E201892B89F49091350486E0989F40
:10049000F0011124E653F54F8491809335048FEFDA
:1004A0009FEF9093E2018093E10190913504809158
:1004B00036049813C0E00E9484859091350486E04C
:1004C000989FF0011124E253F54F259134918C2F20
:1004D000F901099580E090E0CF9108951092CC0841
:1004E0001092CB081092D0081092CF081092CE082C
:1004F0001092CD081092D1088AE090E00E94D9189D
:1005000090933804809337040895CF93DF938091BC
:100510003704909138040E94E218882309F4AFC090
:1005200080913704909138040A9690933804809310
:100530003704E0E0F0E09F0190E05FEFA1E1B7E079
:100540004BE0ED018B8187FF0BC09F5F8D81E80F32
:10055000F11D8981280F311D8E81851708F4582FD0
:100560004150189647FFEDCF5093D108232B41F50A
:1005700020913D0430913E0440913F04509140044D
:10058000BB27A52F942F832F90933C0480933B048B
:10059000AA27BB27281B390B4A0B5B0BCF01AA27C5
:1005A000BB27280F391F4A1F5B1F20933D04309340
:1005B0003E0440933F0450934004E5E0F0E013C054
:1005C00020913B0430913C042E173F0718F4E21BA6
:1005D000F30B02C0E0E0F0E0892F9927880F991F04
:1005E000E80FF91F3596F093CC08E093CB08EF3F66
:1005F000F10578F480911E0190911F018E9F90016A
:100600008F9F300D9E9F300D1124C90164E670E06C
:1006100013C0CF01969587959695879520911E01D9
:1006200030911F01289FA001299F500D389F500D28
:100630001124CA0169E170E00E947C8D7093CE089C
:100640006093CD082091390430913A042E0F3F1F5A
:1006500030933A04209339045EE02131350778F075
:100660008091CF089091D00801969093D008809304
:10067000CF0820513E4030933A0420933904DF9153
:10068000CF910895002422273327442751E0BB2728
:10069000EE27FF27A0E1660F771F881F991F001C18
:1006A000221F331F441F660F771F881F991F001CCE
:1006B000221F331F441F2AF4050E2B1F3E1F4F1FFE
:1006C00004C0051A2B0B3E0B4F0B550FBB1FEE1F23
:1006D000587F556047FD5250AA95E9F6E695B795C3
:1006E0005795E695B7955795852F9B2F0895222707
:1006F000332741E0552768E0880F991F221F331FD9
:10070000880F991F221F331F1AF4240F351F02C0B0
:10071000241B350B440F551F487F456037FD425061
:100720006A9551F75695479556954795842F0895A4
:10073000AA2797FF04C0809590958A1F9A1F77FF7C
:1007400004C0609570956A1F7A1F669F9001779F1D
:10075000A001679F300D411D5A1F300D411D5A1FCA
:10076000889FF001999F2E0F3F1F401D511D899FAB
:10077000300D411D5A1F300D411D5A1FCA01B901CC
:10078000112480CF4FB720E430E0F8948091C90065
:100790008F778093C9008091C9008F7B8093C900B7
:1007A0008091C9008F7D8093C9005A9A52985B9AB4
:1007B000539A832F99278093CD002093CC0080916A
:1007C000C80082608093C80088E18093C90080914E
:1007D000CA008F778093CA008091CA008F7B809374
:1007E000CA008091CA008F7D8093CA008091CA00A0
:1007F0008F7E8093CA008091CA00877F8093CA0051
:100800008091C9008B7F8093C9008091CA00846069
:100810008093CA008091CA0082608093CA00809150
:10082000C80087FF03C08091CE00F9CF8091C90036
:1008300080688093C9004FBF08950F931F93CF9393
:10084000DF93482F4F5F893108F08BC0809171078B
:10085000841720F44F5F409371074150CB018353BD
:100860009B4268E170E00E94908DA42FBB27FD01A0
:10087000EA0FFB1FEE58F84F808191819B01281BE6
:10088000390BC90137FF03C0909581959F4F06979B
:1008900094F480913303883C30F480913303865F75
:1008A0008093330308C088EC8093330380916F00FA
:1008B0008F7D80936F00FD01EA0FFB1FEE58F84F0C
:1008C000808191819C01220F331F280F391F260F31
:1008D000371F37FF02C02D5F3F4FE901D595C79500
:1008E000D595C795CB0101968C179D0714F42197D8
:1008F00006C061507040C617D7070CF4219680914E
:100900003303843BD8F08D010A0F1B1FF801EE580A
:10091000F84F80819181FE01E81BF90BCF0163E064
:1009200070E00E94908DCB01880F991F860F971F52
:100930000A55184FF8019183808307C0AA0FBB1F87
:10094000AA55B84F11961C921E92E42FFF27EE0F66
:10095000FF1FEE58F84FD183C083443011F410923A
:100960009401DF91CF911F910F910895CF93DF9361
:100970002091D208822F9927807F9070409709F0AC
:100980006CC02F3109F046C08091D3088093450494
:100990002091D508209347048091D608809346047F
:1009A000822F99279093730780937207222309F06F
:1009B00054C080914806282F3327220F331FF90196
:1009C000EA55F84F1182108280914906A82FBB2763
:1009D000AA0FBB1FFD01EA55F84F118210828091CA
:1009E0004B06E82FFF27EE0FFF1FCF018A55984FC8
:1009F000EC01198218822E58384FE90119821882A9
:100A0000AE58B84F11961C921E92EE58F84F1182B4
:100A1000108223C0C22FCF70CA30F8F48091D3085F
:100A20008093FC088091D4088093FB088091D508BE
:100A30008093FE088091D6088093FD086091FB08A2
:100A40007091FC088C2F0E941D846091FD087091AC
:100A5000FE088C2F8F5F0E941D84DF91CF91089537
:100A6000CF93C82F8F3F49F4809148048F3F29F4DA
:100A700010924A041092490432C020914A04222361
:100A800039F4CF3111F485E001C084E080934B0448
:100A900080914B04909149048217A0F4892F80958E
:100AA000809349048F3F19F48EEF8093490480911D
:100AB0004904C81711F40E94B68410924A04109297
:100AC00049040BC0E22FFF27EE52F74FC0832F5F80
:100AD00020934A049C0F90934904C0934804CF91FB
:100AE000089590914404933240F4E92FFF27E8528F
:100AF000F74F80839F5F909344040895833218F4E6
:100B00008D5F80934404089590E2EBEDF8E08FE16F
:100B10009193815087FFFCCF0895CF93CFB723E007
:100B200031E0F8948091C9008F778093C90080915B
:100B3000C9008F7B8093C9008091C9008F7D80930D
:100B4000C9005A9A52985B9A539A832F9927809397
:100B5000CD002093CC008091C80082608093C800B3
:100B600088E18093C9008091CA008F778093CA0082
:100B70008091CA008F7B8093CA008091CA008062F6
:100B80008093CA008091CA0080618093CA008091DE
:100B9000CA0088608093CA008091C90084608093F5
:100BA000C9008091CA0084608093CA008091CA0005
:100BB00082608093CA008091C80087FF03C0809143
:100BC000CE00F9CF8091C90080688093C9008091E0
:100BD000C90080648093C9000E948485CFBFCF91F3
:100BE0000895282F99278F709070892B31F42095C4
:100BF00080914304822B8093430408958091F901EE
:100C0000882309F449C08091F80285FD04C08091D1
:100C1000FE01882371F082E98093D80883E28093F3
:100C2000D9088091FE01882309F485E58093DA08CC
:100C300002C08093D8088091FA018F3071F48091BE
:100C400043040E94DC81882341F081E98093D80825
:100C50008093D90881E38093DA081092F90180919A
:100C6000C80085FFFCCF8091C9008F7E8093C900AA
:100C70008091C9008E7F8093C9008091D808882315
:100C800011F48EEF01C08EE78093CE008091430473
:100C90008093FA011092430408951F920F920FB6A9
:100CA0000F9211248F939F93EF93FF939091F901EB
:100CB000992309F040C080914C04882361F480910D
:100CC000D808882311F483E003C0813999F481E0C6
:100CD00080934C040FC0833099F48091D808882306
:100CE00049F09093D8088091C9008E7F8093C90005
:100CF0008EEF1EC08091C90081608093C9000EC034
:100D0000833261F48091C9008E7F8093C9008FEF98
:100D10008093CE0081E08093F90114C080914C044F
:100D2000E82FFF27E852F74F8F5F80934C048081B4
:100D30008093CE0007C010924C048091C90080615E
:100D40008093C900FF91EF919F918F910F900FBEFB
:100D50000F901F901895EF92FF920F931F93CF93D0
:100D6000DF937C018B01EA01452B39F0F801819179
:100D70008F01F70109952197C9F7E6E0CDB7DEB7F6
:100D80000C94088EEF92FF920F931F93CF93DF93F3
:100D90007C018B01EA01452B41F0F8010F5F1F4FE9
:100DA0008491F70109952197C1F7E6E0CDB7DEB749
:100DB0000C94088E0F931F93CF938C01C62F161699
:100DC00034F480E2F8010995C1501C16D4F3CF9198
:100DD0001F910F9108950F931F93CF938C01C62FEE
:100DE000161634F480E3F8010995C1501C16D4F3AB
:100DF000CF911F910F910895A5E3B0E0E2E0F7E8ED
:100E00000C94E08D2E96EEADFFAD2E97882499249C
:100E1000540180914204882321F42C961FAE1EAE0B
:100E20002C975EE4452E512C4C0E5D1E6F01B601D1
:100E300005C0153239F00894C11CD11CF60114917B
:100E40001123B9F7A601461B570B31F02C968EAD36
:100E50009FAD2C970E94C286112309F46AC20894A0
:100E6000C11CD11CFF24FDA6FCA64FEFE42EF9A661
:100E7000F6010894C11CD11C1491153721F0812F63
:100E800080628837B1F4F0FE0AC0F20124E030E05D
:100E9000420E531E80809180A280B3800AC0F2016E
:100EA00042E050E0440E551E808191814C01AA24FD
:100EB000BB24103221F489A58823D1F61DC013323A
:100EC00019F458E0F52AD4CF1A3211F01D3291F4FA
:100ED0001A3259F4F20182E090E0480E591EE08186
:100EE000ECA7EE232CF6E195ECA790E1F92AAFED03
:100EF000FA22BECF1B3211F419A7BACF1E32C1F5A8
:100F0000F6010894C11CD11C14911A3279F4F20133
:100F100022E030E0420E531E408151813FEF4F3FAF
:100F2000530714F44FEF5FEFE42EA2CF40E050E000
:100F3000812F80538A30A0F4CA0133E0880F991FB3
:100F40003A95E1F7840F951F480F591F410F511D26
:100F500040535040F6010894C11CD11C1491E8CFB5
:100F60008FEF4F3F580714F44FEF5FEFE42E85CF1C
:100F7000103329F4F4FC7CCF90E2F92A79CF812F49
:100F800081538930D8F440E050E0CA0123E0880F53
:100F9000991F2A95E1F7840F951F480F591F410F9C
:100FA000511D40535040F6010894C11CD11C1491AE
:100FB000812F80538A3048F34CA75FCF183619F43D
:100FC000A4E0FA2A55CF1C3619F4B1E0FB2A50CF21
:100FD000133661F43E010894611C711CF20122E099
:100FE00030E0420E531E808189833CC1143421F0CD
:100FF000143611F0193651F5143411F431E0F32A96
:10100000F0FE0AC0F20144E050E0440E551E80801C
:101010009180A280B3800CC0F20182E090E0480E83
:10102000591E808191814C01AA2497FCA094BA2C6E
:10103000B7FE0AC0B094A09490948094811C911C37
:10104000A11CB11C8DE289A70AE06FC01F3411F00A
:101050001F3631F41F3411F491E0F92A08E064C01E
:10106000103779F4F201A2E0B0E04A0E5B1E8081F5
:1010700091814C01AA24BB2400E1B0E4FB2A18E7CB
:1010800053C01337C1F5F20122E030E0420E531E87
:10109000608071806114710489F43E010894611CC0
:1010A000711C88E289838EE6F301818385E78B8357
:1010B0008CE68C838D8389E28E831F82E7FC13C0CC
:1010C0008E2D992787FD9095AC0160E070E0C301FB
:1010D0000E94AD8B009729F0382E3618E3140CF0DF
:1010E000C3C03E2CC1C0F30101900020E9F7319745
:1010F0003E2E3618B9C0153511F0153731F41535B7
:1011000011F4F1E0FF2A0AE00FC0183519F0183782
:1011100009F0A0C000E1F3FE07C081149104A1040E
:10112000B10411F020E4F22A19A6EDA6E7FC02C0F2
:101130003FEDF32289E2682E712C6C0E7D1E811426
:101140009104A104B10421F44DA5442309F47BC00A
:10115000802F9927AA27BB278EA79FA7A8ABB9AB3B
:10116000202E332490E0891690E0990691E0A9069C
:1011700090E0B90648F0C501B4012EA53FA548A9E5
:1011800059A90E94A38D17C0AFEF8A169104A1043C
:10119000B10449F040F0C401B1010E947C8D9B0173
:1011A0004427552708C0882D602F0E94708D282F56
:1011B0003327442755272AAB3BAB4CAB5DAB0A30FA
:1011C00059F48AA9880F880F880F9AA9990F890F57
:1011D000382D381B832F10C0003139F48AA982952D
:1011E000807F482D481B842F07C08AA9880F880F4D
:1011F000880F582D581B852F90E02EA53FA548A994
:1012000059A982169306A406B50608F091E08AA8AB
:101210009BA8ACA8BDA88A3010F4805D04C0895A90
:10122000183509F48F7DD3018E933D01992309F080
:1012300099CF083041F4F3FE06C0803321F080E3FB
:10124000FD0182933F01CE010196382E3618F8E257
:101250003F0E0BC0112309F46CC03E010894611CC1
:10126000711C1983B1E03B2E19A6032D2DA4231860
:1012700027FC222489A5882311F00F5F02C0F6FC09
:101280000E5F020DEF2CFF24C70180739070892B35
:1012900049F48CA5801B682F2C968EAD9FAD2C97A2
:1012A0000E94DA8689A5882331F041E050E0BE0132
:1012B000675D7F4F0AC0E6FE0EC080E38AA71BA7CA
:1012C00042E050E0BE01665D7F4F2C968EAD9FAD33
:1012D0002C970E94AB86C70180739070809749F469
:1012E0008CA5801B682F2C968EAD9FAD2C970E94ED
:1012F000EB86622D2C968EAD9FAD2C970E94EB86CF
:10130000832D992787FD9095AC01B3012C968EAD66
:101310009FAD2C970E94AB86E4FE89CD2CA5201BA7
:101320002CA7622F2C968EAD9FAD2C970E94DA864B
:101330007ECDE2E1CB5C0C94FC8D2FB740E0F894BD
:10134000E0E0F0E081E2809357009491E2E0F0E089
:10135000809357003491E4E0F0E08093570084914B
:101360002FBF9E3199F4363941F4893011F441E0B0
:101370000DC08A3059F442E009C0373939F486305B
:1013800011F443E003C0853009F444E0842F992729
:1013900008959FB7F8948091C900877F8093C90012
:1013A0008091C9008F7E8093C9008091C9008F779A
:1013B0008093C9008091C9008F7B8093C900809180
:1013C000C9008F7D8093C90052985A9A53985B9AAE
:1013D0009FBF08951F93CF93DF93182F80914204EE
:1013E000882309F48DC08091F801181709F488C08A
:1013F00080914104882321F40E949D8980934104B7
:1014000086EB9FE09F938F93C3EBD4E1DF93CF9361
:10141000E0915404F091550409950F900F900F90AE
:101420000F90812F99278230910501F1833091052A
:101430002CF4009761F0019769F024C08430910585
:10144000D9F084309105ACF00597C9F01BC086EA4D
:101450009FE002C084E99FE09F938F93DF93CF9337
:10146000E0915404F0915504099518C08BE79FE072
:10147000F3CF88E59FE0F0CF8AE49FE0EDCF82E4F0
:101480009FE0EACF83EC9FE09F938F93DF93CF930E
:10149000E0915404F0915504099510E00F900F90DD
:1014A0000F900F9080914104843011F0823099F4B4
:1014B0000E94C989812F8150833018F40E94906C5A
:1014C0001DC0143019F40E948D8518C01530B1F478
:1014D0000E94C28313C0112389F089ED9FE09F937E
:1014E0008F9383EB94E19F938F93E0915404F09159
:1014F000550409950F900F900F900F901093F801DD
:10150000DF91CF911F9108950F931F9381E08093F6
:1015100042044091F701E2EFFEE020E030E05FE4BA
:10152000849199272F5F3F4F829FB001839F700D59
:10153000929F700D112446275150319657FFF0CFDE
:101540004093F701EAECFEE020E030E057E28491BE
:1015500099272F5F3F4F829FB001839F700D929F0D
:10156000700D112446275150319657FFF0CF40930C
:10157000F70180914104882321F40E949D89809382
:1015800041048091F701833459F088E190E029E229
:101590000FB6F894A895809360000FBE209360006A
:1015A0008CEF96E8909355048093540484EF9FE069
:1015B0009F938F9303EB14E11F930F93E0915404D7
:1015C000F091550409950F900F900F900F9081E6C0
:1015D00090E09F938F9384E590E09F938F931F9269
:1015E0001F92809102016AE00E94708D892F9927D5
:1015F0009F938F93809102010E94708D99279F93F2
:101600008F938AE190E19F938F931F930F93E091C3
:101610005404F0915504099582EF9EE09F938F93B7
:101620001F930F93E0915404F091550409958AECAF
:101630009EE09F938F931F930F93E0915404F0913A
:10164000550409958DB79EB746968DBF8EE490E1FF
:101650009F938F931F930F93E0915404F09155043F
:10166000099583EC8093810080916F008062809364
:101670006F000F900F900F900F901F910F91089592
:1016800080914204882361F08091F801843011F444
:101690000E94FE858091F701833411F0109242047C
:1016A00008951F920F920FB60F9211242F933F931C
:1016B0004F935F936F937F938F939F93AF93BF935A
:1016C000EF93FF932091CE00809108028823B1F020
:1016D0002093C60080910802823029F52F3F19F52A
:1016E0008FEF94E3ACE0B0E0C297A109B109B7FF76
:1016F000FBCF80919A048093CE0015C09091F801A1
:10170000892F8150833020F4822F0E94EB6C0BC014
:10171000943021F4822F0E94F18505C0953019F490
:10172000822F0E943085FF91EF91BF91AF919F91E1
:101730008F917F916F915F914F913F912F910F907A
:101740000FBE0F901F901895FB01DC0102C00590A1
:101750000D9241505040D8F70895FC01415050403F
:1017600030F001900616D1F73197CF010895882700
:1017700099270895A0E0B0E0E0ECFBE80C94E88D38
:101780006C017B01EA01590121978FEFCF3FD80708
:1017900089F086010894C11CD11CC7010894E11C82
:1017A000F11CF5010995F80180832197FFEFCF3FE8
:1017B000DF0779F7EAE0CDB7DEB70C94048ECF925D
:1017C000DF92EF92FF920F931F937C016B01FB015D
:1017D0000995082FC7010196F6010995182FC80130
:1017E0001F910F91FF90EF90DF90CF900895A0E0B0
:1017F000B0E0EDEFFBE80C94EA8D8C017B01EA018F
:10180000690121978FEFCF3FD80771F0F701219140
:101810007F01C8010F5F1F4F622FF60109952197C5
:10182000FFEFCF3FDF0791F7E8E0CDB7DEB70C94CD
:10183000068ECF92DF92EF92FF920F931F936C016F
:101840008B017A01FA010995812F9927682FC6012A
:101850000196F70109951F910F91FF90EF90DF908E
:10186000CF9008955058BB27AA270ED0E0C0D1D002
:1018700030F0D6D020F031F49F3F11F41EF4C6C0F2
:101880000EF4E095E7FBBCC0E92FE2D080F3BA1775
:10189000620773078407950718F071F49EF5FAC084
:1018A0000EF4E0950B2EBA2FA02D0B01B90190017B
:1018B0000C01CA01A0011124FF27591B99F0593FBF
:1018C00050F4503E68F11A16F040A22F232F342F07
:1018D0004427585FF3CF469537952795A795F04055
:1018E0005395C9F77EF41F16BA0B620B730B840B6A
:1018F000BAF09150A1F0FF0FBB1F661F771F881F22
:10190000C2F70EC0BA0F621F731F841F48F4879579
:1019100077956795B795F7959E3F08F0B3CF939568
:10192000880F08F09927EE0F97958795089598D01E
:1019300088F09F5790F0B92F9927B751A0F0D1F0B8
:10194000660F771F881F991F1AF0BA95C9F712C042
:10195000B13081F09FD0B1E008959CC0672F782FFF
:101960008827B85F39F0B93FCCF3869577956795AE
:10197000B395D9F73EF490958095709561957F4F1A
:101980008F4F9F4F0895E89409C097FB3EF49095C0
:101990008095709561957F4F8F4F9F4F9923A9F048
:1019A000F92F96E9BB279395F695879577956795D7
:1019B000B795F111F8CFFAF4BB0F11F460FF1BC01B
:1019C0006F5F7F4F8F4F9F4F16C0882311F096E9AE
:1019D00011C0772321F09EE8872F762F05C066235C
:1019E00071F096E8862F70E060E02AF09A95660F15
:1019F000771F881FDAF7880F9695879597F90895CE
:101A000097F99F6780E870E060E008959FEF80ECB1
:101A1000089500240A941616170618060906089554
:101A200000240A9412161306140605060895092EBA
:101A30000394000C11F4882352F0BB0F40F4BF2B29
:101A400011F460FF04C06F5F7F4F8F4F9F4F089569
:101A500057FD9058440F551F59F05F3F71F047955F
:101A6000880F97FB991F61F09F3F79F08795089544
:101A7000121613061406551FF2CF4695F1DF08C063
:101A8000161617061806991FF1CF86957105610580
:101A900008940895E894BB2766277727CB0197F928
:101AA0000895629FD001739FF001829FE00DF11DA8
:101AB000649FE00DF11D929FF00D839FF00D749FC8
:101AC000F00D659FF00D9927729FB00DE11DF91F74
:101AD000639FB00DE11DF91FBD01CF0111240895D1
:101AE000991B79E004C0991F961708F0961B881F70
:101AF0007A95C9F780950895AA1BBB1B51E107C0D1
:101B0000AA1FBB1FA617B70710F0A61BB70B881F8D
:101B1000991F5A95A9F780959095BC01CD0108951C
:101B200097FB092E07260AD077FD04D0E5DF06D003
:101B300000201AF4709561957F4F0895F6F79095FF
:101B400081959F4F0895A1E21A2EAA1BBB1BFD0190
:101B50000DC0AA1FBB1FEE1FFF1FA217B307E4078C
:101B6000F50720F0A21BB30BE40BF50B661F771FE4
:101B7000881F991F1A9469F76095709580959095C4
:101B80009B01AC01BD01CF01089597FB092E0526ED
:101B90000ED057FD04D0D7DF0AD0001C38F4509582
:101BA0004095309521953F4F4F4F5F4F0895F6F781
:101BB00090958095709561957F4F8F4F9F4F0895B9
:101BC0002F923F924F925F926F927F928F929F924D
:101BD000AF92BF92CF92DF92EF92FF920F931F933B
:101BE000CF93DF93CDB7DEB7CA1BDB0B0FB6F894EC
:101BF000DEBF0FBECDBF09942A88398848885F842C
:101C00006E847D848C849B84AA84B984C884DF809C
